:020000040800F2
:100000000080002039A20008F5820008FB82000869
:1000100001830008078300080D830008000000002A
:100020000000000000000000000000001383000832
:100030001F830008000000002B830008378300089E
:1000400089A2000889A200084583000889A2000847
:1000500089A2000889A20008598300086783000864
:1000600089A2000889A2000889A2000889A20008C4
:1000700089A2000889A2000889A2000881830008DB
:1000800089A2000889A2000889A2000889A20008A4
:100090000000000089A200087383000889A20008FC
:1000A00089A2000889A2000889A2000889A2000884
:1000B00089A2000889A2000889A2000889A2000874
:1000C00089A2000889A2000889A2000889A2000864
:1000D0009583000889A2000889A2000889A2000867
:1000E00089A2000889A20008A983000889A2000843
:1000F00089A20008000000000000000089A200089A
:1001000089A2000889A20008BD83000889A200080E
:1001100089A2000889A2000889A2000889A2000813
:1001200089A2000889A2000889A2000889A2000803
:0801300089A2000889A2000861
:1001400010B5054C237833B9044B13B10448AFF311
:1001500000800123237010BDC803002000000000B0
:1001600054F8020808B5034B1BB103490348AFF329
:10017000008008BD00000000CC03002054F80208F5
:1001800008B50146024800F053FA002008BD00BF40
:10019000C84F002008B5024800F056FA002008BDFC
:1001A000C84F00200146014800F050BAC84F002057
:1001B00030B585B00D460DF10F040146019204489B
:1001C00000942A4600F0E4FC9DF90F0005B030BD14
:1001D000C84F002030B585B00D460DF10F04014623
:1001E0000192044800942A4600F070F89DF90F002F
:1001F00005B030BDC84F002030B583B00D46144661
:10020000014600932A462346024800F01BFC03B037
:1002100030BD00BFC84F002030B583B00D46144636
:10022000014600932A462346024800F05FFC03B0D3
:1002300030BD00BFC84F0020F0B587B08C460C9E83
:10024000009317460DF1130405ADCDE902450146B3
:100250003B460648019662460D9C00F033F9059B2B
:100260009DF91300236007B0F0BD00BFC84F002008
:10027000F0B587B08C460C9E009317460DF1130421
:1002800005ADCDE9024501463B460648019662466A
:100290000D9C00F07FF9059B9DF91300236007B0CA
:1002A000F0BD00BFC84F002030B585B00D460DF140
:1002B0000F0101922B4602460091034800F0CCF951
:1002C0009DF90F0005B030BDC84F00202DE9F04F5B
:1002D0008BB01D46149C0293002323702C7804914C
:1002E000054691467CB1159A184602EB0414114656
:1002F00000260022002348738E6008738873E1E8AB
:100300000423A142F7D1B9F1000F5BD0DDF81080D2
:10031000CDF814800027BA4698F80D30654A5E1E65
:10032000F6B20121172E42FA06F201FA06F100F2A6
:100330009280614812F00102034400F0958011EAB6
:100340000A0F4AEA010A40F0998013F801BCD8F874
:100350000830039305EB8B041846D4F8A41305F07A
:100360008DFE039B014601371846002940F081802D
:10037000D4F8C41305F0A0FE05EBCB0B002878D110
:10038000D8E90001DBE98423994208BF904208F1D3
:10039000100803D1149B4FF004021A704F45BBD1D3
:1003A000049B059C8DF81B60102111FB0737A36887
:1003B000617B0093D4E900232846103401F0D6FF76
:1003C000A742F4D1284601F0C1FB029B1E78002E03
:1003D00059D00024394FDFF8E8A026464FF6FF79C0
:1003E00002E00134152C29D047FA04F3DB07F8D5D5
:1003F00014F80A3003F2AB134FF0010835F813304C
:100400004B4508FA04F224D0D5F834331A4204F1EB
:100410000104E7D00DF11B035FFA84FB009307AAE8
:1004200008AB5946284601F0ABFE029B1B78B3424D
:1004300006F101022BD8149A032313700023C5F888
:100440003433284600F0E8FD029B1E700BB0BDE877
:10045000F08F4444C6E7149AFF231370029B0026D2
:100460001E700BB0BDE8F08F1646149AFF23137070
:10047000EAE7149AFE2313700026E5E7149AFA239C
:1004800013700026E0E7149A02231370D6E7D6B261
:100490001598DDE90823711E00EB0111C1E9002365
:1004A000079A9DF81B3081F80DB081F80C808A60A6
:1004B0008B7397E70F20E000643A0308EF7912008E
:1004C0004C3A03082DE9F04F85B0DDE9108A1D464E
:1004D000DF2388F8003000241023172DCAF80040CD
:1004E00003932AD91746002934D106460C4688F8CA
:1004F00000108B4640F2173901E00A2C20D049FA4F
:1005000004F3DB0704F10104F7D5DDE90E23CDF890
:1005100000B0E1B2304601F0DBFD0028EDD00F9BCA
:1005200001930E9B009303AA03462946384600F028
:1005300051FD88F800000028DFD005B0BDE8F08F3D
:1005400098F90030002BF8D1DDE90E12304600F0AA
:10055000CBFE78B998F90040002CEED1039BCAF885
:1005600000303846514600F069FE88F8004005B07A
:10057000BDE8F08F0F9B01930E9B00932946034625
:1005800003AA384600F026FD044688F80000002C37
:10059000D3D1E3E72DE9F04F85B0DDE9108A1D46A0
:1005A000DF2388F8003000241023182DCAF80040FB
:1005B000039329D9174651BB06460C4688F800100C
:1005C0008B4640F2173901E00A2C20D049FA04F397
:1005D000DB0704F10104F7D5DDE90E23CDF800B007
:1005E000E1B2304601F0A0FD0028EDD00F9B019351
:1005F0000E9B009303AA03462946384600F0EAFC06
:1006000088F800000028DFD005B0BDE8F08F98F929
:100610000040002CF8D1039BCAF800303846514600
:1006200000F00CFE88F8004005B0BDE8F08F00BF78
:1006300010B404200124092202230C70487010BC5D
:100640008A70CB70704700BF00F048BC08B500F05E
:1006500017FF002008BD00BF2DE9F04F8DB000212D
:10066000179D169E2961C5E902112975044631704E
:100670001F46B0F8AEA4164600F0CEFCD4E9E4BCA8
:100680005BEA0C0342D0B6EB0B089A4B9A494FF049
:1006900000024FF0000067EB0C092CF081FDB4F86C
:1006A000ACB402460B464FF0000CCDE90823CDE96F
:1006B00006BC04F0E5FB05F0B7FDDDE906BC0B4622
:1006C000A0FB0B0103FB0B11B0EB0803029361EBE2
:1006D00009030393DDE902234FEA101B4BEA017B78
:1006E0004FEA211C93457CEB0303C0F27181B8EB08
:1006F0000003049369EB01030593DDE904239345AB
:100700007CEB030302DA169A6423137000230020A3
:1007100000210DF12E08C5E90001C5E902332B6166
:100720002B752A460DF12D03CDF8008001212046BE
:1007300000F078FC9DF82D30BDF82E902BB194F888
:10074000F9346B7494F8F734AB740DF12D032A4629
:10075000CDF800800221204600F064FCBDF82E3068
:100760009DF82D20994528BF99462AB194F8F83470
:10077000EB7494F8F734AB740DF12D032A46CDF8E1
:1007800000800321204600F04DFCBDF82E309DF87E
:100790002D20994528BF994692B1584B94F8F724DB
:1007A0005B7BAA7403F2A3134FF6FF7234F8133085
:1007B000ADF82E30934203D0AB6843F40053AB60E6
:1007C0000DF12D032A46CDF800800421204600F0CB
:1007D00029FCBDF82E309DF82D204B4528BF4B46F7
:1007E0009A4528BF9A460AB301232B7494F8F684DD
:1007F000424B04EB48085B7DB8F8C024AA8194F80A
:10080000F824EA7494F8F724AA74B133002154F858
:10081000230005F029FC002878D094F8FB34002B45
:1008200074D1B8F8B834EB81C4E9E667B4F8F434AD
:10083000B3FBFAF20AFB1232AAEB020A1FFA8AFA97
:10084000B4F8B0C4C4F8906353449BB2B3FBFCF259
:100850000CFB1233C4F894730022A4F8F434264934
:10086000244BA4F8ACA40020ADF82EC02CF098FCCA
:1008700004F006FB05F0D8FCA0FB0A8901FB0A99ED
:10088000D4E9E60118EB060649EB07070023301A06
:1008900067EB0101C5E9006784F8FB3405F012FA43
:1008A000174905F001FB1749054605F0E7FB28B19C
:1008B000652384F8FC340DB0BDE8F08F124928465A
:1008C00005F0FAFB0028F3D1D4E9E801301A67EB10
:1008D000010105F0F7F90A4905F0E6FA094905F0C2
:1008E000CDFB002800F09880662384F8FC340DB01E
:1008F000BDE8F08F00001C4000002440643A03086B
:10090000286B6E4E0000704200007043D4E9E8236B
:10091000D4E9E601824273EB010CBCBF02460B46F0
:10092000B01A67EB030105F0CDF93E4905F0BCFABA
:100930004FF0814180462CF011FD3B4981464046F5
:100940002CF00CFD39498346484605F0F9F9384941
:100950008146584605F0F4F90146484605F0E8F8A6
:1009600041468146404605F0EBF9324905F0E8F989
:100970000146484605F0DCF82F498146404605F01F
:10098000DFF90146484605F0D3F82C4905F0D0F8C8
:100990002B4905F0D5F92CF0A3FB05F0BDFB94F82D
:1009A000FB34E8817BB34FF07E53009332463B46E5
:1009B0001621204601F0DAFCAB6843F40013AB606B
:1009C00094F8FB34002B3FF42FAFC4E9E8672DE720
:1009D000DDE90801D4E9E498B4F8AC6404F050FA15
:1009E00005F022FC0B46A0FB060103FB061110EBF1
:1009F000090341EB0802C5E90032169B6421197016
:100A00000DB0BDE8F08F0023009332463B4616211F
:100A1000204601F0ABFCD3E784F8FC040DB0BDE840
:100A2000F08F00BF286B6E4E00004040598207B027
:100A3000DFE0C2343767D9B85A8E863C6A92E43E0A
:100A400000007A442DE9F04F8BB00546DDF8509058
:100A50008846002000210DF11E0B0DF1200AC5E98A
:100A6000E401164611461C4640465B464A46CDF810
:100A700000A000F059FE9DF91E3013BB0DF11F03BD
:100A8000083E0593089FB7424B46224651464046D2
:100A900025D209AF0297059FCDE900B700F096FC7B
:100AA0009DF91E30224628465BB99DF81F10FE298D
:100AB0000BD0099B01F01EF803468DF81E00002B99
:100AC000E0D018460BB0BDE8F08F099A214600F03F
:100AD000ADFE03468DF81E00002BD3D0F1E79DF943
:100AE0001E3018460BB0BDE8F08F00BF2DE9F04F67
:100AF0008BB00F46DDF850900DF11E0B0DF1200A62
:100B00001146154680461C4638465B464A46CDF897
:100B100000A000F009FE9DF91E3013BB0DF11F036C
:100B2000083D0593089EAE424B4622465146384644
:100B300025D209AE0296059ECDE900B600F046FC2E
:100B40009DF91E30224640465BB99DF81F10FE29D4
:100B50000BD0099B01F0DEFB03468DF81E00002B35
:100B6000E0D018460BB0BDE8F08F0999204600F0A0
:100B7000FFFE03468DF81E00002BD3D0F1E79DF950
:100B80001E3018460BB0BDE8F08F00BF000000001B
:100B90002DE9F04F8DB04FF00008169D03931646D7
:100BA00083460C4685F8008000F2CA411C2205A845
:100BB00027F0F0FC56BB0C232B7005A9584600F01B
:100BC0005BFA002840F0238195F9000000284CDBF7
:100BD000B54EB64F002303E05C1C152C234644D0D1
:100BE00046FA03F2D207F7D5DA5D0CA901EB420011
:100BF0000BEB420130F81E2CB1F8C8145C1C91427A
:100C00005846E1B2E9D000F021FCE6E723795F1E07
:100C1000FBB2012B40F2E5804FF0000804EBC60A5E
:100C20004FF00009CDF800B011E09F4A1A41D107FA
:100C300010D5012202FA03F313EA090B00F08B80AE
:100C4000F3232B700834544509D023795F1EFBB27F
:100C5000142BEAD908340A2354452B70F5D195F9A1
:100C60000030DDF800B0002BA7DA039B1B78072BC0
:100C70000AD8F1232B7000230193039B1A46019B92
:100C800013700DB0BDE8F08F0025DFF82C92864E72
:100C9000DFF830A20195CDF800B002E00135182D43
:100CA000EBD0012303FA05F4814B1C42F6D0019BE3
:100CB000179A0133DBB20193013B02EBC307013505
:100CC0003D714FF0000842F83390029516E018F895
:100CD0000330009A02EB4303B3F8C8044FF6FF73E6
:100CE000984206D004F0D8FF0146724805F0DCF8BF
:100CF000386008F10108B8F1150F2AD046FA08F358
:100D0000DB07F6D55AF828301C424946F1D0D7F80F
:100D100000B0584605F0A8F9644B0028D7D118F860
:100D20000320009B03EB4202B2F8C80404F0B4FFB6
:100D30000146604805F0B8F805462946584605F0D2
:100D40009DF90028D5D008F10108B8F1150F3D60D4
:100D5000D4D1029DA3E726684146304649EA0309FB
:100D600005F082F940B3F6232B70266841463046E1
:100D700005F07AF93746F8B14146384605F09CF956
:100D8000002846D13846414605F06EF9B0FA80F3A6
:100D90005B095B429EB295F90030002B7FF452AFA5
:100DA000424B1A46237913440CAA13F8013C02EB78
:100DB000430323F81E6C45E73F49304605F054F9DC
:100DC00000285FD13D49304605F076F928B93C4905
:100DD000304605F053F9002860D0F2232B702768C5
:100DE000CAE72068002105F03FF900283FF414AF5E
:100DF000BDF8142047F230539A4245D0BDF8162072
:100E00009A4241D00B23CDF804802B7035E728702F
:100E1000DCE62949384605F031F90028B2D03946D8
:100E2000244805F041F82CF05BF905F075F91F4BEB
:100E30001695009DCDF8049086B2994623794B44CF
:100E400013F8013C5B4403F2F3130BF10E0B35F87E
:100E50001370384604F0BAFA11A3D3E9002304F062
:100E60002FFB04F00DF804F0EDFD83B2FA1A1F44D5
:100E700093B2B342BFB227D8B74225D3DDF804906E
:100E8000169D88E737467DE79BF9FC34002B7FF4FD
:100E9000F1AE012201938BF8FB24EEE637466BE7B7
:100EA0007B14AE47E17A843FEF7912004C3A030895
:100EB0000F20E0000000C84200FF7F4700002041F3
:100EC0000E74DA3AF8390308BBF1540FB6D1169D07
:100ED000DDF80490F4232B70B4E600BF10B504468F
:100EE00000F09CFD204600F0F7FB204600F0E0FA01
:100EF000204610BD2DE9F0470646324D324F01F035
:100F0000DDF9002303E05C1C152C234610D045FAC4
:100F100003F2D107F7D5DA5D06EB42025C1CB2F8AA
:100F2000C824E1B2304601F07BFA152C2346EED1FD
:100F3000304601F047F9DFF88C90234FDFF89080BE
:100F4000002502E00135152D1AD049FA05F3DA071C
:100F5000F8D5EB5D334493F8E534002BF2D038F943
:100F600015A0002302E00A2C2346EBD04AFA03F234
:100F70005C1CD307F7D5E1B2304601F019FAF2E76D
:100F80000024214686F8FA440E2206F2E64027F0B5
:100F90000FFB0E4B86F8F644DB7803F2A3132146D1
:100FA00036F8130006F2B24333F8022B904201F1F7
:100FB000010103D00429F7D1BDE8F08786F8F614C3
:100FC000BDE8F087EF7912004C3A0308643A030851
:100FD000CC390308F0B41468049EE7188F4215D882
:100FE00005998B4215D8002B0CDD711ECD18C6F16A
:100FF000010600E014687318234411F8014FC4542B
:101000008D42F7D117600020F0BC70476FF02800C8
:10101000FAE76FF02500F7E790F8FA3403B9704764
:1010200068E700BF70B40139124D039C6D5C05F296
:10103000A315002630F815501E704FF6FF76B54206
:10104000258010D0B0F8F464B6FBF5F405FB146508
:10105000ADB255B990680124C9B204FA01F1014357
:101060001C701475916070BC704790F8FB040028E8
:10107000F9D0EFE7643A03082DE9F04F6A4C6B4E64
:1010800007460D4683B000236FF000414FF6FF7016
:1010900044FA03F2D20740F1B180F25C0A4435F819
:1010A0001220B2F5E16F00F0A980824200F0A68024
:1010B000B7F8AE445C482146002340FA03F2D20759
:1010C00006D5F25C013A35F81220914228BF11464C
:1010D0000133152BF1D14FF6FF7291421FD0B4FBB3
:1010E000F1F301FB13439BB28BB94F4C944644FA86
:1010F00003F2D20710D5F25C013A35F812006045D0
:101100000AD0B0FBF1F201FB120292B222B16FF0F1
:101110000F0003B0BDE8F08F0133152BE7D14FF678
:10112000FF71434A404C8E46002352F8040B0007DF
:1011300044FA03FC02D51CF0010F64D10133152BD6
:10114000F3D14FF6FF7399426AD007F2B2430024FD
:1011500002E00134042C09D033F8022B8A42F8D182
:1011600007EB4404B4F8BA440434A4B22E4ADFF8BE
:10117000C4B0DFF8C4A001944FF0000842FA08F3AD
:10118000DB0732D516F80830013B35F81390484696
:1011900004F082FD97F8F9C497F8F834019A0446F0
:1011A00097F8F7044FEA4C0C40005FFA8CFCC0B291
:1011B0005B006044DBB20344134498B204F068FD62
:1011C000594604F0BDFD514604F06EFE014620462E
:1011D00004F054FF144A40B14FF6FF73994504D010
:1011E0006FF0110003B0BDE8F08F08F10108B8F10D
:1011F000150FC3D1002003B0BDE8F08F0133152BCC
:101200007FF446AFF6E7F05C013835F81000704522
:1012100094D0714506D0884290D06FF01000EAE774
:101220000424A3E7014689E7EF7912004C3A03084A
:10123000F83903080000C84200007A44F0B589B0CC
:1012400004460D46274B029302A903A8042227F067
:10125000A1F99DF80F309DF80C009DF80D109DF838
:101260000E20E37020706170A27004A906A83D26CC
:1012700000270822CDE9046727F08CF906A9201D74
:10128000082227F087F92B6802A9103B03A8042243
:10129000029327F07FF99DF80C009DF80D109DF842
:1012A0000E209DF80F302073A273E37361732968D9
:1012B000204601AA03F084FE2B689DF804009DF8E7
:1012C00005102344002218712B68234459712B68A0
:1012D00023449A7128680444E2712B6808332B6018
:1012E00009B0F0BD020904012DE9F047072484B0DC
:1012F00080461746FE200DEB04020D468DF8074090
:1013000003F0B0FD9DF80760039036B3012408F5A3
:10131000926A08F57A79E3B2013B062B0CD8DFE834
:1013200003F0362E463E4E110400B8F8AE0403AB6F
:101330003A46294601F082F9A64204F101030BD096
:101340001C46E8E703AB3A462946504601F0A4FCA8
:10135000A64204F10103F3D10398ADF80A0002227A
:101360000DF10A0102A827F015F99DF808209DF853
:10137000093003982A706B7004B0BDE8F08798F8C4
:10138000F80403AB3A46294601F016FAD4E798F878
:10139000F70403AB3A46294601F00EFACCE703AB5B
:1013A0003A46294608F2B24001F01EFCC4E798F81C
:1013B000F90403AB3A46294601F0FEF9BCE703AB5A
:1013C0003A462946484601F03BFCB5E72DE9F04F87
:1013D00083B0DDE90CA900248AF8004089F80040B8
:1013E0000D460968064608449046427816F801C042
:1013F0008DF8052001A902220DF106009B468DF80B
:1014000004C027F0C7F8BDF806700E9B5F451F604B
:1014100005D9E0238AF8003003B0BDE8F08F57B15A
:10142000234608F1FF312A68F0180133825C01F885
:10143000012F9F42F7D198F8023089F800302B68CD
:101440003B442B6003B0BDE8F08F00BF0B4B0B4457
:1014500010B413F8013C00EB4301B1F8C8449442C6
:1014600004D0013B0344012483F8E6440123A1F89E
:10147000C82410BC80F8FA34704700BF4C3A030807
:101480000139032900D9704710B50446703002F0C5
:10149000B5FA2046012101F011F8044BA366E3667A
:1014A00020460221BDE8104001F008B80000484283
:1014B0002DE9F04140F201530546022280F8F7245D
:1014C000A0F8F8341822724900F2B24005F2E6346E
:1014D00027F060F805F28E4623464FF6FF7223F898
:1014E000022FB342FBD1DFF8D4C16A4B6A4F6B487D
:1014F000DFF8CCE1DFF8CC81694AC5F87CE440F242
:10150000DC51A5F880144FF06411C5E9FACCC5F898
:1015100000C4C5F80CC4C5F8F8C3C5F85834C5F8FC
:101520005C34C5F86034C5F86434C5F86834C5F86F
:101530007034C5F80414C5F80814C5F81414C5F8B7
:101540001C14C5F8F013C5F81084C5F82074C5F84C
:101550002474C5F82874C5F82C74C5F83074C5F81F
:101560003874C5F83C04C5F84004C5F84404C5F80F
:101570004804C5F84C04C5F85404C5F8F423C5F86C
:10158000FC1340224749C5F888E4C5F818C4C5F8DB
:101590003474C5F85004C5F86C3405F56A7026F04B
:1015A000F9FF4149DFF82081DFF820E1DFF820C1B1
:1015B0003E4F3F48C5F8B01300234FF080423D49ED
:1015C000C5F8AC33C5F8A833C5F8BC33C5F8C0338B
:1015D000C5F8C433C5F8DC23C5F8E023C5F8E41327
:1015E000C5F8B483C5F8D0E3C5F8CCC3C5F8C87353
:1015F000C5F8D403334605F2AA414FF6FF7223F82B
:10160000022F8B42FBD147F230520023A5F8AE24C3
:10161000A5F8B0344FF6FF7134F8023F8B4205D085
:10162000B5F8B0249A4238BFA5F8B034B442F3D12B
:10163000214CDFF8A0C00023012744FA03F2D207AF
:1016400011D513F80C2005EB4201013AB1F88E04D4
:10165000B1F8C86486421CBF521982F8E674A1F83A
:10166000C80485F8FA740133152BE6D105F2E54379
:1016700005F2F341012203F8012F8B42FBD195F8CB
:10168000FA340BB9BDE8F0812846BDE8F04131E4F9
:1016900048390308701770172C012C010807080738
:1016A0006400307560390308000020C20024F4494A
:1016B0000050434B00001041EF7912003075307537
:1016C000DC05DC053075640000002A430000AA42F6
:1016D0000000C8424C3A030800220023C0E9E4237A
:1016E000C0E9E623C0E9E823002147F2305330B4D3
:1016F000A0F8AC3480F8F614A0F8F41400F599635F
:1017000000F2E54200F2E4454FF6FF7423F8024F81
:10171000AB4202F8011FF9D1662330BCA0F8FA14DD
:1017200080F8FC34704700BFF0B589B00C460E9DC0
:101730000021172C1E46296003D8DB23337009B023
:10174000F0BD944203D9DA23337009B0F0BD0746E7
:1017500002A93A787B788DF80820BA788DF809309C
:101760008DF80A20FB788DF80B30042203A826F0B0
:1017700011FF039B2C4A934204D0013302D0DE2395
:101780003370DCE70822391D06A826F003FF082283
:1017900006A904A826F0FEFEDDE90423002B08BFFD
:1017A0003D2A07D0002B08BFB2F1FF3F02D0DD2356
:1017B0003370C4E73A7B7B7B8DF80820BA7B8DF8C9
:1017C000093002A9FB7B8DF80A2003A804228DF8BA
:1017D0000B3026F0DFFE039901F11803A34202D07B
:1017E000D8233370ABE701AA3846103103F0E8FB89
:1017F00038199DF8042010F8043C9A4202D0DC23EA
:1018000033709CE79DF8052010F8033C9A42F6D10E
:1018100010F8023C002BF2D110F8013C002BEED165
:1018200010222A6033708AE7020904012DE9F0478B
:1018300086B004AB05AECDE9003604460DF10F03CA
:10184000FE200D4603F0E0FA9DF90F0000285CD160
:101850004FF0010A04F5926904F57A7804F2B24770
:101860005FFA8AF3013B052B77D8DFE803F06B645E
:101870005D5751034A463146284601F061F80AF1A6
:10188000010ABAF1080FEBD10023A4F8B03404F236
:101890008E4504F2E6334FF6FF7033F8022F824292
:1018A00005D0B4F8B014914238BFA4F8B0249D42DA
:1018B000F3D12D4DDFF8B4C00023012745FA03F220
:1018C000D20711D513F80C2004EB4201013AB1F80C
:1018D0008E04B1F8C86486421CBF121982F8E674FF
:1018E000A1F8C80484F8FA740133152BE6D104F288
:1018F000E54304F2F341012203F8012F8B42FBD1AF
:1019000094F8FA342BBB9DF90F0006B0BDE8F087C0
:1019100042463146284600F0CDFFB0E73A46314610
:10192000284600F0A1FFAAE73146284600F02EFF26
:1019300084F8F904A3E73146284600F027FF84F82D
:10194000F8049CE73146284600F020FF84F8F704AD
:1019500095E72046FFF7CEFAD5E73146284600F056
:1019600055FEA4F8AE048AE7EF7912004C3A03085A
:10197000032916D910B582B0027843788DF8042077
:101980000446022201A90DF106008DF8053026F06B
:1019900001FEA378FE2B0CBF00206FF0630002B0A5
:1019A00010BD6FF067007047194B013970B45B5C74
:1019B00000EB43034FF6FF72B3F83A43944206D06C
:1019C000144CD0F8382334F91140944302D000204D
:1019D00070BC7047104CD0F820536456AC43F6D11D
:1019E000B3F87E53B3F872636C1CA5B2B5FBF6F482
:1019F00006FB1454A4B2A3F87E43002CE7D10123C4
:101A000003FA01F11143C0F838131846E0E700BFAC
:101A1000C0390308A0390308B4390308F8B50446EF
:101A200002F0F4F804F5E47002F0D2FF04F12C00A7
:101A300002F054FB04F1700001F0CCFA04F5B07030
:101A400002F0FEFD0A2104F5007002F01FFA0026E4
:101A500004F5327304F5067204F53A75002000218E
:101A600043F8046BAB42E2E80201F9D100204FF0E9
:101A7000000CC4F8200304F5397304F5147104F262
:101A8000233204F547750026002743F804CFAB4204
:101A9000E1E9026702F8010FF7D1C4E9CD0004F5CE
:101AA0004F7304F55275012000214FF6FF7218871D
:101AB000A3F8441023F8022B9D42F8D1A4F8482340
:101AC000A4F84A23A4F84C23A4F84E23A4F85023E6
:101AD000A4F85223A4F85423A4F8562304F256334E
:101AE00004F272314FF6FF7223F8022F8B42FBD1C2
:101AF0002046F8BD10B44C1E11461A46092C06D8D3
:101B0000DFE804F0090D110514050505191E6FF035
:101B1000630010BC704710BC703001F001BB10BCFA
:101B20002C3002F037BD10BC02F07CB810BC00F5C0
:101B3000E47002F067BF10BC00F5B07002F0C8BDE1
:101B400010BC00F5007002F0ADB900BF2DE9F04700
:101B500000239EB00025C0F83833052104468DF8D7
:101B600021308DF822308DF8233009950A950B9598
:101B7000189519951A951B951C951D950C950D9505
:101B8000FFF712FF002800F09280D4F8E402294603
:101B900004F06AFA002840F0208103212046DFF893
:101BA0002CA54FF0FF366FF00047FFF7FDFE002831
:101BB00040F08A8001212046FFF7F6FE38B1D4F8C4
:101BC000E402002104F050FA002840F05B81022179
:101BD0002046FFF7E9FE38B1D4F8E402002104F012
:101BE00043FA002840F0898109212046FFF7DCFEF6
:101BF00038B1D4F8E402002104F036FA002840F0AD
:101C0000108200250A212046FFF7CEFE38B1D4F815
:101C1000E402002104F028FA002840F02F829AF80C
:101C2000053003F2AB114FF6FF7234F811109142F8
:101C300003F1FF3504D0D4F82023560700F1B28019
:101C40009AF8063003F2AB114FF6FF7234F8111018
:101C5000914203F1FF3504D0D4F82023D00700F1DE
:101C600086809AF8073003F2AB114FF6FF7234F812
:101C70001110914203F1FF3503D0D4F820239107CE
:101C80005AD49AF8083003F2AB114FF6FF7234F8C9
:101C90001110914203F1FF3503D0D4F8202312072D
:101CA0002AD40023C4F820331EB0BDE8F087DFF843
:101CB0001CA44FF0FF366FF0004703212046FFF7CA
:101CC00073FE00283FF476AFD4F8E402002104F05C
:101CD000CBF900283FF46EAF0BA90AAACDE9012188
:101CE00009AB0093D4F8CC32D4F8D022D4F8D41273
:101CF000204601F0B3FF5DE7D4E98C6703F1B90238
:101D0000D4F8D41244F8221004EBC303C3E9946757
:101D100000202BF0E5F904F0FFF9254485F82403B1
:101D2000D4F8343343F48073C4F834330023C4F854
:101D300020331EB0BDE8F087D4E9886703F1B9020B
:101D4000D4F8CC1244F8221004EBC303C3E994671F
:101D500000202BF0C5F904F0DFF9254485F82403B1
:101D6000D4F8343343F08003C4F8343389E7D4E93A
:101D7000866703F1B902D4F8C81244F8221004EBC4
:101D8000C303C3E9946700202BF0AAF904F0C4F957
:101D9000254485F82403D4F8343343F04003C4F8D1
:101DA00034335EE7D4E98A6703F1B902D4F8D0127C
:101DB00044F8221004EBC303C3E9946700202BF01E
:101DC0008FF904F0A9F9254485F82403D4F83433B5
:101DD00043F02003C4F8343332E7D4E98C670DF1C3
:101DE00023010DF1340CDFF8E4A203910DF1220080
:101DF0000DF12101CDE90010CDF808C032463B4677
:101E000004F5E47002F026FE9AF80B809DF821009C
:101E100003F03EFF08F1B90904EBC80344F82900B8
:101E2000C3E9946728462BF05BF904F075F908F1D3
:101E3000FF38A04488F82403D4F834339DF82200F6
:101E40009AF80C8043F40063C4F8343303F020FFA5
:101E500008F1B90904EBC803024644F829202846D2
:101E6000C3E994672BF03CF904F056F908F1FF3808
:101E7000A04488F82403D4F8343343F48053C4F8DE
:101E800034331AE7D4F8E032D4F8DC02049318AA09
:101E90000CAD0021CDE9052504F0E6F8B0FA80F597
:101EA0006D099DF822C003959DF821509DF82300EF
:101EB0000B9B0A9A09990290CDE9005C04F170002D
:101EC00001F088F99AF811300C9D03F1B90104EB87
:101ED000C30244F82150013BC2E994670020E51891
:101EE0002BF0FEF804F018F985F82403D4F8343305
:101EF00043F40033C4F8343369E616AD14A812A9CC
:101F000010AA0EABCDE90305CDE9012100930C9990
:101F10000D9B18AA04F12C0002F014F99AF8003075
:101F20000E9D0F9803F1B90104EBC30244F8215050
:101F3000013BC2E99467E5182BF0D2F804F0ECF805
:101F400085F82403D4F834239AF80130109D1198B1
:101F500003F1B90142F00102C4F8342304EBC302D7
:101F600044F82150013BC2E99467E5182BF0B8F81A
:101F700004F0D2F885F82403D4F834239AF8023018
:101F8000129D139803F1B90142F00202C4F8342300
:101F900004EBC30244F82150013BC2E99467E51801
:101FA0002BF09EF804F0B8F885F82403D4F8342315
:101FB0009AF80330149D159803F1B90142F0040218
:101FC000C4F8342304EBC30244F82150013BC2E9B6
:101FD0009467E5182BF084F804F09EF885F8240344
:101FE000D4F834239AF81430169D179803F1B901E8
:101FF00042F00802C4F8342304EBC30244F8215031
:10200000013BC2E99467E5182BF06AF804F084F804
:1020100085F82403D4F8343343F48013C4F83433FC
:10202000E2E5D4E98A89D4F8D832B4F87210029182
:10203000CDE9008903933246D4F8D0123B4604F52B
:10204000B07002F08FFB9AF80D3003F1B90104EB88
:10205000C3020546013B44F821500020C2E994899F
:10206000E6182BF03DF804F057F886F82403D4F86E
:10207000343343F40053C4F83433C3E52A46D4F868
:10208000CC32D4F8D01204F50070D4E98A6701F09C
:1020900025FF9AF80E3003F1B905024604EBC3019F
:1020A00044F82520013BC1E994670020E518099216
:1020B0002BF016F804F030F885F82403D4F8343304
:1020C00043F48043C4F83433A9E500BF4C3A030815
:1020D00010B44C1E11461A469DF80430092C06D83F
:1020E000DFE804F0080C100513050505181D002095
:1020F00010BC704710BC703001F06CBB10BC2C30B1
:1021000002F01CB910BC01F0FFBD10BC00F5E4707A
:1021100002F034BD10BC00F5B07002F0A9BB10BCD9
:1021200000F5007001F01ABF10B44C1E11461A469B
:102130009DF80430092C06D8DFE804F0080C1005DF
:1021400013050505181D002010BC704710BC703029
:1021500001F0B2BB10BC2C3002F064B910BC01F02D
:1021600005BE10BC00F5E47002F054BD10BC00F5D3
:10217000B07002F0DDBB10BC00F5007001F020BFB4
:10218000F0B401390E4C049D645C04F1B90C00EB11
:10219000C40750F82C601660D7E99467C3E900675C
:1021A0000444012294F823332B70D0F8343302FA1C
:1021B00001F123EA0103F0BCC0F83433704700BFDB
:1021C0004C3A03082DE9F04F8446374E374DDFF87F
:1021D000E8A083B0002140F217374FF6FF7E04E0FD
:1021E00001310A2906F101065BD047FA01F3DB074A
:1021F000F6D52F4B13F801800CEB4808B8F83A934A
:10220000F145EDD000231C460120019600FA03F2AF
:102210003A4210D0274E36F911B01BEA020F0AD00D
:10222000234AD25C0CEB4202B2F83A23724502D048
:10223000944238BF144601330A2BE7D1019E002394
:10224000012000FA03F22A420FD096F900B01BEAEF
:10225000020F0AD013F80A2002F2A3123CF812204F
:10226000724502D0944238BF14460133182BE8D18E
:10227000002CB5D0B9FBF4F204FB12991FFA89F3D4
:1022800092B23BB104F0010000EB5404A342A4BF9E
:10229000013292B201310A29A8F8722306F101062F
:1022A000A3D103B0BDE8F08FB43903080F20E000DC
:1022B000C0390308A0390308643A030830B400F5B4
:1022C0004F7300F55275012400214FF6FF721C87F1
:1022D000A3F8441023F8022B9D42F8D1A0F848231C
:1022E000A0F84A23A0F84C23A0F84E23A0F85023CE
:1022F000A0F85223A0F85423A0F8562300F2563336
:102300004FF6FF7200F2723023F8022F8342FBD1A6
:1023100030BC704710B44C1E11461A46092C06D822
:10232000DFE804F0090D110514050505191E6FF00D
:10233000630010BC704710BC703001F0E5BB10BCEE
:102340002C3002F0B3B810BC01F042BD10BC00F557
:10235000E47002F0FFBC10BC00F5B07002F01CBBD2
:1023600010BC00F5007001F05DBE00BFF0B5013992
:102370000E4C14F801C000EBCC0EDEE984459D4202
:1023800008BF944210D00CF1B10C16461F46059BB5
:1023900040F82C30CEE984670122D0F8203302FACD
:1023A00001F10B43C0F82033F0BD00BF643A0308CD
:1023B0004B1EDAB2092A00D97047184A114411F8A5
:1023C000012C00EB4202B2F83A13092BF4D801A217
:1023D00052F823F0052400080B24000811240008FB
:1023E000B923000815240008B9230008B923000800
:1023F000B9230008B9230008FD23000800F5007088
:1024000001F02CBE703001F019BB2C3002F070B816
:1024100001F0FABC00F5E47002F06ABCC0390308B0
:10242000204B0139F0B55B5C1F4FDFF888E003F209
:10243000AB13844620F813200126002340F2173501
:1024400006FA03F42C420DD037F91100204209D0CE
:102450001EF803000CEB4000B0F83A43944288BFEA
:10246000A0F83A2301330A2BEAD1104E1048DFF8C6
:1024700048E00023012505FA03F434420DD050F85A
:1024800021703C4209D01EF803400CEB4404B4F820
:102490004673974288BFA4F846230133182BEAD12C
:1024A000F0BD00BF4C3A0308CC3903080F20E00010
:1024B000F8390308C0390308643A03084B1E092B96
:1024C00010D8124A114411F8012C00EB4202B2F864
:1024D0003A13092B09D8DFE803F0090C0F0811089B
:1024E000080808154FF6FF71F3E77047703001F0E8
:1024F000A5BA2C3001F0FCBF01F086BC00F5E470F9
:1025000002F0F6BB00F5007001F0A8BDC039030869
:10251000F0B50F46096803464C1E00F10B0685B066
:10252000234410460E4401AC13F8015F04F8015B2C
:10253000B342F9D101A90C2226F02CF83B680C33E8
:102540003B6005B0F0BD00BFF0B51C461B680C3306
:10255000934285B003D90132226005B0F0BD0C2250
:102560000F46014601A826F015F801AB0022BD1860
:10257000206813F8016B2E5401320C2AF7D123681E
:102580000C33236005B0F0BDF0B50B6883B0044692
:102590001C440F4610460DF1FF330DF1070614F8E9
:1025A000015B03F8015FB342F9D10822694625F0C7
:1025B000F1FF3B6808333B6003B0F0BD70B51C46CB
:1025C0001B680833934284B003D90132226004B0FF
:1025D00070BD08220D460146684625F0DBFF082243
:1025E0000DEB0200694625F0D5FF0DF1070300222F
:1025F000A818216813F8016F46540132082AF7D150
:1026000023680833236004B070BD00BF10B50B68A9
:10261000C21882B00C465278C35C8DF8052001A91F
:1026200002220DF106008DF8043025F0B3FF236877
:10263000BDF806000233236002B010BD30B51C4661
:102640001B6885B002339342ADF8060003D901320E
:10265000226005B030BD0D4602220DF1060103A82F
:1026600025F098FF23689DF80C20EA5421689DF816
:102670000D3029444B7023680233236005B030BD10
:1026800030B50C460968451883B0034610466A7891
:102690005B5C8DF8052001A902228DF8043025F03D
:1026A00079FF23680233236003B030BD30B51C4688
:1026B0001B680233934283B003D90132226003B016
:1026C00030BD027843788DF800200D46022269461D
:1026D00001A88DF8013025F05DFF23689DF80420E6
:1026E000EA5421689DF8053029444B702368023371
:1026F000236003B030BD00BF30B50A6883B08318D3
:10270000825C8DF8042058789D788DF805000C4681
:102710000422DB788DF807300DEB020168468DF856
:10272000065025F037FF236800980433236003B078
:1027300030BD00BF30B51C461B6885B004339342E2
:10274000019003D90132226005B030BD04220D464C
:1027500003A80DEB020125F01DFF23689DF80C2056
:10276000EA5423689DF80D009DF80E109DF80F2087
:102770002B44587023682B44997021680D44EA70EB
:1027800023680433236005B030BD00BF10B50B686B
:1027900082B00C46C35C8DF8073001220DF10701B1
:1027A0000DF1060025F0F6FE23689DF806000133C2
:1027B000236002B010BD00BF30B51C461B6883B05B
:1027C0005D1C95428DF8070003D90132226003B0E9
:1027D00030BDC81801220DF1070125F0DBFE23688A
:1027E0000133236003B030BD30B50A6885B00D46B3
:1027F0000DF1070310440DF10F0410F8012B03F83D
:10280000012FA342F9D108220DEB0201684625F001
:10281000C1FE2B68DDE9000108332B6005B030BD37
:1028200070B584B0CDE90001089C266808369E4248
:1028300003D90133236004B070BD154608220DEBA7
:102840000200694625F0A6FE0DF107020023E818F4
:10285000216812F8016F46540133082BF7D1236821
:102860000833236004B070BDF0B50B6887B0044630
:10287000013B1C440F4610466B4606AE14F8015F40
:1028800003F8015BB342F9D16946182225F082FEB4
:102890003B6818333B6007B0F0BD00BF30B41C6824
:1028A000651C95429CBF08551A68013230BC1A60FD
:1028B000704700BFF0B50B68ABB00446013B1C4449
:1028C0000F4610466B462AAE14F8015F03F8015B11
:1028D000B342F9D16946A82225F05CFE3B68A833D3
:1028E0003B602BB0F0BD00BF70B51D461B681033B8
:1028F000934288B003D901322A6008B070BD10221B
:102900000DEB02040E460146684625F043FE69467B
:102910001022204625F03EFEC4F101000DF10F0209
:102920000DF11F012B6884181C4412F8013F335528
:102930008A42F7D12B6810332B6008B070BD00BFFE
:10294000F0B50B6889B00446013B1C440F461046A5
:1029500001AB08AE14F8015F03F8015BB342F9D193
:1029600001A91C2225F016FE3B681C333B6009B010
:10297000F0BD00BF30B51C461B680433934283B0E2
:1029800003D90132226003B030BD0288ADF80020C7
:1029900004220D464388ADF8023069460DEB020073
:1029A00025F0F8FD23689DF80420EA5423689DF87B
:1029B00005009DF806109DF807202B4458702368E9
:1029C0002B44997021680D44EA7023680433236016
:1029D00003B030BDF0B50B6885B00446013B1C4424
:1029E0000F4610466B4604AE14F8015F03F8015B16
:1029F000B342F9D16946102225F0CCFD3B68103373
:102A00003B6005B0F0BD00BF30B51C461B6802330B
:102A1000934283B003D90132226003B030BD027803
:102A200043788DF800200D460222694601A88DF8F2
:102A3000013025F0AFFD23689DF80420EA54216899
:102A40009DF8053029444B7023680233236003B09E
:102A500030BD00BF70B503460D6882B00C46411909
:102A600010465A5D8DF8042004224E788D78CB787C
:102A70008DF807300DEB02018DF805608DF80650DA
:102A800025F088FD23680433236002B070BD00BFC9
:102A900030B51C461B6883B05D1C95428DF807005D
:102AA00003D90132226003B030BDC81801220DF1F4
:102AB000070125F06FFD23680133236003B030BDAB
:102AC00030B50C460968451883B0034610466A784D
:102AD0005B5C8DF8052001A902228DF8043025F0F9
:102AE00059FD23680233236003B030BD70B51C4626
:102AF0001B680833934282B003D90132226002B0CE
:102B000070BD08220D460146684625F043FD0DF1D3
:102B1000FF330022A818216813F8016F46540132D0
:102B2000082AF7D123680833236002B070BD00BFC4
:102B300010B50B6882B00C46C35C8DF807300122DB
:102B40000DF107010DF1060025F024FD23689DF924
:102B500006000133236002B010BD00BF70B51D46F2
:102B60001B68143393428AB003D901322A600AB039
:102B700070BD14220DEB02040E460146684625F096
:102B800009FD69461422204625F004FDC4F1010325
:102B90000DF113020DF127012C689818204412F84A
:102BA000014F34548A42F7D12B6814332B600AB09A
:102BB00070BD00BFF0B50B6887B00446013B1C44F4
:102BC0000F46104601AB06AE14F8015F03F8015B37
:102BD000B342F9D101A9142225F0DCFC3B6814337F
:102BE0003B6007B0F0BD00BF70B51D461B681833D1
:102BF00093428CB003D901322A600CB070BD182208
:102C00000DEB02040E460146684625F0C3FC6946FA
:102C10001822204625F0BEFCC4F101030DF1170275
:102C20000DF12F012C689818204412F8014F3454EC
:102C30008A42F7D12B6818332B600CB070BD00BFEF
:102C400070B51D461B68A8339342D4B003D9013236
:102C50002A6054B070BDA8220DEB02040E46014656
:102C6000684625F097FC6946A822204625F092FC8C
:102C7000C4F101030DF1A7020DF24F112C68981851
:102C8000204412F8014F34548A42F7D12B68A833FC
:102C90002B6054B070BD00BF70B51D461B681C335F
:102CA000934288B003D901322A6008B070BD01ACEC
:102CB0001C220E460146204625F06CFCC4F101039F
:102CC0000DF103020DF11F012C689818204412F831
:102CD000014F34548A42F7D12B681C332B6008B063
:102CE00070BD00BFF8B500EB83040D46E768002116
:102CF0003846164603F0B8F9F8B16068314602F07C
:102D000015FF00212AF0AEF9E168034630461C4663
:102D100002F00CFF00212AF0A5F9014620462AF016
:102D2000B3F9014602F004FF294603F0BDF8BDE8FF
:102D3000F8404FF07E512AF0A7B96068394602F09A
:102D4000F5FE29462AF08EF90546D6E72DE9F04F23
:102D500085B005469DF83C40039440689DF840408E
:102D6000029488465F49019316461C4602F0E8FF2C
:102D70009DF838B08246002C5FD10BF1030355F863
:102D8000231002F0D5FE346807462146404602F083
:102D9000CDFE0446688802F07BFF534903F084F8B7
:102DA00005EB8B0903465149D9F81C00009303F049
:102DB0005BF9002867D14E49504602F0C1FF5146E9
:102DC00002F0B6FE00218046204603F075F9002887
:102DD00043D0BBF1010F09BF039BDFF824A10B33E4
:102DE00055F823A0029B33B94146204603F064F90D
:102DF00008B1DFF80CA168683E4902F0A1FF514616
:102E000003F052F8009902F09BFF05460146204668
:102E100003F052F9F8B93168204602F089FE3946CC
:102E2000044603F02BF900B92746019B0BB107F1CB
:102E30000047376005B0BDE8F08F34680BF101033F
:102E400004F10044346055F8231002F06FFE08F1DD
:102E50000048074699E72C46DDE7029B7BB3D9F88B
:102E6000D410009B03F1004003F01EF82AF000FA92
:102E700001464FF07E5002F059FE0146204602F016
:102E80005FFF0446C7E7D9F80400414602F04EFE52
:102E900000212AF0E7F801464FF07E5002F046FE8E
:102EA000014602F04DFF4FF07D5102F049FF1249FB
:102EB00002F046FF114902F03BFE01467CE7204646
:102EC0002AF08AF8414603F0F7F80028C7D0BBF192
:102ED000010FC4D10549D5F8D80002F0E5FF01463D
:102EE000BFE700BFC178C63D0000C84200004040B7
:102EF0009A99993ECBBECB3ECDCC4C3ECDCCCC3D71
:102F00000000E1442DE9F0479DF820C000EB8C075C
:102F100005460E46F8692B49904699460CF1FF3458
:102F200003F0A2F8002833D049464FF07E5002F05B
:102F3000FDFD014602F004FF4FF07D5102F000FF5D
:102F4000214902F0FDFE214902F0F2FD8146D7F849
:102F50000CA07868514602F0E9FD49460746304624
:102F600002F0EEFE314602F0E3FD0146384603F082
:102F700085F82C4428B95046002103F075F8034623
:102F800048B195F8E03023774FF07E50BDE8F087E8
:102F9000DFF83C90DBE7B8F1000F0CD1237FFF2B6B
:102FA0000ED00133DBB2237795F8E0209A4207D99F
:102FB0004FF08040EAE723774FF08040BDE8F0878C
:102FC0000048E3E700004040CDCC4C3ECDCCCC3DAA
:102FD0009A99993EF0B40A263E4A3F4D3F49A0F8DF
:102FE000E26003243E4EA0F8E440C0F8E8203D4CE7
:102FF0003D4AC0F8EC50C1633C4D3D4906643D4E2E
:1030000044648264012400228565C0F8981000257C
:103010004FF07E51C0F89C60374E04708262C264EB
:1030200002654265C2650266826602674267C267E0
:10303000C0F88420C0F88820C0F8902085854166BB
:10304000C1668167C0F88010C0F88C10C0F8941079
:103050002A49C0F8A0600262294E42608260C260C4
:10306000026142618561426280F83840254A264FFC
:10307000C0F8CC6002254FF6FF7440F20226C0F87B
:10308000D810C0F8DC202149214A80F8E050448063
:10309000204D214CDFF884C0C0F8A4C0C0F8A8704F
:1030A0008683C0F8AC10C0F8B410C0F8C010C0F8E7
:1030B000C810C0F8B020C0F8B820C0F8BC20C0F8D4
:1030C000C420C0F8D050C0F8D45004634463F0BCAE
:1030D000704700BF0000604017B7D138894100BF7A
:1030E000CDCCCCBE000040BFE17A94BECDCCCCBDEF
:1030F00052499DBC5F29CB3D76E06C3F00C0A8479C
:10310000D85500644031774CBF0E7C3F0000A04191
:1031100000002042000061450000E1449BE67D3F45
:103120002DE9F04786B004AB05AE04460078CDE942
:1031300000360DF10F030D4601F066FE9DF90F00FC
:10314000E8B94FF0010A04F1E80904F1CE0804F1EE
:10315000CC075FFA8AF3013B052B35D8DFE803F093
:103160002D261F181203424631462846FFF788FADB
:103170000AF1010ABAF1080FEBD19DF90F0006B070
:10318000BDE8F0873A4631462846FFF799FCEFE75D
:1031900004F1E20231462846FFF75CFCE8E704F15F
:1031A0003C0231462846FFF715FCE1E704F1D00266
:1031B00031462846FFF7E8F9DAE704F1D80231464C
:1031C0002846FFF7E1F9D3E74A4631462846FFF79C
:1031D000DBF9CDE72DE9F04F95B015469DF8786005
:1031E0000C969DF87C600A969DF8806005960A46CC
:1031F0009DF88460AD490992044640680D939A4653
:103200000B9602F09DFDAA490746284602F098FD5C
:10321000A8498146284602F08BFC0146484602F048
:1032200043FEDDE923682AF023F8A349814650468E
:1032300002F086FDA14902F037FE494602F080FD0A
:103240009F498146284602F073FC0146484602F039
:103250002BFE9C4902F074FD9B49814602F02CFF35
:10326000002840F00D824FF0404306936388B3F589
:10327000967F4FF00C0200F00E82B3F5E16F00F084
:103280003282642B00F01B82E36B079304F15C0134
:10329000E36C089311A825F07DF9082204F1680178
:1032A0000FA825F077F9D4F8ACB0D4F8BCA08049C9
:1032B000584602F045FD7F498146584602F038FCE9
:1032C0000146484602F0F0FD29F0D2FF7A498146D6
:1032D000504602F035FD794902F0E6FD494602F01C
:1032E0002FFD77498146584602F022FC01464846A8
:1032F00002F0DAFD734902F023FD2AF007F8D4F852
:1033000008A081460021504602F0AEFE002800F0E1
:1033100082814FF07E590899284602F011FD6749D5
:1033200002F0C2FD07998346069802F009FD0146A6
:10333000584602F0FDFB0146099802F0F7FB5146A2
:1033400002F0F4FB494602F0FBFC514602F0F0FBB0
:10335000C8F80000814694F9CD0002F09DFC0146BA
:10336000284602F095FE002800F0208194F9CC0058
:1033700002F092FC0146284602F094FE002800F07C
:10338000158194F8CF0002F087FC0D9D0146284678
:1033900002F07EFE002800F0098194F8CE0002F0D1
:1033A0007BFC0146284602F07DFE0A9B002800F0C7
:1033B000FD80002B00F0FA800B9B002B40F0BB80BF
:1033C0002298002102F050FE002800F0CC81A56A6E
:1033D0000021284602F048FE002800F0E681A0689F
:1033E000002102F041FE18B1C4F80890D8F800900E
:1033F0002069002102F038FE58B13946A06802F079
:1034000095FB494602F058FE18B1C4F81090D8F860
:103410000090059B029301250223CDE90053494604
:103420002046002304F10802FFF790FC20690021E8
:1034300002F01AFE002800F07C81E068002102F012
:1034400013FE10B1D8F80030E3606069002102F08B
:103450000BFED8F8009060B13946E06802F066FBD8
:103460000146484602F00AFE18B1C4F81490D8F894
:103470000090059B0293022549462046CDE9005560
:10348000002304F10C02FFF761FC6069002102F0E7
:10349000EBFD002800F05A81D8F80090A06849465A
:1034A00002F0F6FD002840F08A800FE0C178C63DAA
:1034B000C3F58C41B81E73438195C3400000C842D8
:1034C0003393884333B358430AD7233C2069494692
:1034D00002F0E8FD051E18BF012501234A463946C2
:1034E0002046FFF7FFFB0C9B002B6AD00A9B002BAA
:1034F00067D00121034600912A4639462046FFF74E
:1035000001FD2062D8F80090E068494602F0C0FD55
:10351000002800F0FC804A46022339462046FFF787
:10352000E1FB0546022100910A9A2B4639462046C6
:10353000FFF7E8FC6062A5680021284602F094FDD0
:1035400008B1D8F80050D4F80CA0D4F8209000218D
:10355000504602F089FD08B1D8F800A03560D4F8D3
:1035600010800021404602F07FFD20B128463946F8
:1035700002F0DCFA8046C6F80880C6F81090C6F85B
:1035800004A065690021284602F06EFD20B139468D
:10359000504602F0CBFA0546F560636A736194F811
:1035A0003830012B20D015B0BDE8F08F0B9B002BDD
:1035B000C1D1A068494602F06BFD002886D00125E4
:1035C0008BE794F8E020227700232362D8F800509C
:1035D00002232A4639462046FFF784FB94F8E03060
:1035E000637700206062A6E77749484602F03CFD19
:1035F00058B1059B4BB1D4F8D030D4F8D420236314
:103600000023626384F83830CDE7704B2363636333
:1036100015B0BDE8F08F4946069802F087FA0146DA
:10362000814602F08DFB119902F08AFB12998246C5
:10363000484602F085FB0146504602F079FA13999C
:1036400002F076FA59468146284602F06FFA604940
:1036500002F02AFC0F9902F073FB109902F068FA4D
:103660000146484602F06CFB4FF07F5129F00CFDFB
:103670004FF07C5129F0F6FCD4F808A081464AE6C8
:10368000484629F043FE63880690B3F5967F4FF0D5
:103690000C027FF4F2AD636C079304F18401636D57
:1036A000089311A824F076FF082204F190010FA8D6
:1036B00024F070FFD4F8B4B0D4F8C4A0F7E5A36C3C
:1036C000079304F19801A36D089311A824F062FFF9
:1036D000082204F1A4010FA824F05CFFD4F8B8B0CC
:1036E000D4F8C8A0E3E5236C079304F17001236DBF
:1036F000089311A824F04EFF082204F17C010FA8C2
:1037000024F048FFD4F8B0B0D4F8C0A0CFE502232D
:103710004A4639462046D4F814A0FFF7E3FA494652
:103720000546504602F0BEFC031E18BF01230A9353
:10373000F8E6059B0095CDE9015304F11002D8F895
:1037400000102B462046FFF701FB76E60123CDE96A
:103750000053059A0292D8F8001004F11402204692
:10376000FFF7F4FA98E6229802F0B0FC04EB40036D
:103770000546B3F8E000D4F8289002F089FA014633
:10378000484602F0D3F93935824654F8250029F02D
:103790006FFD0146504602F087FB0146484602F0A5
:1037A000C5F9A062D8F8009078E6A08D02F070FA12
:1037B0000146284602F0BAF90146002029F052FCE1
:1037C000A062D8F8009069E6000040400000E144A3
:1037D0000000C8422DE9F047072484B00646904611
:1037E00000788DF807400DEB04020D4601F03AFB1E
:1037F0009DF8077003902FB3012406F1E80A06F143
:10380000CE09E3B2013B062B0BD8DFE803F0352DE0
:10381000453D4D10040003AB424629465046FEF795
:10382000CDFEA74204F101030BD01C46E9E703AB30
:10383000424629464846FEF739FFA74204F10103F4
:10384000F3D10398ADF80A0002220DF10A0102A893
:1038500024F0A0FE9DF808209DF8093003982A70F6
:103860006B7004B0BDE8F08703AB4246294606F111
:10387000D000FEF7A3FED4E703AB4246294606F18B
:10388000D800FEF79BFECCE703AB4246294606F183
:10389000E200FFF76FF8C4E703AB4246294606F1A2
:1038A0003C00FFF721F8BCE703AB4246294606F18E
:1038B000CC00FFF7A9F8B4E72DE9F04784B006463D
:1038C000174600780D240DF107020D468DF80740CC
:1038D00001F0C8FA9DF807800390B8F1000F29D0D5
:1038E000012406F1300A06F12009E3B2013B0C2B5A
:1038F0000FD8DFE803F06C647B745D554E474039A8
:103900003114070096F8380003AB3A462946FEF713
:1039100053FFA04504F101030BD01C46E5E703ABC0
:103920003A4629465046FEF749FEA04504F10103F8
:10393000F3D10398ADF80A0002220DF10A0102A8A2
:1039400024F028FE9DF808209DF8093003982A707D
:103950006B7004B0BDE8F08796F8E00003AB3A4620
:103960002946FEF729FFD4E7706803AB3A4629469B
:10397000FEF7E0FECDE7B08D03AB3A462946FEF7F1
:103980005DFEC6E7B06A03AB3A462946FEF7D2FEB3
:10399000BFE703AB3A4629464846FEF70FFEB8E7B5
:1039A00003AB3A46294606F11C00FEF77FFEB0E75E
:1039B000708803AB3A462946FEF740FEA9E703AB01
:1039C0003A46294606F11000FEF7F8FDA1E703ABE1
:1039D0003A46294606F10800FEF7F0FD99E7708B9C
:1039E00003AB3A462946FEF729FE92E7308B03AB3C
:1039F0003A462946FEF722FE8BE700BF30B402218B
:103A00004FF6FF72002340F20225012480F8E010F7
:103A100042800021084A858380F83840836230BCA8
:103A2000036243608360C3600361436143628185D5
:103A300081610263426370470000E14438B54FF68C
:103A4000FF73994230D043888B420C4605462BD0F9
:103A5000B1F5967F418028D0B1F5E16F244B42D07B
:103A6000642940D0A3FB01235A09642101FB1242BF
:103A700092B25B09312A1F4888BF0133AB8529F018
:103A800045FC29F0A9FA1C4902F00EFA6860BCB99D
:103A90001A4829F0B0FC014602F04AF829F0A0FAD1
:103AA00002F03AFB85F8E00038BD03238385144813
:103AB00029F02CFC29F090FA0F4902F0F5F9686022
:103AC00047F23053B3FBF4F004FB10339BB280B2E7
:103AD00033B104F0010101EB5404A342A8BF01304B
:103AE00002F0D6F8D5E7A3FB042306485B09C5E737
:103AF0001F85EB51304C463F502C633E00FF7F4703
:103B00000AD7233F9A99193F2DE9F04786B004ABB5
:103B100005AE04460078CDE900360DF10F030D46E1
:103B200001F072F99DF90F0000BB4FF0010A04F19A
:103B3000300904F1200804F11C075FFA8AF3013B05
:103B40000B2B5BD8DFE803F0534C46403A342E226F
:103B50001C2815064A4631462846FEF715FD0AF18F
:103B6000010ABAF10E0FE8D19DF90F0006B0BDE8C9
:103B7000F08731462846FEF709FE84F8E000EEE7BC
:103B800031462846FEF742FDA085E8E73146284643
:103B9000FEF7B2FDA062E2E731462846FEF7ACFD33
:103BA0006060DCE7424631462846FEF7EDFCD6E78A
:103BB0003A4631462846FEF763FDD0E731462846AF
:103BC000FEF724FD6080CAE731462846FEF71EFD59
:103BD0006083C4E731462846FEF718FD2083BEE720
:103BE00004F1100231462846FEF7CEFCB7E704F197
:103BF000080231462846FEF7C7FCB0E731462846A2
:103C0000FEF7C4FD84F83800A9E700BF10B5032310
:103C1000044600F8043B01F07FFA204601F0F6F973
:103C2000204610BD70B586B004AB05AE04460078E2
:103C3000CDE900360DF10F030D4601F0E5F89DF9D1
:103C40000F0008B106B070BD284604F120023146CD
:103C5000FEF75EFC9DF90F0006B070BD2DE9F84F30
:103C60000D46044608462749DDF83090DDE90ABADA
:103C700017461E4602F00CFA00B1224DD4F810800F
:103C80000021404602F0F0F9002833D1284665684B
:103C900029F03CFB216901F049FF294602F050F868
:103CA000414601F045FFCBF80000656938462946DA
:103CB00001F03CFFA16802F043F8294601F038FF0B
:103CC000CAF80000A5693046294601F02FFFE168D7
:103CD00002F036F8294601F02BFFC9F80000DBF8A6
:103CE00000302361DAF800306361D9F80030A36155
:103CF000BDE8F88F284629F009FB676180462061FE
:103D0000A661C3E7000020412DE9F04184B0012500
:103D10000646904600788DF807500DF107020F46D1
:103D200001F0A0F89DF80750039035B1203600242B
:103D3000ACB10134A542FBD10398ADF80A000222D0
:103D40000DF10A0102A824F025FC9DF808209DF839
:103D5000093003983A707B7004B0BDE8F08103AB82
:103D6000424639463046FEF7EFFBE2E72DE9F041E7
:103D700084B001250646904600788DF807500DF175
:103D800007020F4601F06EF89DF80750039035B119
:103D900010360024ACB10134A542FBD10398ADF834
:103DA0000A0002220DF10A0102A824F0F3FB9DF89B
:103DB00008209DF8093003983A707B7004B0BDE884
:103DC000F08103AB424639463046FEF7BDFBE2E7E1
:103DD00070B586B004AB05AE04460078CDE9003678
:103DE0000DF10F030D4601F00FF89DF90F0008B11A
:103DF00006B070BD284604F110023146FEF788FB7C
:103E00009DF90F0006B070BDF0B5044685B00846B8
:103E100001F03EFF01461C4802F046F84FF07C518D
:103E200001F08EFF01460546206A02F03DF84FF092
:103E30007E573946064602F03FF9F0B10197294610
:103E4000606A02F031F84FF07E573946064602F0BC
:103E500033F9B0B102972946A06A02F025F84FF075
:103E60007E563146054602F027F940B10396201DE3
:103E700001A901F0E7F805B0F0BD0196DFE7039571
:103E8000F5E70296E7E700BF0000C84210B5044618
:103E900000F8041B01F04EF9204601F0CBF8204653
:103EA00010BD00BF70B586B004AB05AE0446007807
:103EB000CDE900360DF10F030D4600F0A5FF9DF989
:103EC0000F0008B106B070BD284604F1100231465B
:103ED000FEF75AFB9DF90F0006B070BD2DE9F041C9
:103EE00004460F46184600211D46904602F0D0F8C1
:103EF00000282DD11749284602F0DEF830BBA6680D
:103F00000021304602F0B0F800B13E463146384656
:103F100001F00CFE616801F013FF314601F008FE6C
:103F20002169A0600646284601F00AFF616901F098
:103F3000FFFD294601F0FCFD41460246304600F0F7
:103F4000D7FFBDE8F041034929F09EB8014DD6E7FF
:103F5000014DD4E70000C84217B7D1382DE9F04130
:103F600084B001250646904600788DF807500DF183
:103F700007020F4600F076FF9DF80750039035B119
:103F800010360024ACB10134A542FBD10398ADF842
:103F90000A0002220DF10A0102A824F0FBFA9DF8A2
:103FA00008209DF8093003983A707B7004B0BDE892
:103FB000F08103AB424639463046FEF797FDE2E713
:103FC0002DE9F04184B007469046007801240DF1B8
:103FD00007020E468DF8074000F044FF9DF8075099
:103FE00003902DB10024ACB10134A542FBD103985C
:103FF000ADF80A0002220DF10A0102A824F0CAFA63
:104000009DF808209DF8093003983270737004B051
:10401000BDE8F081B86803AB42463146FEF78AFB43
:10402000E2E700BF70B586B004AB05AE0446007889
:10403000CDE900360DF10F030D4600F0E5FE9DF9C8
:104040000F0008B106B070BD31462846FEF754FB9C
:1040500003469DF90F00A36006B070BDF8B5054694
:10406000084601F015FE0146194801F01DFF4FF00A
:104070007C5101F065FE4FF07E570146154801F076
:1040800013FF394629F000F81349064601F058FE9F
:1040900029F04CF8014601F053FE0446014601F0B8
:1040A0004FFE214601F044FD29F0A5F939460346AB
:1040B00030461E4601F0D8FF40B92146304601F097
:1040C00035FD014601F034FD6860F8BD6F60F8BD54
:1040D0000000C84299D4503CDB0FC93F30B40224E1
:1040E00000224FF4FA7196250470027132244FF0C9
:1040F000814241800E49C58004724FF4C8750D4C51
:10410000026141614FF07C524FF47A710583C461C2
:10411000094D0A4C02628184002209498562846348
:10412000C26030BCC26202634263C1630164704713
:104130000000204100007041CDCCCC3DEC518542C7
:10414000000048422DE9F84F1768DDF828B0044612
:10415000384615469846894601F0E8FC06466088D0
:1041600001F096FDA968034638461F4601F0DEFCC3
:104170000146304601F098FE8246E08801F088FD55
:104180000146504601F0DCFD8246207A01F080FDB8
:104190000146504601F0CCFC8246207901F078FDC2
:1041A000514628F05FFF0146384628F06DFFE16870
:1041B0000746304601F0C4FD0646207A01F068FD4E
:1041C0000146304601F0B4FC0646207901F060FD5E
:1041D000314628F047FF4FF07E510646404601F039
:1041E0004DFF00286ED1E7632664CBF800702B6981
:1041F000CBF804300B9B0B9A1E602B695360A06BAD
:10420000314601F04FFF002852D0208B01F040FDD5
:1042100021690746304601F093FD394601F088FCDC
:1042200080464146384628F01DFF0C9B0C9A1860CA
:104230002B695360A08C01F02BFDE16AA76A03464D
:1042400030461E4601F07CFD216B01F071FC0146F9
:10425000384829F083F80146384628F003FF014624
:10426000304628F011FF0D9B0D9A18602B695360A2
:104270006E68676B4946304601F058FCE9680446B1
:10428000304601F053FC0146204601F00DFE2A495C
:1042900001F056FD284928F0F7FE0146384628F07F
:1042A000E1FE0E9B0E9A18606B695360BDE8F88FB3
:1042B0006169304601F044FD8046208B01F0E8FC46
:1042C0000746AEE74146404601F03AFDD4F83CA02F
:1042D00080463946504601F0D1FE80B1384641460D
:1042E00001F02EFD414607464FF07E5001F01EFCC6
:1042F000514601F025FD394601F01AFC0746D4F875
:1043000040A03146504601F0B9FE00283FF46DAFA1
:104310003046414601F014FD414606464FF07E50BE
:1043200001F004FC514601F00BFD314601F000FCA8
:1043300006465AE7000020410000C8422DE9F0433C
:1043400085B006461746007808240DF107020D4691
:104350008DF8074000F086FD9DF807800390B8F1C6
:10436000000F23D0012406F11009E3B2013B072B13
:104370000BD8DFE803F0423B5049342D1004306A7B
:1043800003AB3A462946FEF7D5F9A04504F10103EF
:104390000BD01C46E9E703ABF0693A462946FEF725
:1043A000C9F9A04504F10103F3D10398ADF80A005F
:1043B00002220DF10A0102A824F0ECF89DF8082071
:1043C0009DF8093003982A706B7005B0BDE8F08342
:1043D000308B03AB3A462946FEF730F9D5E703ABFD
:1043E0003A4629464846FEF781FBCEE7708803AB84
:1043F0003A462946FEF722F9C7E7307903AB3A4639
:104400002946FEF7D9F9C0E7307A03AB3A46294688
:10441000FEF7D2F9B9E7F08803AB3A462946FEF732
:104420000DF9B2E72DE9F04184B0804616460078D8
:1044300002240DF107020D468DF8074000F012FD31
:104440009DF807700390F7B101240DE0022B32466E
:1044500003AB294603D1D8F84000FEF76BF9A74219
:1044600004F101030ED01C46E3B2012BEED103ABE5
:10447000D8F83C0032462946FEF75CF9A74204F121
:104480000103F0D10398ADF80A0002220DF10A01F0
:1044900002A824F07FF89DF808209DF809300398C1
:1044A0002A706B7004B0BDE8F08100BF70B586B0B3
:1044B00004AB05AE04460078CDE900360DF10F03DC
:1044C0000D4600F0A1FC9DF90F0008B106B070BDCB
:1044D00031462846FEF710F93146E0632846FEF7DC
:1044E0000BF903469DF90F00236406B070BD00BFB1
:1044F0002DE9F8434FF6FF7399423CD00446C0883B
:10450000237A18440D4601F0C7FBB5F5967F0646A1
:1045100036D0B5F5E16F30D0642D2ED0DFF868903D
:10452000E06928F0F3FE0546207A01F0B1FB014670
:10453000304601F0FBFA8046206A28F0E7FE01468B
:10454000284601F0F3FA414601F0AEFC0746484622
:1045500028F0DCFE28F040FD0146404601F0A4FCB6
:104560003946E060E762304601F0EAFB0146284642
:1045700001F0DCFA2063BDE8F883DFF81090CFE7A4
:10458000DFF80C90CCE700BF304C463F9A99193FBA
:104590000AD7233F2DE9F04186B004AB05AF0546AD
:1045A0000078CDE900370DF10F030E4600F02CFC2A
:1045B0009DF90F00B0B9012405F11008E3B2013BE9
:1045C000062B36D8DFE803F02F29231D171104002E
:1045D00039463046FEF790F8E8610134092CEDD1F8
:1045E0009DF90F0006B0BDE8F08139463046FEF770
:1045F0000DF82883F1E7424639463046FDF7C4FFFF
:10460000EBE739463046FEF7C1F82872E5E7394650
:104610003046FDF7FBFFE880DFE739463046FDF71F
:10462000F5FF6880D9E739463046FEF7AFF82871C4
:10463000D3E739463046FEF75FF82862CDE700BF82
:1046400030B409241549164A164D0470164C4160C1
:1046500002611649164A45618461164D164C416245
:1046600082621649164AC5628463164D164CC163B0
:1046700002641649C56400226FF0004504654FF0DE
:10468000FF34C0E91645016630BC8260C260C26179
:1046900002620263426342648264704707F0963D9F
:1046A0001C7CE13D3480D73F0000A040CDCC0C3EC7
:1046B00067D5273EE63F4CC091ED3CBFFB3A403FFB
:1046C000B15083405DFEE33E363C85BF0000404074
:1046D0002DE9F04786B004AB05AE04460078CDE97D
:1046E00000360DF10F030D4600F08EFB9DF90F0013
:1046F000E0B94FF0010A04F1400904F12C0804F17B
:1047000018075FFA8AF3013B032B24D8DFE803F094
:104710001D1711024A4631462846FEF74BFA0AF1A8
:10472000010ABAF1060FECD19DF90F0006B0BDE801
:10473000F087424631462846FEF73CFAEFE73A4614
:1047400031462846FEF736FAE9E7221D314628466B
:10475000FEF730FAE3E731462846FDF7CDFF206645
:10476000DDE700BF2DE9F04782B0DDE90A9ABDF828
:104770003040B4F5E16F0546884617461E466FD0B7
:1047800028D941F270739C422ED047F230539C429C
:1047900008BF012408D1D5E916014FF0FF326FF0B0
:1047A000004300F02DFC08B300244FF0FF326FF0FF
:1047B00000433846314600F023FC08B9C5E91676B7
:1047C0002146404601F0B2F90D9901F0AFF902B06F
:1047D000BDE8F087642C05D0B4F5967F08BF0424AB
:1047E000D9D0E1E70524D6E70224D4E7D5E91601BC
:1047F000B9EB00006AEB010100F034FE1AA3D3E923
:10480000002300F087FF0B460246CDE900230FFA94
:1048100084F901F037F905EB840455F82910824634
:1048200001F08EFA616901F083F9A16A8146504670
:1048300001F086FADDE9002382461946104600F0B1
:104840003FFE01F01FF90146504601F071F9E16B9E
:1048500001F06EF90146484601F026FB0446A4E744
:10486000046EA2E7AFF300800000000065CDCD41EB
:104870002DE9F04784B007469046007805240DF1F5
:1048800007020D468DF8074000F0ECFA9DF807602E
:1048900003902EB3012407F1400A07F12C09E3B27B
:1048A000013B042B0AD8DFE803F03B0F342D030053
:1048B000386E03AB42462946FDF73CFFA64204F1A1
:1048C00001030CD01C46EAE703AB4246294607F138
:1048D0001800FEF743F9A64204F10103F2D1039850
:1048E000ADF80A0002220DF10A0102A823F052FEDF
:1048F0009DF808209DF8093003982A706B7004B069
:10490000BDE8F08703AB424629465046FEF726F93C
:10491000D4E703AB424629464846FEF71FF9CDE7E8
:1049200003AB42462946381DFEF718F9C6E700BF1B
:104930002DE9F04387B080469146007801240DF1BF
:104940000F020E468DF80F4000F08CFA9DF80F50C4
:10495000059035B1002405AFACB10134A542FBD1BF
:104960000598ADF8120002220DF1120104A823F0FF
:1049700011FE9DF810209DF811300598327073706B
:1049800007B0BDE8F0830097D8E916014B463246E0
:10499000FDF746FFE1E700BF70B586B004AB05AE9A
:1049A00004460078CDE900360DF10F030D4600F006
:1049B0002BFA9DF90F0008B106B070BD31462846AC
:1049C000FDF712FFC4E916019DF90F0006B070BD96
:1049D00030B40524094D0470012400220849C56142
:1049E000846200250024C0E90245C0E90845C1628F
:1049F00030BC02614261826102637047C9B28B536D
:104A000023291D5670B586B004AB05AE0446007868
:104A1000CDE900360DF10F030D4600F0F5F99DF9D3
:104A20000F0008B106B070BD31462846FDF764FEA0
:104A30003146A0612846FEF77BF8314684F828000D
:104A40002846FDF759FE03469DF90F00E36206B0C4
:104A500070BD00BF2DE9F8430446D0E902011646B7
:104A60001F46D4E90823B6EB000867EB010942456D
:104A700073EB0903099D03DB864277EB010361DADF
:104A800000234FF00009236184F82A90C4E90267EB
:104A900094F82980B8F1000F0FD1D4E90201301A3F
:104AA00067EB010101F00EF9616901F041F8A169BC
:104AB000606101F0F7FA00285AD194F82B307BB9E5
:104AC000D4E90201301A67EB010101F0FBF8216B18
:104AD00001F02EF8E16A206301F0E4FA002843D1E6
:104AE000B9F1000F0ED1D4E90201301A67EB0101D0
:104AF00001F0E8F8216901F01BF8E169206101F09B
:104B0000D1FA68BB012E77F10003089B0B9ABCBF5A
:104B100001260027C4E9026783F8008094F82A3050
:104B20002B7094F82B3013702B782BB9E56900218A
:104B3000284601F099FA58B10A9A4FF07E53136053
:104B4000BDE8F88350EA010394F82A90A0D19DE7CC
:104B50002069294601F0A8F90A9B1860BDE8F8838E
:104B6000012384F82A30CDE7012384F82B30B7E7FE
:104B70004FF0010884F829809FE700BF2DE9F0413C
:104B800084B007469046007803240DF107020D46D5
:104B90008DF8074000F066F99DF807600390C6B1F4
:104BA000012406E0012B2ED0A64204F101030FD010
:104BB0001C46E3B2022B1ED0032BF3D103ABF86AE1
:104BC00042462946FDF7B6FDA64204F10103EFD1A6
:104BD0000398ADF80A0002220DF10A0102A823F0A1
:104BE000D9FC9DF808209DF8093003982A706B7055
:104BF00004B0BDE8F08197F9280003AB424629468E
:104C0000FDF746FFD0E7B86903AB42462946FDF7FA
:104C100091FDC9E72DE9F04186B00646904600783F
:104C200007240DF10F020D468DF80F4000F01AF920
:104C30009DF80F70059017B30124E3B2013B062BDA
:104C40000BD8DFE803F0352E463E4D100400306BE4
:104C500005AB42462946FDF76DFDA74204F101036D
:104C60000CD01C46E9E705AB96F82B0042462946D6
:104C7000FDF714FEA74204F10103F2D10598ADF847
:104C8000120002220DF1120104A823F083FC9DF80A
:104C900010209DF8113005982A706B7006B0BDE8A1
:104CA000F081706905AB42462946FDF743FDD4E724
:104CB00005AB0093D6E9020143462A46FDF7B0FD55
:104CC000CBE796F8290005AB42462946FDF7E6FDFD
:104CD000C3E7306905AB42462946FDF72BFDBCE72B
:104CE00096F82A0005AB42462946FDF7D7FDB4E702
:104CF0004FF6FF7399421BD090F92820114B01FB0E
:104D000002F202EB5202A2FB0323B1F5967FC0E947
:104D1000082307D0B1F5E16F07D0642902D00A4B10
:104D2000C3617047094BC3617047094BC36170474A
:104D300000230361002100220023C0E9022380F840
:104D40002A10704780969800C9B28B53C9B28B5213
:104D500076845F51F0B587B004AB05AF05460078A7
:104D6000CDE900370DF10F030E4600F04DF89DF927
:104D70000F00C0B90124E3B2013B052B3ED8DFE8A8
:104D800003F036302A1F1403059BF25C003A03F14E
:104D9000010318BF012285F82B2005930134082C4C
:104DA000E9D19DF90F0007B0F0BD059BF25C003A18
:104DB00003F1010318BF012285F82A200593EDE7CE
:104DC000059BF25C003A03F1010318BF012285F84C
:104DD00029200593E2E739463046FDF78DFC28612E
:104DE000DCE739463046FDF787FC6861D6E739468F
:104DF0003046FDF7F9FCC5E90201CFE739463046F8
:104E0000FDF77AFC2863C9E72DE9F04182B0DDE9BE
:104E100008751C46032A4FF000032B6023703B608B
:104E200004D89823237002B0BDE8F08104232B60DE
:104E30000A784B788DF8042080460E46022201A99C
:104E40000DF106008DF8053023F0A4FBBDF8063007
:104E50003B60B37843451CBF9C23237002B0BDE880
:104E6000F08100BF10B414780CB19C4203D2002032
:104E700010BC10707047887010BC0420704700BFD1
:104E800038B504460D4628F023F8164B002200F0F2
:104E900089FD78B1144B00222046294600F096FD8A
:104EA00058B9124B00222046294600F099FD70B1F6
:104EB000002400252046294638BD0B4B20462946B4
:104EC000002200F047F9BDE8384028F005B8064B4D
:104ED00020462946002200F03BF9BDE8384027F083
:104EE00077BF00BF000030430000E03F0000E0BF9C
:104EF000F8B505460C4610460021164601F0BEF8EE
:104F0000002855D12B49304601F0D6F800284CD165
:104F10002849304600F0C8FF28F0D0F92649064657
:104F2000284600F00DFF25490746284600F000FE00
:104F30000146384600F0B8FF314600F0F9FD1F4940
:104F4000054600F0FDFE294605461B4800F0EEFD33
:104F50000146284600F0A8FF1749064600F0F0FE7B
:104F600016490546304600F0E3FD0146284600F0AC
:104F70009BFF11490546204600F0E2FE0F49064618
:104F8000204600F0D5FD0146304600F08DFF014679
:104F9000284600F0CBFD28F06BF9064900F0D0FE62
:104FA000BDE8F840034928F06FB84FF07E50B3E7F2
:104FB0000020B1E70000C842C3F58C41B81E73431E
:104FC000002917DD30B401380C4D44184FF6FF733B
:104FD00010F8011F4B40D9B2844235F8111081EA14
:104FE0001323F5D1DB43D9B2C3F3072330BC1170CF
:104FF0005370704700231370537070477C3A030856
:10500000994206BF9042012000207047037F074A63
:1050100007490162426282623BB10022012B0261B8
:1050200003D0022B426118BF826170470AD7233B2D
:105030000AD7A33C027B00230361436102B1836072
:10504000704700BFF8B50C4605463249206800F0AD
:1050500077FE28F06BF8014600F072FE0646014626
:1050600000F06EFE314600F063FD28F0C4F93146D1
:1050700000F05CFD014600F05BFD4FF07E572860BC
:105080002068394600F0F0FF00B12F6021496068C8
:1050900000F056FE28F04AF8014600F051FE0646A0
:1050A000014600F04DFE314600F042FD28F0A3F924
:1050B000314600F03BFD014600F03AFD4FF07E57CF
:1050C00068606068394600F0CFFF00B16F60114939
:1050D000A06800F035FE28F029F8014600F030FE07
:1050E0000646014600F02CFE314600F021FD28F076
:1050F00082F9314600F01AFD014600F019FD4FF02B
:105100007E57A860A068394600F0AEFF00B1AF60DE
:10511000F8BD00BFDB0FC93F4FF07C51002210B437
:1051200003240476016010BC41608160C2600261AA
:105130004261704710B401244FF07C510022047288
:10514000016010BC4260704781F0004102E000BF86
:1051500083F0004330B54FEA41044FEA430594EA37
:10516000050F08BF90EA020F1FBF54EA000C55EA72
:10517000020C7FEA645C7FEA655C00F0E2804FEA43
:105180005454D4EB5555B8BF6D420CDD2C4480EA25
:10519000020281EA030382EA000083EA010180EA55
:1051A000020281EA0303362D88BF30BD11F0004FA3
:1051B0004FEA01314FF4801C4CEA113102D04042D9
:1051C00061EB410113F0004F4FEA03334CEA133314
:1051D00002D0524263EB430394EA050F00F0A7802C
:1051E000A4F10104D5F1200E0DDB02FA0EFC22FA27
:1051F00005F2801841F1000103FA0EF2801843FA1B
:1052000005F359410EE0A5F120050EF1200E012A0B
:1052100003FA0EFC28BF4CF0020C43FA05F3C01849
:1052200051EBE37101F0004507D54FF0000EDCF1C2
:10523000000C7EEB00006EEB0101B1F5801F1BD36B
:10524000B1F5001F0CD349085FEA30004FEA3C0C6F
:1052500004F101044FEA445212F5800F80F09A8065
:10526000BCF1004F08BF5FEA500C50F1000041EB69
:10527000045141EA050130BD5FEA4C0C404141EB6D
:105280000101013C28BFB1F5801FE9D291F0000F68
:1052900004BF01460020B1FA81F308BF2033A3F117
:1052A0000B03B3F120020CDA0C3208DD02F1140C0E
:1052B000C2F10C0201FA0CF021FA02F10CE002F149
:1052C0001402D8BFC2F1200C01FA02F120FA0CFC42
:1052D000DCBF41EA0C019040E41AA2BF01EB04518B
:1052E000294330BD6FEA04041F3C1CDA0C340EDC89
:1052F00004F11404C4F1200220FA04F001FA02F3CC
:1053000040EA030021FA04F345EA030130BDC4F189
:105310000C04C4F1200220FA02F001FA04F340EA7E
:105320000300294630BD21FA04F0294630BD94F02F
:10533000000F83F4801306BF81F480110134013D16
:105340004EE77FEA645C18BF7FEA655C29D094EA87
:10535000050F08BF90EA020F05D054EA000C04BF05
:105360001946104630BD91EA030F1EBF00210020F0
:1053700030BD5FEA545C05D14000494128BF41F08F
:10538000004130BD14F580043CBF01F5801130BDF3
:1053900001F0004545F0FE4141F470014FF000007E
:1053A00030BD7FEA645C1ABF194610467FEA655C2F
:1053B0001CBF0B46024650EA013406BF52EA0335D1
:1053C00091EA030F41F4002130BD00BF90F0000FBF
:1053D00004BF0021704730B54FF4806404F13204FB
:1053E0004FF000054FF0000150E700BF90F0000FB4
:1053F00004BF0021704730B54FF4806404F13204DB
:1054000010F0004548BF40424FF000013EE700BFAA
:1054100042004FEAE2014FEA31014FEA02701FBF3A
:1054200012F07F4393F07F4F81F06051704732F06C
:105430007F4208BF704793F07F4F04BF41F40021C3
:10544000704730B54FF4607401F0004521F0004121
:105450001CE700BF50EA010208BF704730B54FF0AB
:1054600000050AE050EA010208BF704730B511F0AC
:10547000004502D5404261EB41014FF4806404F1E4
:1054800032045FEA915C3FF4D8AE4FF003025FEA6A
:10549000DC0C18BF03325FEADC0C18BF033202EBEE
:1054A000DC02C2F1200300FA03FC20FA02F001FA48
:1054B00003FE40EA0E0021FA02F11444BDE600BFEB
:1054C00070B54FF0FF0C4CF4E06C1CEA11541DBF9A
:1054D0001CEA135594EA0C0F95EA0C0F00F0DEF865
:1054E0002C4481EA030621EA4C5123EA4C5350EA4A
:1054F000013518BF52EA033541F4801143F480139B
:1055000038D0A0FB02CE4FF00005E1FB02E506F02B
:105510000042E0FB03E54FF00006E1FB03569CF080
:10552000000F18BF4EF0010EA4F1FF04B6F5007F86
:1055300064F5407404D25FEA4E0E6D4146EB0606F8
:1055400042EAC62141EA55514FEAC52040EA5E5081
:105550004FEACE2EB4F1FD0C88BFBCF5E06F1ED82B
:10556000BEF1004F08BF5FEA500E50F1000041EB62
:10557000045170BD06F0004646EA010140EA02000F
:1055800081EA0301B4EB5C04C2BFD4EB0C0541EA31
:10559000045170BD41F480114FF0000E013C00F346
:1055A000AB8014F1360FDEBF002001F0004170BD6A
:1055B000C4F10004203C35DA0C341BDC04F1140483
:1055C000C4F1200500FA05F320FA04F001FA05F20F
:1055D00040EA020001F0004221F0004110EBD370DC
:1055E00021FA04F642EB06015EEA430E08BF20EA08
:1055F000D37070BDC4F10C04C4F1200500FA04F3AB
:1056000020FA05F001FA04F240EA020001F000413C
:1056100010EBD37041F100015EEA430E08BF20EAAF
:10562000D37070BDC4F1200500FA05F24EEA020EF7
:1056300020FA04F301FA05F243EA020321FA04F026
:1056400001F0004121FA04F220EA020000EBD370DD
:105650005EEA430E08BF20EAD37070BD94F0000FDD
:105660000FD101F00046400041EB010111F4801F11
:1056700008BF013CF7D041EA060195F0000F18BFC2
:10568000704703F00046520043EB030313F4801FFE
:1056900008BF013DF7D043EA0603704794EA0C0FB8
:1056A0000CEA135518BF95EA0C0F0CD050EA4106CE
:1056B00018BF52EA4306D1D181EA030101F000414B
:1056C0004FF0000070BD50EA410606BF1046194673
:1056D00052EA430619D094EA0C0F02D150EA01367F
:1056E00013D195EA0C0F05D152EA03361CBF1046C0
:1056F00019460AD181EA030101F0004141F0FE415F
:1057000041F470014FF0000070BD41F0FE4141F4E2
:10571000780170BD70B54FF0FF0C4CF4E06C1CEAE2
:1057200011541DBF1CEA135594EA0C0F95EA0C0F97
:1057300000F0A7F8A4EB050481EA030E52EA033552
:105740004FEA013100F088804FEA03334FF0805573
:1057500045EA131343EA12634FEA022245EA1115A0
:1057600045EA10654FEA00260EF000419D4208BF51
:10577000964244F1FD0404F5407402D25B084FEAFE
:105780003202B61A65EB03055B084FEA32024FF4AA
:1057900080104FF4002CB6EB020E75EB030E22BF07
:1057A000B61A754640EA0C005B084FEA3202B6EBC7
:1057B000020E75EB030E22BFB61A754640EA5C0076
:1057C0005B084FEA3202B6EB020E75EB030E22BF06
:1057D000B61A754640EA9C005B084FEA3202B6EB07
:1057E000020E75EB030E22BFB61A754640EADC00C6
:1057F00055EA060E18D04FEA051545EA16754FEA28
:1058000006164FEAC30343EA52734FEAC2025FEA45
:105810001C1CC0D111F4801F0BD141EA00014FF0D4
:1058200000004FF0004CB6E711F4801F04BF0143A5
:105830000020B4F1FD0C88BFBCF5E06F3FF6AFAEC1
:10584000B5EB030C04BFB6EB020C5FEA500C50F151
:10585000000041EB045170BD0EF0004E4EEA1131D4
:1058600014EB5C04C2BFD4EB0C0541EA045170BDDB
:1058700041F480114FF0000E013C90E645EA060E1F
:105880008DE60CEA135594EA0C0F08BF95EA0C0F4D
:105890003FF43BAF94EA0C0F0AD150EA01347FF495
:1058A00034AF95EA0C0F7FF425AF104619462CE76C
:1058B00095EA0C0F06D152EA03353FF4FDAE1046CF
:1058C000194622E750EA410618BF52EA43067FF420
:1058D000C5AE50EA41047FF40DAF52EA43057FF4B0
:1058E000EBAE12E74FF0FF3C06E000BF4FF0010CBB
:1058F00002E000BF4FF0010C4DF804CD4FEA410C1F
:105900007FEA6C5C4FEA430C18BF7FEA6C5C1BD0EB
:1059100001B050EA410C0CBF52EA430C91EA030F6C
:1059200002BF90EA020F0020704710F1000F91EAC9
:10593000030F58BF994208BF90422CBFD8176FEA97
:10594000E37040F0010070474FEA410C7FEA6C5C65
:1059500002D150EA013C07D14FEA430C7FEA6C5C6C
:10596000D6D152EA033CD3D05DF8040B704700BF98
:105970008446104662468C461946634600E000BFE6
:1059800001B5FFF7B7FF002848BF10F1000F01BDB8
:105990004DF808EDFFF7F4FF0CBF012000205DF883
:1059A00008FB00BF4DF808EDFFF7EAFF34BF012008
:1059B00000205DF808FB00BF4DF808EDFFF7E0FFA1
:1059C00094BF012000205DF808FB00BF4DF808EDF2
:1059D000FFF7CEFF94BF012000205DF808FB00BF59
:1059E0004DF808EDFFF7C4FF34BF012000205DF83B
:1059F00008FB00BF4FEA410212F5001215D211D583
:105A00006FF47873B3EB625212D94FEAC12343F0BB
:105A1000004343EA505311F0004F23FA02F018BF3D
:105A2000404270474FF00000704750EA013005D106
:105A300011F0004008BF6FF0004070474FF00000C9
:105A4000704700BF4A0011D212F5001211D20DD5D5
:105A50006FF47873B3EB62520ED44FEAC12343F074
:105A6000004343EA505323FA02F070474FF000001E
:105A7000704750EA013002D14FF0FF3070474FF0CD
:105A8000000070474FEA4102B2F1E04324BFB3F592
:105A9000001CDCF1FE5C0DD901F0004C4FEAC002A5
:105AA0004CEA5070B2F1004F40EB830008BF20F089
:105AB0000100704711F0804F21D113F13872BCBF43
:105AC00001F00040704741F480114FEA5252C2F198
:105AD0001802C2F1200C10FA0CF320FA02F018BFE1
:105AE00040F001004FEAC1234FEAD32303FA0CFC34
:105AF00040EA0C0023FA02F34FEA4303CCE77FEAC3
:105B0000625307D150EA01331EBF4FF0FE4040F40C
:105B10004000704701F0004040F0FE4040F40000BB
:105B2000704700BF80F0004002E000BF81F00041FC
:105B300042001FBF5FEA410392EA030F7FEA226C33
:105B40007FEA236C6AD04FEA1262D2EB1363C1BFC3
:105B5000D218414048404140B8BF5B42192B88BF32
:105B6000704710F0004F40F4000020F07F4018BF55
:105B7000404211F0004F41F4000121F07F4118BF75
:105B8000494292EA030F3FD0A2F1010241FA03FC1D
:105B900010EB0C00C3F1200301FA03F100F0004305
:105BA00002D5494260EB4000B0F5000F13D3B0F1CD
:105BB000807F06D340084FEA310102F10102FE2A3C
:105BC00051D2B1F1004F40EBC25008BF20F00100AC
:105BD00040EA03007047490040EB0000013A28BF4B
:105BE000B0F5000FEDD2B0FA80FCACF1080CB2EBCE
:105BF0000C0200FA0CF0AABF00EBC250524218434C
:105C0000BCBFD0401843704792F0000F81F40001F0
:105C100006BF80F400000132013BB5E74FEA4103C3
:105C20007FEA226C18BF7FEA236C21D092EA030F2F
:105C300004D092F0000F08BF0846704790EA010FA9
:105C40001CBF0020704712F07F4F04D1400028BFD6
:105C500040F00040704712F100723CBF00F50000B8
:105C6000704700F0004343F0FE4040F400007047EE
:105C70007FEA226216BF08467FEA2363014642029A
:105C800006BF5FEA412390EA010F40F480007047AD
:105C90004FF0000304E000BF10F0004348BF404253
:105CA0005FEA000C08BF704743F0964301464FF08F
:105CB00000001CE050EA010208BF70474FF00003EB
:105CC0000AE000BF50EA010208BF704711F000432C
:105CD00002D5404261EB41015FEA010C02BF8446FC
:105CE0000146002043F0B64308BFA3F18053A3F55B
:105CF0000003BCFA8CF2083AA3EBC25310DB01FAA2
:105D000002FC634400FA02FCC2F12002BCF1004F25
:105D100020FA02F243EB020008BF20F001007047B6
:105D200002F1200201FA02FCC2F1200250EA4C000A
:105D300021FA02F243EB020008BF20EADC70704750
:105D40004FF0FF0C1CEAD0521EBF1CEAD15392EA5E
:105D50000C0F93EA0C0F6FD01A4480EA010C40023A
:105D600018BF5FEA41211ED04FF0006343EA501094
:105D700043EA5111A0FB01310CF00040B1F5000FD6
:105D80003EBF490041EAD3715B0040EA010062F185
:105D90007F02FD2A1DD8B3F1004F40EBC25008BF6F
:105DA00020F00100704790F0000F0CF0004C08BF8D
:105DB00049024CEA502040EA51207F3AC2BFD2F15A
:105DC000FF0340EAC250704740F400004FF0000368
:105DD000013A5DDC12F1190FDCBF00F000407047A2
:105DE000C2F10002410021FA02F1C2F1200200FAE0
:105DF00002FC5FEA310040F1000053EA4C0308BFA7
:105E000020EADC70704792F0000F00F0004C02BFF7
:105E1000400010F4000F013AF9D040EA0C0093F072
:105E2000000F01F0004C02BF490011F4000F013BCC
:105E3000F9D041EA0C018FE70CEAD15392EA0C0F3A
:105E400018BF93EA0C0F0AD030F0004C18BF31F0A5
:105E5000004CD8D180EA010000F00040704790F07B
:105E6000000F17BF90F0004F084691F0000F91F01F
:105E7000004F14D092EA0C0F01D142020FD193EAE5
:105E80000C0F03D14B0218BF084608D180EA01006D
:105E900000F0004040F0FE4040F40000704740F049
:105EA000FE4040F4400070474FF0FF0C1CEAD05217
:105EB0001EBF1CEAD15392EA0C0F93EA0C0F69D073
:105EC000A2EB030280EA010C49024FEA402037D0DE
:105ED0004FF0805343EA111143EA10130CF00040D5
:105EE0008B4238BF5B0042F17D024FF4000C8B42C5
:105EF00024BF5B1A40EA0C00B3EB510F24BFA3EBA5
:105F0000510340EA5C00B3EB910F24BFA3EB910374
:105F100040EA9C00B3EBD10F24BFA3EBD10340EACE
:105F2000DC001B0118BF5FEA1C1CE0D1FD2A3FF614
:105F300050AF8B4240EBC25008BF20F001007047C9
:105F40000CF0004C4CEA50207F32C2BFD2F1FF036C
:105F500040EAC250704740F400004FF00003013A9D
:105F600037E792F0000F00F0004C02BF400010F441
:105F7000000F013AF9D040EA0C0093F0000F01F055
:105F8000004C02BF490011F4000F013BF9D041EA77
:105F90000C0195E70CEAD15392EA0C0F08D14202AA
:105FA0007FF47DAF93EA0C0F7FF470AF084676E77D
:105FB00093EA0C0F04D14B023FF44CAF08466EE756
:105FC00030F0004C18BF31F0004CCAD130F0004224
:105FD0007FF45CAF31F000437FF43CAF5FE700BF7C
:105FE0004FF0FF3C06E000BF4FF0010C02E000BFA5
:105FF0004FF0010C4DF804CD4FEA40024FEA410347
:106000007FEA226C18BF7FEA236C11D001B052EAFC
:10601000530C18BF90EA010F58BFB2EB030088BFC2
:10602000C81738BF6FEAE17018BF40F00100704731
:106030007FEA226C02D15FEA402C05D17FEA236C13
:10604000E4D15FEA412CE1D05DF8040B704700BF5A
:10605000844608466146FFE70FB5FFF7C9FF0028F1
:1060600048BF10F1000F0FBD4DF808EDFFF7F4FF2A
:106070000CBF012000205DF808FB00BF4DF808EDC3
:10608000FFF7EAFF34BF012000205DF808FB00BFE6
:106090004DF808EDFFF7E0FF94BF012000205DF808
:1060A00008FB00BF4DF808EDFFF7D2FF94BF0120B9
:1060B00000205DF808FB00BF4DF808EDFFF7C8FFB2
:1060C00034BF012000205DF808FB00BF4FEA40020A
:1060D000B2F1FE4F0FD34FF09E03B3EB12620DD916
:1060E0004FEA002343F0004310F0004F23FA02F080
:1060F00018BF404270474FF00000704712F1610F27
:1061000001D1420205D110F0004008BF6FF00040FD
:1061100070474FF00000704742000ED2B2F1FE4FC0
:106120000BD34FF09E03B3EB126209D44FEA002366
:1061300043F0004323FA02F070474FF0000070472D
:1061400012F1610F01D1420202D14FF0FF307047CE
:106150004FF00000704700BF7BB972B90029BEBF85
:1061600000204FF0004106E008BF00281CBF6FF080
:1061700000414FF0FF3000F0F7B9ADF1080C6DE9C8
:1061800004CE002909DB002B1ADB00F085F8DDF8CE
:1061900004E0DDE9022304B07047404261EB4101B5
:1061A000002B1BDB00F078F8DDF804E0DDE90223CA
:1061B00004B0404261EB4101524263EB430370473C
:1061C000524263EB430300F067F8DDF804E0DDE9D9
:1061D000022304B0404261EB41017047524263EB3D
:1061E000430300F059F8DDF804E0DDE9022304B0D0
:1061F000524263EB4303704753B94AB9002908BFC1
:1062000000281CBF4FF0FF314FF0FF3000F0ACB959
:10621000ADF1080C6DE904CE00F03EF8DDF804E0C5
:10622000DDE9022304B0704738B505460C46284620
:10623000214600220023FFF7B5FB28B92846214656
:10624000BDE8384000F00AB8284604F1004100F0EB
:1062500005F8404261EB410138BD00BFD0B50C4BA1
:10626000002206460F46FFF72BF9FFF7EBFB04462B
:10627000FFF7ACF8074B0022FFF722F902460B4666
:1062800030463946FEF764FFFFF7DCFB2146D0BD00
:106290000000F03D0000F0412DE9F047089E0D465A
:1062A00004468846002B4DD18A42944668D9B2FAFA
:1062B00082F252B101FA02F3C2F1200120FA01F197
:1062C0000CFA02FC41EA030894404FEA1C45210CF9
:1062D000B8FBF5FE1FFA8CF705FB1E8341EA03436A
:1062E0000EFB07F199420BD91CEB03030EF1FF30B3
:1062F00080F01E81994240F21B81AEF1020E634490
:106300005B1AA4B2B3FBF5F005FB103344EA034477
:1063100000FB07F7A7420AD91CEB040400F1FF3386
:1063200080F00881A74240F2058164440238E41BF2
:1063300040EA0E4000211EB1D4400023C6E90043CC
:10634000BDE8F0878B4208D9002E00F0EE800021D6
:10635000C6E900050846BDE8F087B3FA83F10029D5
:106360004AD1AB4202D3824200F2F980841A65EB33
:10637000030301209846002EE2D0C6E90048DFE77B
:1063800002B9FFDEB2FA82F2002A40F09180A1EB5E
:106390000C054FEA1C471FFA8CFE0121B5FBF7F3F1
:1063A00007FB1350250C45EA00450EFB03F0A842FD
:1063B00008D91CEB050503F1FF3802D2A84200F210
:1063C000CB8043462D1AA4B2B5FBF7F007FB10555E
:1063D00044EA05440EFB00FEA64508D91CEB040464
:1063E00000F1FF3502D2A64500F2BB802846A4EB9F
:1063F0000E0440EA03409EE7C1F120078B4022FAD9
:1064000007FC4CEA030C20FA07F405FA01F31C43DD
:10641000FD404FEA1C4900FA01F3B5FBF9F8200CE6
:106420001FFA8CFE09FB185540EA054508FB0EF0E3
:10643000A84202FA01F20BD91CEB050508F1FF3A5C
:1064400080F08880A84240F28580A8F10208654467
:106450002D1AA4B2B5FBF9F009FB105544EA054525
:1064600000FB0EFEAE4508D91CEB050500F1FF341C
:106470006CD2AE456AD90238654440EA0840A0FBB8
:106480000294A5EB0E05A542C846A64656D353D0A6
:106490005EB1B3EB080265EB0E0505FA07F722FAC9
:1064A00001F3CD401F43C6E900750021BDE8F08728
:1064B000C2F1200320FA03F10CFA02FC25FA03F3DF
:1064C00095400D434FEA1C471FFA8CFEB3FBF7F1D2
:1064D00007FB11302B0C43EA004301FB0EF09842FE
:1064E00004FA02F408D91CEB030301F1FF382FD2A0
:1064F00098422DD9023963441B1AADB2B3FBF7F0B1
:1065000007FB103345EA034500FB0EF3AB4208D905
:106510001CEB050500F1FF3816D2AB4214D9023846
:106520006544ED1A40EA014138E73146304607E755
:106530008646E5E61846FAE64B45A9D2B9EB0208CD
:1065400064EB0C0E0138A3E74046EAE7204694E7E7
:106550004146D1E7D0467BE7023B654432E7084637
:1065600009E76444023842E7704700BF034613F866
:10657000012B002AFBD1181A0138704700000000D7
:1065800001F0FF01102A2BDB10F0070F08D010F8E4
:10659000013B013A8B422DD010F0070F42B3F6D1E8
:1065A000F0B441EA012141EA014122F007047FF001
:1065B00000070023F0E80256083C85EA010586EA58
:1065C000010685FA47F5A3FA87F586FA47F6A5FA94
:1065D00087F68EB9EED1F0BC01F0FF0102F00702A0
:1065E00032B110F8013B013A83EA010313B1F8D14B
:1065F0000020704701387047002D06BF354603382C
:10660000073815F0010F07D1013015F4807F02BF64
:10661000013015F4C03F0130F0BC0138704700BFB5
:106620004FEA410C7FEA6C5C02D150EA013C0AD18E
:106630004FEA430C7FEA6C5C02D152EA033C02D180
:106640004FF0000070474FF0010070474FEA4002E2
:106650004FEA41037FEA226C02D15FEA402C08D165
:106660007FEA236C02D15FEA412C02D14FF0000097
:1066700070474FF00100704780B485B000AF78607C
:106680004FF0B0431A6E4FF0B0417B6813430B6676
:106690004FF0B0431A6E7B681340FB60FB6800BF8D
:1066A0001437BD4680BC704780B483B000AF7860BB
:1066B0004FF0B0431A6E7B68DB434FF0B04113409C
:1066C0000B6600BF0C37BD4680BC704780B500AF7D
:1066D000234B244A1A60224B4FF000425A60204B51
:1066E00000229A601E4B0022DA601D4B00221A61C4
:1066F0001B4B04225A611A4B00221A76184B0022B7
:106700005A76174B00229A76154B0122DA61144B08
:10671000002283F82020124B00225A62104B0022E4
:106720009A620F4B002283F82C200D4B4FF48052BD
:106730001A630B4B07225A63094B07229A63084BD3
:10674000002283F83C20064B0022DA64044808F05B
:106750001FFB0346002B01D001F074FA00BF80BD7F
:10676000E40300200024014080B582B000AF7860CF
:106770007B681B68054A934203D14FF40070FFF712
:106780007BFF00BF0837BD4680BD00BF002401402D
:1067900080B582B000AF78607B681B68054A934281
:1067A00003D14FF40070FFF77FFF00BF0837BD46ED
:1067B00080BD00BF0024014080B400AF034B044AF9
:1067C0001A6000BFBD4680BC704700BFE4030020D4
:1067D0000024014080B582B000AF00233B8000233D
:1067E0007B6000F069F803467B802D4800F098F844
:1067F00078602C4B1A882C4B1B889A4226D0294B48
:106800001A88294B1B889A421CD07B887A6802FB25
:1068100003F39B08254AA2FB03235B091A46224B7C
:106820001B88D31A642203FB02F21E4B1B881946F5
:106830001D4B1B88CB1A92FBF3F39BB21E339BB20A
:106840001BB201E047F6FF733B801DE07B887A684E
:1068500003FB02F2164BA3FB0213D21A5208134495
:10686000DB0A4FF47A7202FB03F3A3F53923A3F595
:106870000C63104A82FB03129212DB17D31A9BB2ED
:106880001E339BB21BB23B803B881BB21B021BB268
:106890003B803B881BB218460837BD4680BD00BF11
:1068A000001000B0C875FF1FA875FF1F9F00EE09FC
:1068B00001011000AD8BDB6880B582B000AF002312
:1068C000FB8000233B60134800F02AF838603B68E7
:1068D000002B02D10023FB8016E00F4B1B884FF6E4
:1068E000FF7293420BD00C4B1B881A4640F6E443D0
:1068F00003FB02F23B68B2FBF3F3FB8004E0074AC0
:106900003B68B2FBF3F3FB80FB8818460837BD46B3
:1069100080BD00BF002000B4AA75FF1FD8084C003E
:1069200080B586B000AF786000237B6107F1080373
:1069300000221A605A609A60FFF7C8FE1A4809F0F0
:1069400056F80346002B01D001F07CF97B68BB6050
:106950000023FB6000233B6107F10803194612483E
:1069600008F062FD0346002B01D001F06BF90E48E0
:1069700008F03EFC0346002B01D001F063F94FF014
:10698000FF31094808F0ACFC074808F077FC0648DE
:1069900008F03DFD7861044808F0AEFB7B691846BD
:1069A0001837BD4680BD00BFE403002080B485B029
:1069B00000AF78604FF0B0439A6C4FF0B0417B6805
:1069C00013438B644FF0B0439A6C7B681340FB60B9
:1069D000FB6800BF1437BD4680BC704780B500AF70
:1069E0000420FFF7E3FF0120FFF7E0FF0022022170
:1069F0000F2009F0A2F90F2009F0B9F900BF80BDFE
:106A000080B400AF064B1B6903F40023B3F5002FDD
:106A100001D1012300E000231846BD4680BC704729
:106A20000040005880B58CB000AFF860B9607A6063
:106A30003B600023FB62FB6803F17842564B1B6806
:106A40009902564B0B40B2FBF3F101FB03F3D31A4F
:106A5000DB0ABB61FA687B68134403F17843013BAE
:106A60004D4A126891024D4A0A40B3FBF2F101FB14
:106A700002F29B1ADB0A7B617B68BB62FB687B626C
:106A8000BB683B62BB68002B09D07B6803F007033F
:106A9000002B04D1FB6803F00703002B02D06FF03A
:106AA000040374E03E4B5B69002B02DA6FF00303D2
:106AB0006DE0BA697B699A4205D0FB68C3F30A03AB
:106AC000C3F50063BB62BB69FB615BE07B6AB96ACB
:106AD000184600F0F8F80346002B37D03B68002B2F
:106AE00002D16FF0040352E0FB6903F58033DB024F
:106AF0004FF400621946386820F04AFB7B6AC3F302
:106B00000A033A681344396ABA6A92B2184620F006
:106B10003FFB00220121F86900F065F80346002BD5
:106B200003D06FF00103FB6230E0FB6903F58033B3
:106B3000DB024FF400623968184600F08AF8034619
:106B4000002B10D06FF00203FB621FE03B6ABA6AB1
:106B50001946786A00F07DF80346002B03D06FF0E9
:106B60000203FB6212E07A6ABB6A13447B623A6AF0
:106B7000BB6A13443B627A68BB6AD31ABB62FB6987
:106B80000133FB61FA697B699A429FD9FB6A184617
:106B90003037BD4680BD00BFE075FF1F00FCFF031E
:106BA0000040005880B584B000AFF860C7E900230A
:106BB0000BE000BFFFF724FF0346002BFAD1D7E913
:106BC0000023F968012009F0D9FCFB68D3E9002310
:106BD000D7E90001994208BF9042EAD10023184644
:106BE0001037BD4680BD80B58AB000AFF8600B4657
:106BF0007A607B810223BB61FB68FB617B893B621E
:106C00007B68002B08D007F11803184609F054FEE2
:106C1000034687F827300AE007F1140207F118034A
:106C20001146184609F0F0FD034687F8273097F81B
:106C30002730002B08D097F82730022B01D10123F1
:106C400003E06FF0010300E0002318462837BD463B
:106C500080BD80B58AB000AFF860B9607A60BB686B
:106C60007B6200233B620023FB6120E007F11003FD
:106C70000822796A184620F08BFAD7E90423B3F189
:106C8000FF3F08BFB2F1FF3F05D0D7E90423F86802
:106C9000FFF788FF3862FB680833FB607B6A0833C4
:106CA0007B623B6A002B08D1FB690133FB617B6887
:106CB000DB08FA699A42D9D300E000BF3B6A184664
:106CC0002837BD4680BD80B485B000AF786039609C
:106CD0000AE07B685A1C7A601B78FF2B01D00123E5
:106CE00039E03B68013B3B607B6803F00703002B06
:106CF000EFD17B68FB600023BB6010E0FB6803F111
:106D00000802FA60D3E90023B3F1FF3F08BFB2F1F4
:106D1000FF3F01D001231EE0BB680133BB603B682D
:106D2000DB08BA689A42E9D3BB68DB003A68D31A39
:106D30003B60FB687B600AE07B685A1C7A601B78CA
:106D4000FF2B01D0012306E03B68013B3B603B6821
:106D5000002BF1D1002318461437BD4680BC704784
:106D600080B485B000AF78604FF0B043DA6C4FF07C
:106D7000B0417B681343CB644FF0B043DA6C7B685F
:106D80001340FB60FB6800BF1437BD4680BC7047F2
:106D900080B586B000AF3B1D00221A605A609A6031
:106DA000DA601A610220FFF7DBFF0420FFF7D8FF4B
:106DB0000120FFF7D5FF002208214FF090400AF094
:106DC00084F801224FF400714FF090400AF07DF8F2
:106DD000012201215F480AF078F8012204214FF0D6
:106DE00090400AF072F801224FF400414FF09040B9
:106DF0000AF06BF801224FF4004157480AF065F899
:106E000001224FF4804154480AF05FF801224FF408
:106E1000806151480AF059F8012201214FF0904059
:106E20000AF053F801224FF400714B480AF04DF874
:106E300008237B600123BB600023FB6000233B61D0
:106E40003B1D19464FF0904009F0FAFD4FF40073D6
:106E50007B600123BB600023FB6000233B613B1D83
:106E600019464FF0904009F0EBFD01237B600123B0
:106E7000BB600023FB6000233B613B1D1946354886
:106E800009F0DEFD04237B600123BB600023FB606F
:106E900000233B613B1D19464FF0904009F0D0FDA7
:106EA0004FF400437B600123BB600023FB6002239F
:106EB0003B613B1D19464FF0904009F0C1FD4FF476
:106EC00000437B600123BB600023FB6002233B6126
:106ED0003B1D1946204809F0B3FD4FF400737B6059
:106EE0000123BB600023FB6000233B613B1D19466F
:106EF000194809F0A5FD4FF480437B600123BB6076
:106F00000023FB6000233B613B1D1946124809F03A
:106F100097FD4FF480637B600023BB600123FB601F
:106F200000233B613B1D19460B4809F089FD0123F5
:106F30007B604FF40413BB600123FB6000233B61C3
:106F40003B1D19464FF0904009F07AFD00BF1837FD
:106F5000BD4680BD000800480004004880B586B0EA
:106F600000AF3B1D00221A605A609A60DA601A6115
:106F700008237B600323BB600023FB6000233B618D
:106F80003B1D19464FF0904009F05AFD00BF1837DD
:106F9000BD4680BD80B586B000AF3B1D00221A60A3
:106FA0005A609A60DA601A6108237B600123BB6033
:106FB0000023FB6000233B613B1D19464FF09040CE
:106FC00009F03EFD00BF1837BD4680BD80B483B0D8
:106FD00000AF78604FF0B043D3F8903023F0180240
:106FE0004FF0B0417B681343C1F8903000BF0C37BD
:106FF000BD4680BC704780B485B000AF7860002388
:10700000FB600023BB607B68FB600BE041F6BD23A7
:10701000BB6000BFBB685A1EBA60002BFAD1FB6888
:10702000013BFB60FB68002BF0D100BF00BF1437B1
:10703000BD4680BC7047000080B584B000AF78606A
:107040000023FB7321497868FFF722F80346002BE1
:1070500002D00023FB7333E01D497868FFF718F86E
:107060000346002B02D00123FB7329E019497868FD
:10707000FFF70EF80346002B02D00223FB731FE03C
:1070800015497868FFF704F80346002B02D0032364
:10709000FB7315E011497868FEF7FAFF0346002BF1
:1070A00002D00423FB730BE00D497868FEF7F0FF74
:1070B0000346002B02D00523FB7301E00623FB737C
:1070C000FB7B18461037BD4680BD00BF000048421C
:1070D0000000C842000016430000484300007A4305
:1070E0000000AF43F0B58FB006AF7D4A07F1100343
:1070F00092E8030083E803000023BB600023FB60E9
:1071000007F06AFC00F044FDFFF742FE00F008FFC4
:1071100000F048FF4FF4FA60FFF76DFF06F030FC17
:1071200006F068FC06F051FC0220FFF764FFFF2325
:1071300000935A234FF4947280216A4806F07AFD36
:10714000684806F0C9FDFF2006F0A6FE07F1080317
:10715000184601F01EFA6449644822F09DF80023A5
:107160000193FF230093624B604A0421002007F043
:1071700059F93B7A1E467B7A9C46BB7AFA7A397B70
:10718000787BBC7BFD7B0595049403900291019272
:107190000093634632465749544822F07DF8002355
:1071A0000193FF230093524B504A0421282007F0FB
:1071B00039F951494D4822F06FF800230193FF231C
:1071C00000934B4B494A1621002007F02BF93B7CDA
:1071D0001E467B7C9C46BB7CFA7C397D787DBC7DE1
:1071E000FD7D0595049403900291019200936346FE
:1071F000324640493D4822F04FF800230193FF23D7
:1072000000933B4B394A1621282007F00BF93B49E4
:10721000364822F041F800230193FF230093344BBA
:10722000324A3221002007F0FDF835492F4822F07C
:1072300033F800230193FF2300932D4B2B4A442165
:10724000002007F0EFF8FFF737FB0346BB612D4B3B
:10725000BA692D49254822F01FF800230193FF2326
:107260000093234B214A5A21002007F0DBF8022328
:10727000029301230193002300932D234FF4947272
:107280002D21012006F0FEFE204B0193204B0093A0
:10729000204B214A21494FF0000005F0C9FA03466E
:1072A000BB8097F90430002B0AD000230193FF2301
:1072B00000930F4B1A4A7021002007F0B3F83DE00D
:1072C00097F90530002B2FD000230193FF23009363
:1072D000074B144A7021002007F0A4F82EE000BFED
:1072E00058F902084C04002070F802084C290020CC
:1072F0009000002074F802089CF80208A0F8020828
:10730000B4F80208CCF80208D0F8020805C8000852
:10731000D9C7000855C50008D1C4000851C40008E9
:10732000E4F8020800F9020800230193FF23009308
:10733000974B984A7021002007F074F806F020FB64
:10734000954806F0CBFA06F040FB40F2DC50FFF720
:1073500052FE06F015FBFF2006F09EFD022302936D
:10736000002301930023009380234FF494720121A2
:10737000012006F031FF0123029300230193002333
:10738000009302234FF494720221012006F07AFE4A
:1073900001230293002301930023009301234FF460
:1073A00094720121012006F06DFE01230293002357
:1073B00001930023009320234FF494722021012095
:1073C00006F060FE01230293002301930023009343
:1073D0005A234FF494725A21012006F053FE0123E0
:1073E000029301230193002300932023942201217F
:1073F000942006F047FE012302930123019300230A
:1074000000937F2362225A21622006F03BFE012373
:10741000029301230193002300937F23C5225A2165
:10742000C52006F02FFE01F073F803461A465B4BA9
:107430001A705A4B1B78DBB2184606F0ABFB0023E0
:107440000193FF230093564B002205214FF48270D5
:1074500007F05CF900230193FF230093514B0022B6
:1074600005210A2007F052F900230193FF2300931E
:107470004D4B00222321012007F048F900230193FE
:10748000FF230093494B06222A21F02007F03EF902
:1074900000230193FF230093454B00225C21EC2045
:1074A00007F034F900230193FF230093414B00229E
:1074B0005C210A2007F02AF900230193FF2300939F
:1074C0003D4B00225C216E2007F020F90023019340
:1074D000FF230093394B3A4A03213C2007F0BCF8C4
:1074E00000230193FF230093344B364A0321B0203D
:1074F00007F0B2F800230193FF230093324B334A85
:107500003221582007F0A8F800230193FF230093AD
:107510002D4B2F4A3221A02007F09EF80023019323
:10752000FF230093254B2B4A5E212A2007F094F875
:1075300000230193FF230093204B274A5E219620CE
:1075400007F08AF8144806F0C9F906F03EFA00235D
:10755000FB610BE0104AFB69134419781F4AFB6971
:1075600013440A461A70FB690133FB61FB69B3F5EA
:10757000945FEFDB06F004FA0749184806F010F9AB
:1075800006F023FA02F030F802F036F8FCE700BF0C
:107590009000002014F902084C040020D429002097
:1075A0000801002010010020E00000200001002060
:1075B000F8000020E8000020F000002098000020E3
:1075C0002CF9020834F90208A40000203CF9020852
:1075D00044F9020848F9020850F90208CC160020C4
:1075E000B0B596B004AF0346FB7307F11403184619
:1075F00020F038F8002387F843307E4B0122002129
:1076000002201FF0A7FA7C4B1B78012B2FD1FF2300
:1076100000931D23222205210A2006F06FFC00237F
:107620000193FF230093754B012205210A2007F0E7
:107630006DF80FF0C1FD034687F8433097F94330EA
:10764000002B05D101F08EF803466D4A136004E06B
:107650000FF0B2FD034687F843306A4B0122002148
:1076600002201FF077FA644B02221A706CE0624B22
:107670001B78022B68D1644B1B78DBB2002B27D11F
:1076800001F070F802465E4B1B68019300925F4B5D
:107690000122002102201FF05DFA01F063F802468A
:1076A000574B1B68D31A43F6982293424CD90FF0DC
:1076B00083FD034687F8433001F054F80346504AEF
:1076C0001360534B0122002102201FF043FA3BE0DC
:1076D0003B4618461FF0C6FF07F114033A4692E8EE
:1076E000030083E803007B694A4A934226D97B69F9
:1076F000494A934222D87B6907F11C021146184679
:1077000020F06EF87C6A3D6AFB69BA6AF96A013159
:10771000386B00F26C7003900291019200932B463B
:1077200022463E493E4821F0B7FD3D4B0122002153
:1077300002201FF00FFA304B03221A70394B01223E
:10774000002102201FF006FA374B5B69374A1268A6
:1077500011461846FEF788FC0346002B20D1FF2374
:1077600000935023DC223221A02006F0C7FB2E4BD1
:107770005B691846FEF7AAFC03461A462C492848BE
:1077800021F08AFD00230193FF230093294B244A13
:107790003221A02006F060FF234B5B69234A13606F
:1077A000214BDB68244A126811461846FEF75CFC40
:1077B0000346002B5DD1FF230093782361225E21D5
:1077C000282006F09BFB184BDB684FF000011846A1
:1077D000FEF768FC0346002B32D0134BDB681846DB
:1077E000FDF716FE02460B4614490D4821F054FDE4
:1077F00031E000BF60F902084804002010010020B9
:10780000D029002070F90208CC29002078F902085C
:1078100094F90208682A2A63FF757A96A8F9020883
:107820004C290020D4F90208FC2C0020D829002083
:10783000DCF90208A4000020DC290020E4F9020899
:10784000A74BDB681846FDF7E3FD02460B46A5494A
:10785000A54821F021FD00230193FF230093A34BB2
:10786000A14A5E212A2006F0F7FE9D4BDB68A04A64
:1078700013609B4B1B699F4A126811461846FEF71E
:10788000F3FB0346002B20D1FF2300937D23C4226A
:107890005E21962006F032FB914B1B691846FDF7DE
:1078A000B7FD02460B468F498F4821F0F5FC0023B7
:1078B0000193FF2300938D4B8B4A5E21962006F0A7
:1078C000CBFE874B1B698B4A13608B4B1B6818469A
:1078D000FFF7B2FB03461A46884B1B689A421DD03D
:1078E000854B1B681846FFF7A7FB03461A46834BD8
:1078F0001A60FF2300934E234FF48A722A21F0204E
:1079000006F0FCFA7D4B1B68DAB200230193FF23DB
:1079100000937B4B2A21F02006F0F8FE704B1B7978
:107920001A46784B1B689A4219D06D4B1B791A4640
:10793000744B1A60FF2300937C234FF486725C2102
:10794000EC2006F0DBFA6F4B1B68DAB200230193E0
:10795000FF2300936C4B5C21EC2006F0D7FE6B4BB1
:107960001B78DBB21A466A4B1B689A4229D0674BD8
:107970001B78DBB21846FEF78BF90346584A1360B2
:10798000624B1B78DBB2184606F004F9FF23009324
:107990001D2340F2111205214FF4827006F0AEFA59
:1079A00000230193FF2300935A4B002205214FF43B
:1079B000827006F0ABFE554B1B78DBB21A46544B77
:1079C0001A60554B1B78032B43D13B4618461FF0DA
:1079D00049FE07F114033A4692E8030083E80300E6
:1079E0007B6907F11C02114618461FF0F9FEFF23C0
:1079F00000931F23822203213C2006F07FFAFB6ABA
:107A00005A1CBB6A4549384821F046FC00230193C3
:107A1000FF230093354B344A03213C2006F01CFE23
:107A2000FF2300931F23F6220321B02006F066FAFD
:107A30007B6A9A1C3B6A3A492B4821F02DFC0023B3
:107A40000193FF230093294B274A0321B02006F01E
:107A500003FE05F095FF334B1B780133DAB2314B4F
:107A60001A70314B1B780133DAB22F4B1A702E4B40
:107A70001B78782B04D82D4B1B78DBB2012B27D138
:107A80002A4B1B78DBB2012B02D1284B02221A7041
:107A9000274B01221A70274805F020FF00237B6442
:107AA0000BE0244A7B6C13441978234A7B6C134403
:107AB0000A461A707B6C01337B647B6CB3F5945F70
:107AC000EFDB194B00221A70194B00221A7047E0A5
:107AD000144B1B78092B33D8184B01221A7035E050
:107AE000FC2C0020ECF902084C2900209800002012
:107AF000DC290020E0290020D829002000000020F7
:107B000000010020E4290020F8000020D4290020F2
:107B1000E82900200801002048040020F4F90208A8
:107B200000FA0208EC290020ED2900201F2D00207A
:107B30001E2D00204C040020CC1600204C310020CB
:107B40000D4B00221A700D4B00221A700C4B0122B3
:107B50001A700C490C4805F023FE094B00221A70DC
:107B600005F033FF094B0122002102201EF0F2FF35
:107B700000BF4837BD46B0BDEC2900204C31002085
:107B80001E2D00204C040020CC1600200CFA020808
:107B900080B59AB000AF07F12003482200211846B3
:107BA00020F006FD07F1080300221A605A609A606F
:107BB000DA601A615A6109F0B7F90020FFF706FA96
:107BC0001F4B1B6823F4C0631D4A43F4007313600A
:107BD0001B4B1B6803F4C0637B607B6824233B6200
:107BE0008123FB6201233B6400237B64B023BB64DD
:107BF0000023FB6407F12003184609F0E1FC03466B
:107C0000002B01D000F01EF84F23BB600023FB6067
:107C100000233B6100237B610023BB610023FB61E8
:107C200007F10803022118460AF066F80346002B04
:107C300001D000F007F800BF6837BD4680BD00BF27
:107C40000004005880B400AF72B600BFFEE780B4F5
:107C500000AF4FF0B043D3F890304FF0B04243F450
:107C60000043C2F8903000BFBD4680BC704780B46E
:107C700085B000AF78604FF0B0439A6D4FF0B041DF
:107C80007B6813438B654FF0B0439A6D7B6813405C
:107C9000FB60FB6800BF1437BD4680BC7047000026
:107CA00080B58CB000AF3B1D2C220021184620F07F
:107CB0007FFC224B224A1A60204B1F229A601F4BE6
:107CC00000221A611D4B00225A611C4B00229A614E
:107CD0001A4B4FF08042DA61184B00221A62174BA0
:107CE0004FF480725A6215480AF0C2FC0346002B1A
:107CF00001D0FFF7A7FF11480AF0B0FF0346002BA1
:107D000001D0FFF79FFF00233B620023BB600023ED
:107D1000BB614FF00053FB614FF48073FB623B1D6E
:107D20000022194605480AF01DFD0346002B01D02C
:107D3000FFF788FF00BF3037BD4680BDF029002027
:107D40000028004080B590B000AF786007F10803CC
:107D500038220021184620F02BFC7B681B68164A4D
:107D6000934225D14FF48033BB604FF48073FB63A3
:107D700007F1080318460AF061FB0346002B01D007
:107D8000FFF760FFFFF763FF4FF48060FFF76FFFBF
:107D900000220021022007F0D0FF022007F0E7FFB9
:107DA000002200212A2007F0C8FF2A2007F0DFFF69
:107DB00000BF4037BD4680BD0028004080B485B07C
:107DC00000AF78604FF0B043DA6C4FF0B0417B68A1
:107DD0001343CB644FF0B043DA6C7B681340FB6015
:107DE000FB6800BF1437BD4680BC704780B485B0C7
:107DF00000AF78604FF0B0439A6D4FF0B0417B68B0
:107E000013438B654FF0B0439A6D7B681340FB6062
:107E1000FB6800BF1437BD4680BC704780B483B098
:107E200000AF78604FF0B0439A6D7B68DB434FF052
:107E3000B04113408B6500BF0C37BD4680BC704716
:107E400080B483B000AF78604FF0B0439A6B4FF0CE
:107E5000B0417B6813438B6300BF0C37BD4680BCC9
:107E6000704780B483B000AF78604FF0B0439A6B36
:107E70007B68DB434FF0B04113408B6300BF0C378E
:107E8000BD4680BC704780B485B000AF78604FF0CD
:107E9000B0431A6E4FF0B0417B6813430B664FF04E
:107EA000B0431A6E7B681340FB60FB6800BF143759
:107EB000BD4680BC704780B483B000AF78604FF09F
:107EC000B0431A6E7B68DB434FF0B04113400B6642
:107ED00000BF0C37BD4680BC704780B483B000AF94
:107EE00078604FF0B0431A6C4FF0B0417B68134399
:107EF0000B6400BF0C37BD4680BC704780B483B0B4
:107F000000AF78604FF0B0431A6C7B68DB434FF0F2
:107F1000B04113400B6400BF0C37BD4680BC7047B6
:107F200080B500AF4FF48050FFF7ADFF1B4B1C4AEC
:107F30001A601A4B4FF482725A60184B00229A60F2
:107F4000164B4FF4E062DA60144B00221A61134BB7
:107F500000225A61114B4FF400729A610F4B1822A4
:107F6000DA610E4B00221A620C4B00225A620B4B54
:107F700000229A62094B0722DA62084B00221A6338
:107F8000064B00225A6305480AF0F6FE0346002B12
:107F900001D0FFF757FE00BF80BD00BF282A002098
:107FA0000030014080B500AF4FF48040FFF71EFF66
:107FB0001B4B1C4A1A601A4B4FF482725A60184BC2
:107FC0004FF440429A60164B4FF4E062DA60144B73
:107FD00000221A61124B00225A61114B4FF40072B9
:107FE0009A610F4B3022DA610D4B00221A620C4B62
:107FF00000225A620A4B00229A62094B0722DA6277
:10800000074B00221A63064B08225A6304480AF001
:10801000B3FE0346002B01D0FFF714FE00BF80BD66
:108020008C2A00200038004080B596B000AF786000
:1080300007F1440300221A605A609A60DA601A61FC
:1080400007F10C0338220021184620F0B1FA7B68B2
:108050001B682F4A934217D14FF48050FFF713FF4C
:108060000220FFF7ABFE38237B640223BB640023AE
:10807000FB6402233B6505237B6507F14403194636
:10808000244808F0DDFC3EE07B681B68224A9342EE
:1080900039D11023FB604FF40073BB6107F10C036F
:1080A00018460AF0CBF90346002B01D0FFF7CAFDB2
:1080B0004FF48040FFF79AFE0220FFF77FFE042076
:1080C000FFF77CFE4FF400537B640223BB64002364
:1080D000FB6402233B6505237B6507F144031946D6
:1080E0000C4808F0ADFC02237B640223BB64002330
:1080F000FB6402233B6503237B6507F144031946B8
:10810000064808F09DFC00BF5837BD4680BD00BF43
:1081100000300140000400480038004000080048DA
:1081200080B588B000AF786007F10C0300221A60B8
:108130005A609A60DA601A617B681B683F4A934212
:108140002FD13F480BF060FB4FF48050FFF7C5FE86
:108150004FF48050FFF7D2FE4FF48050FFF7ABFE94
:108160007B68002283F85D2000223821354808F022
:10817000ACFE3821334808F0C3FD002238213148D5
:1081800008F0A3FE3823FB6001233B6100237B61E1
:108190000223BB6107F10C0319462A4808F050FC82
:1081A00048E07B681B68284A934243D127480BF07C
:1081B0002BFB4FF48040FFF743FE4FF48040FFF766
:1081C00050FE4FF48040FFF729FE7B68002283F8C1
:1081D0005D204FF408511B4808F092FD02211C4815
:1081E00008F08EFD00224FF40851164808F06DFE8D
:1081F0004FF40853FB6001233B6100237B610223A2
:10820000BB6107F10C0319460E4808F019FC002267
:1082100002210F4808F059FE0223FB6001233B6155
:1082200000237B610223BB6107F10C031946084858
:1082300008F006FC00BF2037BD4680BD003001407D
:10824000282A002000040048003800408C2A002022
:108250000008004880B400AF034B0122C3F8882017
:1082600000BFBD4680BC70470004005880B400AF1A
:1082700000BFBD4680BC704780B400AF00BFBD46A4
:1082800080BC704780B500AF06F0C6FBFFF7E2FF89
:10829000FEF764FE0548FFF743FF0548FFF740FF80
:1082A000012008F0D3FE00BF80BD00BF282A0020B7
:1082B0008C2A002080B500AF06F0BCFB00F0A8FFC0
:1082C000FFF72EFE00BF80BD80B500AF06F0A4FB17
:1082D0000121002008F036FE00BF80BD80B500AF50
:1082E00006F0A8FB00BF80BD80B400AF00BFBD4654
:1082F00080BC704780B400AFFEE780B400AFFEE7FB
:1083000080B400AFFEE780B400AFFEE780B400AFFA
:10831000FEE780B400AF00BFBD4680BC704780B4AC
:1083200000AF00BFBD4680BC704780B400AF00BF47
:10833000BD4680BC704780B400AF00BFBD4680BC66
:108340007047000080B500AF02480AF0C3FC00BFD0
:1083500080BD00BFF029002080B500AF012008F0EB
:10836000CBFD00BF80BD80B400AF00BFBD4680BC68
:10837000704780B400AF00BFBD4680BC70470000AE
:1083800080B500AF024807F089FF00BF80BD00BF85
:108390009C2B002080B500AF02480CF0C9FB00BF49
:1083A00080BD00BF0C2B002080B500AF02480AF052
:1083B00041FB00BF80BD00BFF029002080B500AFA9
:1083C00002480CF0BDF800BF80BD00BFF02A0020BD
:1083D00080B485B000AF78604FF0B0435A6E4FF074
:1083E000B0417B6813434B664FF0B0435A6E7B68D5
:1083F0001340FB60FB6800BF1437BD4680BC70476C
:1084000080B500AF064B08221A6005480BF01CFE31
:108410000346002B01D0FFF715FC00BF80BD00BF55
:10842000F02A002080B582B000AF78600120FFF70D
:10843000CFFF00220021322007F07FFC322007F01E
:1084400096FC00BF0837BD4680BD80B483B000AF46
:1084500078604FF0B0439B6823F400424FF0B04186
:108460007B6813438B6000BF0C37BD4680BC7047F0
:1084700080B400AF024B1B681846BD4680BC7047F5
:108480008075FF1F80B400AF034B1B68DBB218463A
:10849000BD4680BC704700BF8475FF1F80B400AF2D
:1084A000034B1B681B0A1846BD4680BC704700BFC3
:1084B0008475FF1F80B500AF0020FFF7C6FF1FF0D7
:1084C00045FB0D4B01221A701EF016FB0B481EF0E7
:1084D000C1FB0B4B4FF400421A6102201EF0C8FB97
:1084E000FEF76AF900F094F91EF0ACFD01210120BD
:1084F0001EF0E8FD00BF80BDFC2A0020C5860008F4
:108500000040005880B500AF1EF00CFE00BF80BDDB
:1085100080B582B000AF0023FB71FEF7CDF90346B2
:10852000BB80BB8840F6B832934202D96423FB710A
:1085300012E0BB88B3F5FA6F02D20023FB710BE0A7
:10854000BB88A3F5FA631A46642302FB03F3054ACA
:10855000A2FB03239B09FB71FB7918460837BD4634
:1085600080BD00BFD34D621080B588B000AF00233E
:10857000FB833B1D184600F019F9BB681846FDF750
:10858000A5FD0346FB83B7F91E3018462037BD46CC
:1085900080BD90B587B000AF786000237B61FFF7A6
:1085A00067FF78617B69B3F1FF3F38D106F050FA7D
:1085B000044606F061FA034623443B6106F052FA92
:1085C000F8603B691A0E7B680733D2B21A703B69B8
:1085D0001A0C7B680633D2B21A703B691A0A7B68A0
:1085E0000533D2B21A707B6804333A69D2B21A707A
:1085F000FB681A0E7B680333D2B21A70FB681A0C40
:108600007B680233D2B21A70FB681A0A7B680133A6
:10861000D2B21A70FB68DAB27B681A7031E07B68FC
:1086200007337A69D2B21A707B691A0A7B680633FB
:10863000D2B21A707B691A0C7B680533D2B21A70F9
:108640007B691A0E7B680433D2B21A70FFF71AFFE7
:1086500078617B6803337A69D2B21A70FFF71EFF24
:1086600078617B6802337A69D2B21A707B691A0A20
:108670007B680133D2B21A707B691B0CDAB27B685B
:108680001A7000BF1C37BD4690BD90B583B000AFD7
:1086900000237B60FFF7ECFE78607B68B3F1FF3F5F
:1086A0000BD106F0D5F9044606F0DCF903465C4030
:1086B00006F0E2F9034663407B607B6818460C379E
:1086C000BD4690BD80B586B002AF7860396007F1D5
:1086D000080318461EF0C6FFBB68B7F90C200092CD
:1086E000074A1021786800F01DF87868FDF73EFF12
:1086F00003469AB23B681A8000BF1037BD4680BD62
:108700001CFA020880B500AF012102201EF0AAFC6D
:1087100000BF80BD80B500AF002102201EF0A2FC8A
:1087200000BF80BD0CB480B584B000AF7860396004
:1087300007F11C03FB603968FB68BA6978681FF0B1
:10874000A9FD00BF1037BD46BDE8804002B07047AC
:1087500080B483B000AF7860002318460C37BD4664
:1087600080BC704780B582B000AF00237B60074BB0
:108770001B78002B02D1064B1B6803E000F0D0F9F8
:1087800078607B6818460837BD4680BDFC2A00200B
:108790006831002080B582B000AF78607B681846F1
:1087A00000F045FA00BF0837BD4680BD80B586B0F1
:1087B00000AF7860114B7B61114B3B61114BFB604B
:1087C000FEF708F803461B121BB21846FDF764FAC1
:1087D00003463B617B687A699A607B683A695A60B4
:1087E0007B68FA681A607B68074ADA607B68074A28
:1087F0001A61002318461837BD4680BD0000484264
:108800000000904100007A440D093E00AB030500D2
:1088100080B483B000AF00237B607B6818460C37C0
:10882000BD4680BC704780B400AF01231846BD46EA
:1088300080BC704780B582B000AF786039601FF0AF
:108840007FFE034616221A604FF0FF3318460837A2
:10885000BD4680BD80B582B000AF78604FF0FF317B
:108860007868FFF7E7FFFEE780B586B000AFF860F5
:10887000B9607A6000237B610AE0AFF300800146B3
:10888000BB685A1CBA60CAB21A707B6901337B613B
:108890007A697B689A42F0DB7B6818461837BD46D8
:1088A00080BD80B586B000AFF860B9607A60002303
:1088B0007B6109E0BB685A1CBA601B781846AFF3AD
:1088C00000807B6901337B617A697B689A42F1DBC6
:1088D0007B6818461837BD4680BD80B483B000AFB2
:1088E00078604FF0FF3318460C37BD4680BC7047A8
:1088F00080B483B000AF786039603B684FF40052B9
:108900005A60002318460C37BD4680BC704780B4BF
:1089100083B000AF7860012318460C37BD4680BC99
:10892000704780B485B000AFF860B9607A6000230A
:1089300018461437BD4680BC7047000080B586B02D
:1089400000AF7860144A154BD31A7B617B693B6199
:10895000134B1B68002B02D1114B124A1A60104BAB
:108960001A687B6813443A699A4207D21FF0E8FDFF
:1089700003460C221A604FF0FF3309E0084B1B68D6
:10898000FB60074B1A687B681344054A1360FB6859
:1089900018461837BD4680BD00800020001000003A
:1089A000002B0020D854002080B483B000AF786042
:1089B0007B689B6818460C37BD4680BC704700003A
:1089C00080B582B000AF0023FB71144B1B7883F09D
:1089D0000103DBB2002B1BD0114B4FF0FF321A63A7
:1089E000FFF75EF900F056F84FF480710C4809F07B
:1089F000C5FF0B4B4FF0FF321A6309480AF0FCF831
:108A0000002000F0D3F900F05FF8044B01221A7047
:108A1000FB7918460837BD4680BD00BF042B0020F7
:108A2000F029002080B58EB000AF7860002387F871
:108A3000373007F108032C22002118461FF0B8FD3B
:108A400000F028F8114B1B687A6813447B60002300
:108A50007B627B68DB43FB600023FB614FF00053CC
:108A60003B624FF480733B6307F108030122194610
:108A7000074809F077FE0346002B01D0FFF7E2F824
:108A800097F8373018463837BD4680BD082B002090
:108A9000F029002080B582B000AF0023FB71084BA5
:108AA0000122DA654FF48071064809F067FF054B33
:108AB0004FF0FF321A63FB7918460837BD4680BD78
:108AC00000280040F029002080B500AF00F08EF9AA
:108AD0000346034A1360024B1B68184680BD00BF63
:108AE000082B002080B400AF024B1B681846BD461F
:108AF00080BC7047082B002080B582B000AF0023F7
:108B00007B6000F073F90246044B1B68D31A7B604C
:108B10007B6818460837BD4680BD00BF082B002083
:108B200080B582B000AF00237B60064B1B78002B22
:108B300002D000F05BF978607B6818460837BD46C4
:108B400080BD00BF042B002080B483B000AF0023A1
:108B50007B6003237B607B6818460C37BD4680BC76
:108B60007047B0B584B000AF78600021F9607968D3
:108B700000200A460346950D94024FF47A724FF096
:108B8000000320462946FDF737FB02460B461346F5
:108B9000FB60FB6818461037BD46B0BD2DE9B00F2D
:108BA00085B000AF78600021F960796800200C463C
:108BB0000546204629464FF0000A4FF0000B4FEAC9
:108BC000411B4BEAD06B4FEA401A50465946021BF4
:108BD00061EB05034FF000004FF00001990041EAFE
:108BE0009271900002460B4612EB040843EB050914
:108BF0004FF000024FF000034FEAC90343EA5873F5
:108C00004FEAC80290469946404649464FF0000256
:108C10004FF00003820A42EA81528B0A1346FB603E
:108C2000FB6818461437BD46BDE8B00F704780B5E5
:108C300084B000AF78607868FFF793FFF86000F0C9
:108C4000D5F8B86000E000BF00F0D0F80246BB687D
:108C5000D31AFA689A42F6D800BF00BF1037BD4653
:108C600080BD80B582B000AF78601FF0BDF800BF56
:108C70000837BD4680BD80B584B000AF786000F095
:108C8000A5F8F860FB680133184600F08FF800BFC4
:108C90001037BD4680BD2DE9B04F8CB000AF786174
:108CA0000023FB6200F0A2F8B86200F08FF878624F
:108CB0007B6A0022BB60FA604FF000024FF00003B5
:108CC000B9680B000022B96A00200C46054612EB79
:108CD000040843EB0509C7E90689D7E906014FF007
:108CE00000024FF00003820A42EA81528B0A1346C7
:108CF000FB62BB6900223B607A603B68C3F3090AF0
:108D00004FF0000BC7E906ABBB691846FFF746FFFB
:108D100003469AB27B691A80FB6A18463037BD4613
:108D2000BDE8B08F80B582B000AF78607A6800216E
:108D3000034809F0F3FF00BF0837BD4680BD00BF00
:108D4000F029002080B582B000AF78607A680121F8
:108D5000034809F0E3FF00BF0837BD4680BD00BFF0
:108D6000F029002080B582B000AF00237B60002195
:108D7000044809F0EBFF78607B6818460837BD4669
:108D800080BD00BFF029002080B582B000AF002375
:108D90007B600121044809F0D9FF78607B681846A0
:108DA0000837BD4680BD00BFF029002080B582B0E5
:108DB00000AF78607A680221034809F0AFFF00BF76
:108DC0000837BD4680BD00BFF029002080B582B0C5
:108DD00000AF0221044809F0B9FF78607B681846AB
:108DE0000837BD4680BD00BFF029002080B582B0A5
:108DF00000AF0B48FFF7D8FD786003E00848FFF7A5
:108E0000D3FD78600648FFF7CFFD02467B689342AA
:108E1000F4D17B68DB4318460837BD4680BD00BFF0
:108E20000028004080B485B000AF78604FF0B043B8
:108E3000DA6C4FF0B0417B681343CB644FF0B04322
:108E4000DA6C7B681340FB60FB6800BF1437BD46DB
:108E500080BC704780B485B000AF78604FF0B043FD
:108E60001A6E4FF0B0417B6813430B664FF0B0436E
:108E70001A6E7B681340FB60FB6800BF1437BD4669
:108E800080BC704780B483B000AF78604FF0B043CF
:108E90001A6E7B68DB434FF0B04113400B6600BF96
:108EA0000C37BD4680BC704780B500AF224B234ACB
:108EB0001A60214B4FF4E1325A601F4B00229A6036
:108EC0001D4B0022DA601C4B00221A611A4B0C2247
:108ED0005A61194B00229A61174B0022DA61164B36
:108EE00000221A62144B00225A62134B00229A622B
:108EF00011480BF0E4FC0346002B01D0FEF7A2FE64
:108F000000210D480DF05BFD0346002B01D0FEF75C
:108F100099FE002108480DF090FD0346002B01D07A
:108F2000FEF790FE04480DF00FFD0346002B01D024
:108F3000FEF788FE00BF80BD0C2B002000380140EA
:108F400080B596B000AF786007F1440300221A6044
:108F50005A609A60DA601A6107F10C033822002126
:108F600018461FF025FB7B681B68384A934268D17E
:108F70000123FB60364B3B6107F10C03184609F0F7
:108F80005DFA0346002B01D0FEF75CFE4FF48040F3
:108F9000FFF760FF0220FFF745FF40237B640223B9
:108FA000BB640023FB6403233B6507237B6507F158
:108FB00044031946274807F043FD80237B640323BD
:108FC000BB640023FB6400233B6507F1440319469F
:108FD000204807F035FD002280211E4807F075FF6C
:108FE0001D4B1E4A1A601C4B12225A601A4B10224B
:108FF0009A60194B0022DA60174B80221A61164BD7
:1090000000225A61144B00229A61134B0022DA614C
:10901000114B00221A62104806F0C6FE0346002BD0
:1090200001D0FEF70FFE7B680B4A9A670A4A7B68FD
:10903000936200220221242006F07FFE242006F005
:1090400096FE00BF5837BD4680BD00BF00380140C6
:1090500001000300000400489C2B0020580002403F
:1090600080B582B000AF78607B681B680B4A934282
:109070000FD14FF48040FFF705FFC021084807F0EB
:109080003FFE7B689B6F184606F036FF242006F0F3
:109090007CFE00BF0837BD4680BD00BF00380140E0
:1090A0000004004880B483B000AF78604FF0B04354
:1090B0001A6C4FF0B0417B6813430B6400BF0C3750
:1090C000BD4680BC704780B483B000AF78604FF07D
:1090D000B0431A6C7B68DB434FF0B04113400B6424
:1090E00000BF0C37BD4680BC7047000080B483B021
:1090F00000AF7860064BD3F8802005497B681343A6
:10910000C1F8803000BF0C37BD4680BC704700BF3F
:109110000008005880B582B000AF7860074A7B68CD
:109120001360FDF75BFCFFF7BFFE4FF00060FFF739
:10913000DDFF002318460837BD4680BD002C002007
:1091400080B500AF4FF48040FFF7ACFF4FF4804094
:10915000FFF7B9FF0448FFF783FF0F2006F015FE65
:109160000023184680BD00BF0C2B002080B582B0C4
:1091700000AF78600B467B807B881A46796804488C
:109180000BF044FC002318460837BD4680BD00BFE5
:109190000C2B002080B584B000AF7860194A7B6842
:1091A00013604FF40013BB6007F1080393E8060057
:1091B00015480DF03CFB00BF134B1B68DB6903F443
:1091C0008033B3F5803FF7D000BF0F4B1B68DB69DE
:1091D00003F48003B3F5800FF7D10B4B1B689A683B
:1091E000094B1B6842F480029A6007480DF07AFB35
:1091F0000122064904480BF0B3FB00231846103740
:10920000BD4680BD042C00200C2B0020FC2B002030
:1092100080B500AF08480BF052FB0346002B01D08D
:10922000FEF710FD054806F0BFFD0346002B01D0F8
:10923000FEF708FD00BF80BD0C2B00209C2B0020FA
:1092400080B582B000AF7860034B1B680020984760
:1092500000BF0837BD4680BD002C002080B582B01D
:1092600000AF78600B4B1B68002B0AD07B68D3F8EB
:109270008C30002B05D1074B1B68002201210648CA
:1092800098470122044978680BF06AFB00BF083751
:10929000BD4680BD042C0020FC2B002080B400AF14
:1092A000034B00221A7000BFBD4680BC704700BF50
:1092B000FA2C002080B400AF024B1B781846BD4644
:1092C00080BC7047FA2C002080B582B000AF786077
:1092D000064B1B789BB21A46054978681DF058FF6B
:1092E000024B1B7818460837BD4680BDFA2C00207B
:1092F000082C002080B483B000AF03460A46FB71FF
:109300001346BB801C4B1B78EE2B01D900232DE0AC
:10931000194B1B785A1CD1B2174A11701946174ABB
:10932000FB795354144B1B785A1CD1B2124A11705A
:109330001A46124B65219954BB881B0A99B20E4BF1
:109340001B785A1CD0B20C4A10701A46C9B20B4B8B
:109350009954094B1B785A1CD1B2074A11701A460E
:10936000BB88D9B2054B9954034B1B7818460C3770
:10937000BD4680BC704700BFFA2C0020082C00209E
:1093800080B584B000AF03463960FB71214B1B7878
:10939000EE2B01D9002338E01F493868FCF7D0FCD8
:1093A00003461846FCF792FE0346FB81194B1B78D7
:1093B0005A1CD1B2174A11701946184AFB795354F6
:1093C000144B1B785A1CD1B2124A11701A46134B17
:1093D00067219954B7F90E301B1219B20D4B1B7847
:1093E0005A1CD0B20B4A10701A46C9B20B4B995492
:1093F000084B1B785A1CD1B2064A11701A46FB89D9
:10940000D9B2064B9954034B1B7818461037BD460A
:1094100080BD00BFFA2C002000002041082C002055
:1094200090B583B000AF03463960FB71194B1B78D0
:10943000EF2B01D9002329E0164B1B785A1CD1B21F
:10944000144A11701946144AFB795354114B1B7876
:109450005A1CD1B20F4A11701A460F4B6821995409
:109460003B6819461846FCF763FB03461846094B50
:109470001B785A1CD1B2074A11701C46FCF74CFEEF
:109480000346DAB2044B1A55024B1B7818460C37C8
:10949000BD4690BDFA2C0020082C002080B584B079
:1094A00000AF03463960FB71214B1B78EE2B01D9CD
:1094B000002338E01F493868FCF742FC0346184691
:1094C000FCF704FE0346FB81194B1B785A1CD1B2F2
:1094D000174A11701946184AFB795354144B1B78DC
:1094E0005A1CD1B2124A11701A46134B7321995467
:1094F000B7F90E301B1219B20D4B1B785A1CD0B2A3
:109500000B4A10701A46C9B20B4B9954084B1B7882
:109510005A1CD1B2064A11701A46FB89D9B2064BC1
:109520009954034B1B7818461037BD4680BD00BFC9
:10953000FA2C002000002041082C002080B584B0C7
:1095400000AF03463960FB71254B1B78ED2B01D929
:10955000002341E03868FCF7B9FD0346FB60FB6877
:1095600023F07F43FB601E4B1B785A1CD1B21C4A70
:10957000117019461B4AFB795354194B1B785A1C1E
:10958000D1B2174A11701A46164B7D219954FB68C7
:109590001914134B1B785A1CD0B2114A10701A467A
:1095A000C9B2104B9954FB6819120D4B1B785A1C09
:1095B000D0B20B4A10701A46C9B20A4B9954084BE4
:1095C0001B785A1CD1B2064A11701A46FB68D9B2F0
:1095D000044B9954024B1B7818461037BD4680BD8A
:1095E000FA2C0020082C002080B500AFFEF762FFA7
:1095F00000F020F800BF80BD80B500AF4FF0FF3015
:109600001DF000FE00BF80BD80B400AFBFF34F8FE0
:1096100000BF064BDB6803F4E0620449044B1343CC
:10962000CB60BFF34F8F00BF00BFFDE700ED00E050
:109630000400FA0580B586B004AF00237B600023E8
:1096400002930223019301230093594B002200212E
:1096500002201DF07FFA00230293042301930223CA
:109660000093544B0022002102201DF073FA0023C6
:10967000029302230193012300934F4B0022002108
:1096800002201DF067FA3B1D194600200EF078F904
:109690007B681B0EDBB21A467B681B0CDBB21946DB
:1096A0007B681B0ADBB2029301910092434B0022BC
:1096B000002102201DF04EFA3B1D194601200EF03C
:1096C0005FF97B681B0EDBB21A467B681B0CDBB2B2
:1096D00019467B681B0ADBB27868C0B2039002931C
:1096E00001910092364B0022002102201DF032FA37
:1096F00000230093334B002240F6B83132481EF06D
:1097000035FA00230093314B01224DF6C021304839
:109710001EF02CFA002300932E4B00224FF4FA6126
:109720002D481EF023FA2D4A002101201DF066FE6F
:109730002B4A002102201DF061FE2A4A002104204C
:109740001DF05CFE284A002108201DF057FE274A24
:10975000002110201DF052FE00F002FD4FF081713B
:1097600023480DF017FA23480DF060FA16481EF052
:1097700033FA17481EF030FA1F4B1B781F4A127835
:10978000114618460DF0A4FB1D4B1B78002B0BD186
:109790001C4B1968002300931B4B00221B481EF032
:1097A000E5F91A481EF018FA00BF0837BD4680BD1B
:1097B00048FA02086CFA020890FA0208B4FA0208A1
:1097C000D8FA02088D9B0008642E00206D9C0008CA
:1097D0007C2E002029A00008402D0020AD6E01083D
:1097E0004D9900084DA00008A99F0008919C000811
:1097F000200000206C0000201C000020252D0020EF
:10980000262D002080000020699B0008282D0020C4
:1098100080B483B000AF0346FB8000BF0C37BD4669
:1098200080BC7047B0B58AB006AF7860396000235D
:10983000FB733B68002B7AD03B681B78002B4DD024
:109840007B68002B4AD07B681B78FB737B685B6866
:10985000002B43D07B681B78022B21D0032B3FD1F8
:109860007B685B78012B17D17B685B681B78022BC8
:109870000ED0022B12DC002B02D0012B04D00DE005
:1098800000200DF0C1FC0AE001200DF0BDFC06E057
:1098900002200DF0B9FC02E000BF24E000BF22E08E
:1098A0007B685B78012B1DD17B685B681B7803F0BC
:1098B0000103DAB2204B1A701F4B1B78002B06D124
:1098C0001E4B0022002103201DF044F90AE01C4B2E
:1098D0000022002103201DF03DF903E000BF02E05B
:1098E00000BF00E000BF3B681B7C052B1FD83B6816
:1098F000DB68FA7B396891F908100C463968097CF5
:109900000846104951F82010386890F909000546BA
:10991000386890F90A000590049503910294019229
:109920000093094B0022002103201DF013F900BF12
:109930001037BD46B0BD00BF4A2E0020FCFA020819
:1099400008FB02080400002014FB020890B587B051
:1099500002AFFF23FB720023FB60FEF703FF78607A
:109960000023FB706E4B1B78DBB200936D4B012222
:10997000002102201DF0EEF86B4B02221A70FFF757
:109980008DFCFC78631CFB70684B9B68684918462B
:10999000FCF78AFA034619462046FFF77FFDFB785D
:1099A0005A1CFA70614AD26811461846FFF7E8FC63
:1099B000FB785A1CFA705D4A126911461846FFF787
:1099C0002FFDFC78631CFB70584B5B6959491846A6
:1099D000FCF7B6F9034619462046FFF7AFFDFC78C1
:1099E000631CFB70514B9B6952491846FCF7A8F960
:1099F000034619462046FFF7A1FDFB785A1CFA7072
:109A00004A4A127992B211461846FFF773FCFB7866
:109A10005A1CFA70424A1278D2B292B211461846D3
:109A2000FFF768FC444B1B78082B02D0424B1B7895
:109A3000012B3D4B5B681846FFF746FCFFF73AFCED
:109A400003461A46384B5A7017E0FEF78BFE024663
:109A50007B68D31AB3F5FA6F06D9384B012200217F
:109A600002201DF077F812E0354B01220021022080
:109A70001DF070F80120FDF7BEFA324B1B78DBB207
:109A8000002BE2D1304B1B78DBB2002BDDD12A4B0F
:109A9000DB780022194624480DF0B6FA0346FB7223
:109AA00097F90B30002B0BD1284B1B680133274A49
:109AB0001360274B0122002101201DF04BF816E016
:109AC00097F90B3013F1060F11D10DF0F7F9F8608B
:109AD000FB68002B0BD0FB681E4AA2FB03239B09EB
:109AE00000931D4B0122002101201DF033F81B4B78
:109AF0001B78002B0FD11A481EF0DCF8194B1A689E
:109B0000FB68934238BF1346194615481EF042F9C8
:109B100013481EF061F800BF1437BD4690BD00BF6A
:109B2000D42900205CFB020884000020FC2C0020CB
:109B30000000C84200007A446C00002068FB020864
:109B400080FB02081D2D00201E2D0020202D00204E
:109B50009CFB0208D34D6210ACFB0208262D0020AE
:109B6000282D00208000002080B582B000AF7860F2
:109B7000002102201DF064FC03481EF02DF800BFF8
:109B80000837BD4680BD00BF282D002080B582B0BB
:109B900000AF78602B4B1B78002B05D1FEF7B8FC8B
:109BA00003461A46284B1A70264B1B780133DAB24B
:109BB000244B1A70234B1B78132B10D9214B0022F6
:109BC0001A70FDF7E7F9002208214FF0904007F0E6
:109BD0007CF9FEF79DFC03461A461B4B1A7003F0F6
:109BE0006BFC1A4B01221A70194B1B78002B02D008
:109BF000174B00221A7017481DF0EEFF164B1B681A
:109C0000092B0FDD154B1B78002B0BD1144800F0EE
:109C100077F9144B0122002102201CF09BFF0F4B0F
:109C200001221A70104B1B78DBB2002B06D10E4BB1
:109C300001221A70012110201DF002FC00BF08371C
:109C4000BD4680BD942E0020D4290020242D002064
:109C50001C2D0020642E0020202D0020952E002099
:109C600028CF0D00CCFB02081F2D002080B582B04C
:109C700000AF7860054B01221A70012110201DF001
:109C8000DFFB00BF0837BD4680BD00BF1C2D002094
:109C900080B500AF0020FDF7A3FC00BF80BD000031
:109CA00080B586B004AF78607B68002B46D07B68B7
:109CB0001B78002B42D0FDF76DF9012208214FF0EF
:109CC000904007F002F91F4B0022002102201CF0F7
:109CD00041FF7B68DB687A68127C11467A6892F9EA
:109CE0000A2010467A6892F9182003920290019196
:109CF0000093154B0022002103201CF02BFF134B77
:109D00000022002103201CF025FF7B681B7A012B19
:109D10000ED17B685B7A002B01D00D4B00E00D4B20
:109D200000930D4B0022002103201CF013FF05E0DF
:109D30000A4B0022002103201CF00CFF00BF083753
:109D4000BD4680BDE4FB020818FC02084CFC02087A
:109D50005CFC020860FC020868FC02087CFC02084B
:109D600080B584B002AF78607B68002B2BD07B6815
:109D700093F90530002B1DD115481DF09BFF154BA5
:109D80000022002102201CF0E5FE7B689B79012B5C
:109D900006D1114B0022002102201CF0DBFE05E061
:109DA0000E4B0022002102201CF0D4FE0C4B01229D
:109DB0001A7008E00B4B1B6800930B4B002200212C
:109DC00002201CF0C7FE00BF0837BD4680BD00BFA3
:109DD0004C2E00208CFC0208A4FC0208C4FC0208E3
:109DE00048040020202D0020E4FC0208F0B593B0C8
:109DF0000CAF78617B69002B56D07B695B78022BB6
:109E000008D0032B49D02B4B0022002102201CF04C
:109E1000A1FE4AE07B691B7C18467B69B3F91230CE
:109E20001C467B6993F914301D467B69DB687A69AF
:109E300052687969497D0E467969897D3961796908
:109E4000C97DF9607969097EB9607969497E79606F
:109E50007969897E39607969C97E0B91D7F800C02C
:109E6000CDF828C0D7F804C0CDF824C0D7F808C072
:109E7000CDF820C0D7F80CC0CDF81CC039690691C8
:109E80000596049203930295019400900A4B0022D8
:109E9000002102201CF05EFE07E0084B002200219A
:109EA00002201CF057FE00E000BF00BF1C37BD467B
:109EB000F0BD00BF04FD02081CFD020890FD020871
:109EC00080B584B002AF0346FB71FB79064AD35CD0
:109ED0000093064B0022002102201CF03BFE00BF35
:109EE0000837BD4680BD00BFCCFD0208B0FD0208AA
:109EF00080B500AF002101201DF0A2FA00BF80BD97
:109F000080B582B000AF78600D4A7B6813600C4B5F
:109F10001B68002B03D10A4B44F620621A600948E3
:109F20001DF0C8FE064B1B68194606481DF032FF9F
:109F300004481DF051FE00BF0837BD4680BD00BF7C
:109F400080000020282D002080B483B000AF03469D
:109F5000FB71044AFB79D37000BF0C37BD4680BC4F
:109F6000704700BF6C00002080B483B000AF034690
:109F7000FB71044AFB79137300BF0C37BD4680BCEC
:109F8000704700BF6C00002080B500AF0DF029FDC8
:109F90000346002B06D10DF01BF80346012B01D11F
:109FA000FFF732FB00BF80BD80B500AF17481DF042
:109FB00081FE0DF009FD0346002B06D0144B002254
:109FC000002102201CF0C6FD1AE0124B00220021E5
:109FD00002201CF0BFFD104B01221A700F4B002213
:109FE000002102201CF0B6FD0D480CF01FFE0A4BAC
:109FF0001B78012118460CF06BFF04481DF0ECFDA6
:10A0000008481DF0E9FD00BF80BD00BF282D0020DD
:10A01000D0FD0208F0FD02081C00002004FE02082A
:10A020006C000020402D002080B582B000AF786029
:10A03000054B1B78022B03D1002108201DF000FAEC
:10A0400000BF0837BD4680BD1C00002080B582B02F
:10A0500000AFFF23FB710DF0D1FC0346FB7197F9B4
:10A06000073013F1080F06D10A4B0022002102200D
:10A070001CF070FD0AE097F90730B3F1FF3F05D1FE
:10A08000054B0022002102201CF064FD00BF0837B0
:10A09000BD4680BD24FE02083CFE020880B582B0A9
:10A0A00000AF0346FB71FB79012B06D1084B002260
:10A0B000002102201CF04EFD05E0064B002200218D
:10A0C00002201CF047FD00BF0837BD4680BD00BF21
:10A0D00054FE020868FE020880B582B000AF7860C6
:10A0E000396006F08FFA0346002B1CD1104B1B6819
:10A0F0009A02104B13404FF47C32B2FBF3F101FB98
:10A1000003F3D31ADB0A002201211846FCF76BFD8A
:10A110000346002B05D100233A6879680648FCF70E
:10A1200081FC06F091FA00BF0837BD4680BD00BF34
:10A13000E075FF1F00FCFF0300F0030880B582B04C
:10A1400000AF786039603B689BB21A460349786873
:10A150001DF01EF800BF0837BD4680BD00F00308A3
:10A1600080B500AF184B00221A60174B00225A60CE
:10A17000154B00229A60144B0022DA60124B5B6888
:10A1800043F02003104A53600F4B5B6843F4807325
:10A190000D4A53600C4B5B68002B0CD10B4B00221B
:10A1A000002100201CF0D6FC00BF1CF0C1FC0346BF
:10A1B000012BFAD1FEE7044B0022DA60024B0322A6
:10A1C0001A6000BF80BD00BF982E00207CFE0208F0
:10A1D00080B400AF024B1846BD4680BC704700BF3C
:10A1E000982E002080B500AF04F058FB03461846B7
:10A1F00080BD80B582B000AF0346FB71FB79184685
:10A2000004F080FB034618460837BD4680BD80B584
:10A2100000AF04F0C5FB0346184680BD80B500AF13
:10A2200004F0C5FB0346184680BD80B500AF04F0BE
:10A23000C5FB0346184680BD0D48854604F0C5FBA6
:10A240000C480D490D4A002302E0D458C450043391
:10A25000C4188C42F9D30A4A0A4C002301E0136067
:10A260000432A242FBD31EF071F9FCF73BFFFEE77C
:10A270000080002000000020C803002028460308BA
:10A28000C8030020D8540020FEE780B584B000AF9A
:10A290007860786800F001F90346FB7397F90F3096
:10A2A000002B20D179687B680122D02000F0B1F822
:10A2B0000346FB7397F90F30002B14D17B681B7892
:10A2C000612B0ED1786802F0A6F80346FB7397F96C
:10A2D0000F30002B07D1786801F099FF0346FB731C
:10A2E00001E0FD23FB7397F90F3018461037BD4688
:10A2F00080BDB0B58AB000AFF860B9607A603B60ED
:10A3000000233B6107F1140300221A605A609A602F
:10A31000DA60386801F057FD034687F8273097F96F
:10A320002730002B6CD1FB68002B69D0BB68002B59
:10A3300066D07B68002B5DD07B680A2B5AD800233F
:10A34000BB8434E03B681B7B002B18D1BB8CFA68C4
:10A3500013441B783968184601F074FC034687F8EB
:10A360002730BB8CFA6813441A78BB8C5B0002F070
:10A370007F02D2B228333B4403F8182C09E0BB8C8F
:10A38000FA681A44BB8C5B00127828333B4403F80C
:10A39000182CBB8CBA681A44BB8C5B000133127852
:10A3A00028333B4403F8182CBB8C0133BB84BB8C93
:10A3B0007A689A42C6D897F92730002B1ED13B689D
:10A3C0005C6C387C7B685B005A1E3B685D6807F1FB
:10A3D0001003591C2B46A04703461A463B6883F8D6
:10A3E0004C203B6893F94C30002B07D0FE2387F8B4
:10A3F000273003E0FC2387F8273004E000BF02E0A9
:10A40000FF2387F8273097F9273018462837BD46AD
:10A41000B0BD90B587B000AFB9607A603B600346CD
:10A42000FB73386801F0CFFC0346FB7597F91730D2
:10A43000002B2AD1BB68002B27D03B681B7B002B4D
:10A440000ED1FB7B3968184601F0FCFB0346FB7517
:10A4500097F91730002B03D1FB7B63F07F03FB736D
:10A460003B681C6C3B685B68F87B7A68B968A047FE
:10A4700003461A463B6883F84C203B6893F94C30FE
:10A48000002B04D0FE23FB7501E0FF23FB7597F939
:10A49000173018461C37BD4690BD80B584B000AF5C
:10A4A0007860E023BB73B6237B73786801F08BFC84
:10A4B0000346FB7397F90F30002B2BD17B681B7B76
:10A4C000002B04D1786801F022FC0346FB7397F956
:10A4D0000F30002B1ED107F10D0107F10E007B6834
:10A4E0000122FFF706FF0346FB737B689B6C7A68CB
:10A4F0005268114642F21070984797F90F30002BBE
:10A5000008D17B681B7B002B04D1786801F0FFFB2E
:10A510000346FB7397F90F3018461037BD4680BDD0
:10A5200080B588B000AF786039600023BB77012325
:10A530007B777C4A07F1140392E803001860043328
:10A5400019700023FB6000233B7407F11C0339687A
:10A55000184600F04AF90346FB7797F91F30002BA5
:10A5600005D13968002000F0DFF80346FB777B68EF
:10A57000002B02D1FF23FB77B2E097F91F30002BAD
:10A5800040F0AE80387D07F10C013B680522FFF7F3
:10A5900040FF0346FB773B68002283F84D2097F984
:10A5A0001F30002B08D17B6803333A680721184617
:10A5B00001F0DCFB0346FB7797F91F30002B08D135
:10A5C0007B6801333A680521184601F0CFFB03464A
:10A5D000FB7797F91F30002B08D17B6802333A686C
:10A5E0000521184601F0C2FB0346FB7797F91F309F
:10A5F000002B07D17B683A680521184601F0B6FBAD
:10A600000346FB7797F91F30002B08D17B68043392
:10A610003A680821184601F0A9FB0346FB7797F931
:10A620001F30002B5CD13B7C5BB223F01C035AB281
:10A630007B68DB789B005BB203F01C035BB21343C7
:10A640005BB2DBB23B74FB7B5BB203F01F035AB21D
:10A650007B685B785B015BB213435BB2DBB2FB737D
:10A66000FB7B5BB223F01C035AB27B689B789B0098
:10A670005BB203F01C035BB213435BB2DBB2FB7350
:10A680007B7B5BB223F007035AB27B681B785BB21B
:10A6900003F007035BB213435BB2DBB27B737B68EF
:10A6A0001B79082B04D07B681B79BB7700237B7751
:10A6B0003B7C5BB203F01F035AB2BB7F5B015BB212
:10A6C00013435BB2DBB23B743B7B5BB203F07F03B3
:10A6D0005AB27B7FDB015BB213435BB2DBB23B73ED
:10A6E00097F91F30002B09D107F10C0107F1140075
:10A6F0003B680522FFF7FDFD0346FB773B7F002B00
:10A700000AD097F91F30002B06D13B7F39681846D5
:10A7100000F00AF80346FB7797F91F3018462037F8
:10A72000BD4680BDCCFE020880B584B000AF0346B4
:10A730003960FB710023BB7374233B7307F10D0178
:10A740003B6801227420FFF764FE0346FB7397F910
:10A750000F30002B1DD17B7B03F00303BB73BB7B4E
:10A76000002B16D07B7B23F00303DBB27B7307F156
:10A770000D0107F10C003B680122FFF7BAFD03460B
:10A78000FB733B689B6C3A685268114642F210704A
:10A790009847BB7B002B03D097F90F30002BCDD00F
:10A7A000FB79002B1BD097F90F30002B17D17B7B47
:10A7B0005BB223F003035AB297F9073003F00303A7
:10A7C0005BB213435BB2DBB27B7307F10D0107F1A0
:10A7D0000C003B680122FFF78CFD0346FB7397F9E1
:10A7E0000F3018461037BD4680BD80B584B000AF2D
:10A7F000786039607B68002B0FD007F10E013B6851
:10A8000001227420FFF705FE0346FB73BB7B03F0B8
:10A810000303DAB27B681A7001E0FF23FB7397F938
:10A820000F3018461037BD4680BD000080B58AB095
:10A8300000AF0346B9607A60FB7300233B62344A81
:10A8400007F1140392E80300186004331980BB6811
:10A85000002B58D0BB6801337A680521184601F0F7
:10A8600085FA034687F8273097F92730002B09D15E
:10A87000BB6802337A680521184601F077FA03466F
:10A8800087F8273097F92730002B08D1BB687A6802
:10A890000521184601F06AFA034687F8273097F930
:10A8A0002730002B2FD1BB685B7828333B4413F84B
:10A8B000143CFB61BB689B7828333B4413F8143C81
:10A8C0001A46FB691344FB61BB681B7828333B4481
:10A8D00013F8143C1A46FB691344FB61FB6940F210
:10A8E000AB7202FB03F33B623B6A03F274733B629D
:10A8F0003B6A03F651133B62FB7B022B03D03B6A9E
:10A9000003F57A733B623B6A18462837BD4680BD23
:10A91000D4FE0208B0B59AB000AFB9607A603B606F
:10A920000346FB73002387F86630002387F8653001
:10A93000002387F8643007F1580300221A605A6038
:10A940009A6007F110034822002118461DF030FEDE
:10A9500007F11003BB6507F110031833FB6507F11E
:10A96000100330333B66386801F02DFA034687F850
:10A97000673097F96730002B40F0C180BB68002B2F
:10A9800000F0BD80FB7B012B1CD13A68B968002028
:10A9900000F0F0FD034687F8673097F96730002B29
:10A9A00040F0A180BB681B785BB2002B03DA012367
:10A9B00087F8643097E0002387F86430022387F833
:10A9C000673090E0FB7B022B03D0FB7B032B40F036
:10A9D000878007F158033968184600F00BFF0346DB
:10A9E00087F86730002387F86430002387F86630E3
:10A9F00014E097F866309B0068333B4453F8103CF2
:10AA00001B785BB2002B04DA97F86430013387F8C7
:10AA1000643097F86630013387F8663097F866300F
:10AA2000022B03D897F96730002BE2D0002387F878
:10AA300066301CE097F86630013387F865300DE02A
:10AA400007F1580297F8651097F86630184601F03C
:10AA500065FB97F86530013387F8653097F8653006
:10AA6000022BEDD997F86630013387F8663097F8F6
:10AA70006630012B03D897F96730002BDAD000231A
:10AA800087F866301CE097F866309B0068333B44DB
:10AA900053F8101C97F8662013465B001344DB0044
:10AAA0001A46BB6813441C460D460FCD0FC495E8EB
:10AAB000030084E8030097F86630013387F86630B6
:10AAC00097F86630022B03D897F96730002BDAD05D
:10AAD00097F86430002B06D1022387F8673002E034
:10AAE000012387F867307B68002B03D1FF2387F8A9
:10AAF000673007E07B6897F864201A7002E0FF2354
:10AB000087F8673097F9673018466837BD46B0BD9B
:10AB100080B588B000AF0346B9607A60FB7300234C
:10AB20003B7700237B7747F27013BB82BB68002B17
:10AB30006ED079680020FFF7F7FD0346FB7797F9A1
:10AB40001F30002B08D107F11C02F97B7B68B86825
:10AB500001F058F90346FB7797F91F30002B59D1C4
:10AB600007F118017B6802227020FFF752FC0346B0
:10AB7000FB7797F91F30002B4CD1BB681B78012B5A
:10AB80000BD10023BB777B689B68012B02D102238A
:10AB90007B7706E001237B7703E00123BB7700236B
:10ABA0007B773B7E5BB223F008035AB2BB7FDB00AE
:10ABB0005BB203F008035BB213435BB2DBB23B76DC
:10ABC0007B7E5BB223F00F035AB23B7F5BB203F094
:10ABD0000F035BB213435BB2DBB27B767B7E5BB26F
:10ABE00023F030035AB27B7F1B015BB203F03003CA
:10ABF0005BB213435BB2DBB27B7607F1180107F15E
:10AC000014007B680222FFF774FB0346FB7701E028
:10AC1000FF23FB7797F91F3018462037BD4680BDCC
:10AC2000B0B586B000AF786039607868FBF730F86F
:10AC300003464FF08D411846FBF736F903461C4694
:10AC40003B68DB8B1846FBF723F803464FF089413E
:10AC50001846FBF729F9034619462046FAF766FF1E
:10AC600003461C463B68B3F920301846FBF714F83E
:10AC7000034619462046FBF763F803467B61786874
:10AC8000FBF706F803464FF090411846FBF70CF926
:10AC900003461C463B68DB8B1846FAF7F9FF034670
:10ACA0004FF08C411846FBF7FFF803461946204643
:10ACB000FAF73CFF03461C467868FAF7E9FF0346BB
:10ACC0004FF090411846FBF7EFF803461D463B68EE
:10ACD000DB8B1846FAF7DCFF03464FF08C41184631
:10ACE000FBF7E2F8034619462846FAF71FFF03462A
:10ACF00019462046FBF724F803461C463B6893F9A7
:10AD000022301846FAF7C8FF03464FF08341184631
:10AD1000FBF716F8034619462046FBF711F80346E1
:10AD20003B6139697869FAF703FF03461A463B68C5
:10AD30009A633B689B6B05491846FBF7B5F80346D9
:10AD4000FB60FB6818461837BD46B0BD0000A04543
:10AD500090B587B000AF786039603B689B6B4FF06F
:10AD600080411846FBF7A0F80346A8491846FAF7B1
:10AD7000DDFE03463B6139693869FAF7E1FF0346B6
:10AD80001C463B6893F92E301846FAF785FF0346B8
:10AD90004FF090411846FBF787F8034619462046C6
:10ADA000FAF7CEFF0346FB603B68B3F92C30184638
:10ADB000FAF772FF034639691846FAF7C1FF0346EE
:10ADC00019461846FAF7B4FE03461946F868FAF72A
:10ADD000AFFE0346FB604FF08141F868FBF764F873
:10ADE00003461C463B68B3F92A301846FAF754FF6D
:10ADF00003464FF08F411846FAF7A2FF0346194663
:10AE00002046FAF795FE0346FB603B6893F928302D
:10AE10001846FAF741FF034639691846FAF790FFDA
:10AE2000034639691846FAF78BFF03464FF08D4108
:10AE30001846FBF739F803461C463B68B3F9263041
:10AE40001846FAF729FF034639691846FAF778FFDA
:10AE5000034619462046FAF76BFE03464FF092412F
:10AE60001846FBF721F803463B614FF08E413869E5
:10AE7000FBF71AF803464FF07E511846FAF758FED2
:10AE800003461C463B689B8C1846FAF701FF0346B5
:10AE900019462046FAF754FF03463B617868FAF7F3
:10AEA000F7FE034619464FF09340FAF73FFE03467C
:10AEB0007B613869FBF70AF90346002B00F09D809F
:10AEC0004FF08B41F868FAF7EFFF034619467869AF
:10AED000FAF72CFE03464E491846FAF731FF0346AF
:10AEE00039691846FAF7E0FF03467B613B68B3F91E
:10AEF00032301846FAF7D0FE034679691846FAF759
:10AF00001FFF034679691846FAF71AFF03464FF008
:10AF10009E411846FAF7C8FF03463B613B68B3F908
:10AF200030301846FAF7B8FE03464FF08E41184607
:10AF3000FAF7BAFF034619467869FAF701FF0346A4
:10AF4000FB604FF087417869FAF7AEFF03461C4675
:10AF50004FF087417869FAF7A7FF03461946204664
:10AF6000FAF7EEFE03461C464FF087417869FAF780
:10AF70009BFF034619462046FAF7E2FE03461C46AD
:10AF80003B6893F834301846FAF786FE03464FF0D4
:10AF900090411846FAF788FF034619462046FAF70B
:10AFA000CFFE0346BB60F9683869FAF7C1FD034676
:10AFB000B9681846FAF7BCFD03461C463B6893F98E
:10AFC0002F301846FAF768FE03464FF086411846C0
:10AFD000FAF7B6FE034619462046FAF7A9FD0346DE
:10AFE0004FF083411846FAF75FFF03461946786928
:10AFF000FAF79EFD03467B6102E04FF000037B61A0
:10B000007B6918461C37BD4690BD00BF00007A47DB
:10B010000050C345B0B588B000AF03463960FB802F
:10B020003B689B6B68491846FAF73EFF0346BB61D5
:10B03000FB881846FAF72CFE04463B681B8A184624
:10B04000FAF726FE03464FF083411846FAF778FEDA
:10B0500003461D463B6893F914301846FAF71CFE68
:10B0600003464FF080411846FAF71EFF0346B969C0
:10B070001846FAF765FE034619462846FAF758FDC2
:10B08000034619462046FAF751FD03467B613B68AB
:10B090005B8A1846FAF7FCFD03464FF091411846CB
:10B0A000FAF702FF03461C463B6893F91530184631
:10B0B000FAF7F2FD03464FF08D411846FAF7F4FE19
:10B0C0000346B9691846FAF73BFE03464FF07E5136
:10B0D0001846FAF72DFD03461D463B6893F91630D6
:10B0E0001846FAF7D9FD03464FF093411846FAF790
:10B0F000DBFE0346B9691846FAF722FE0346B96932
:10B100001846FAF71DFE034619462846FAF710FDC1
:10B11000034619462046FAF713FE03461946786996
:10B12000FAF70EFE03463B613B68DB7D1846FAF7F3
:10B13000AFFD03464FF08D411846FAF7B5FE0346C2
:10B14000FB603B6893F918301846FAF7A5FD0346F3
:10B150004FF094411846FAF7A7FE0346BB60B96961
:10B16000B868FAF7EDFD0346F9681846FAF7E0FC0F
:10B17000034639691846FAF7E3FD0346396918466C
:10B18000FAF7DEFD034619463869FAF7D1FC0346A3
:10B19000FB610E49F869FAF78FFF0346002B02D0D6
:10B1A0000A4BFB610AE04FF00001F869FAF766FF0D
:10B1B0000346002B02D04FF00003FB61FB691846E9
:10B1C0002037BD46B0BD00BF0000A0450000C8420A
:10B1D000B0B5A8B000AF03463A60FB800B467B7168
:10B1E000FB881846FAF754FD0346C7F89C307B7974
:10B1F000012202FA03F31846FAF74AFD0346C7F89C
:10B200009830474B07F148041D460FCD0FC40FCDB2
:10B210000FC40FCD0FC495E80F0084E80F00414B19
:10B2200007F108041D460FCD0FC40FCD0FC40FCD7D
:10B230000FC495E80F0084E80F003B6893F93E3097
:10B240001846FAF729FD034637491846FAF778FDFC
:10B25000034636491846FAF76BFC0346C7F89430A4
:10B260007B799B00A0333B4453F8583C3049184647
:10B27000FAF71AFE03464FF07E511846FAF758FCCB
:10B2800003461946D7F89400FAF75AFD0346C7F863
:10B2900090307B799B00A0333B4453F8983C244981
:10B2A0001846FAF701FE03464FF07E511846FAF7AA
:10B2B0003FFC0346C7F88C301E49D7F88C00FAF7DC
:10B2C0003FFD0346D7F898101846FAF739FD0346B4
:10B2D0001C464FF08841D7F89C00FAF727FC03463C
:10B2E000D7F890101846FAF7DFFD03464FF07E516D
:10B2F0001846FAF71DFC034619462046FAF720FDCA
:10B30000034619464FF07E50FAF7CEFD0346C7F8C4
:10B310008830D7F888301846A037BD46B0BD00BF8A
:10B32000DCFE02081CFF02080000A0400080A744C9
:10B330000000C842BD37063490B587B000AF034661
:10B340000A46FB8013467B717B794FF4802222FAF8
:10B3500003F37B61FB88A3F500733B613A691346F5
:10B360005B0013443B613B6903F580533B617869A3
:10B37000FAF78EFC03460A491846FAF7E1FC034641
:10B380001C463869FAF788FC034619462046FAF746
:10B390008BFD0346FB60FB6818461C37BD4690BD1D
:10B3A0000024744990B589B000AF03463960FB8032
:10B3B000FB88B3F5C87F02D94FF4C873FB803B68A4
:10B3C00093F919301846FAF767FC03464FF08341AA
:10B3D0001846FAF769FD03464E491846FAF7A8FBE6
:10B3E0000346FB613B68B3F91A301846FAF754FC80
:10B3F00003464FF08E411846FAF756FD034646497C
:10B400001846FAF79DFC034644491846FAF790FBA4
:10B410000346BB613B6893F91C301846FAF73CFCC5
:10B4200003464FF089411846FAF73EFD03467B611B
:10B43000FB881846FAF72CFC0346B9691846FAF758
:10B440007FFC03464FF07E511846FAF771FB034626
:10B450001946F869FAF774FC03463B613B6893F9B7
:10B460000E301846FAF718FC034679691846FAF7C1
:10B4700067FC034619463869FAF75AFB0346FB6036
:10B480003B6893F83C301846FAF702FC03464FF04D
:10B4900081411846FAF74CFB034619464FF08140AC
:10B4A000FAF702FD0346F9681846FAF749FC034625
:10B4B0001C463B6893F93D301846FAF7EDFB03460E
:10B4C00017491846FAF73CFC03464FF07E511846E0
:10B4D000FAF72EFB034619464FF07E50FAF7E4FCCC
:10B4E000034619462046FAF72BFC03460D49184639
:10B4F000FAF71CFB03460C491846FAF721FC0346F1
:10B500001846FAF709FE0346FB72FB7A1846243701
:10B51000BD4690BD000044426F12033A75021A3BCB
:10B520006F12033B0000C8419A99594080B485B01E
:10B5300000AF0346FB800023FB73FB88B3F57C6FF1
:10B5400008D3FF23BB730FE0FB889B08FB80FB7BCA
:10B550000133FB73FB883F2BF6D8FB88DAB2FB7B09
:10B560009B01DBB21344BB73BB7B18461437BD464B
:10B5700080BC704780B58EB000AF0346B9607A607A
:10B58000FB73002387F8373000233B6107F1140376
:10B5900000221A605A609A601A73052387F83630C1
:10B5A00019E1FB7B1A4612011344DBB21D33D8B2FA
:10B5B00007F110017B681122FEF72BFF034687F885
:10B5C0003730BB68002B03D1FF2387F837300BE1FE
:10B5D0003B7C23F07F03DAB2BB681A703B7C03F03C
:10B5E0000F03DAB2BB685A707A7CBB689A70BB7C76
:10B5F0001A03FB7C1B0113433A7D1209D2B2134399
:10B600003B637B7D1A03BB7D1B011343FA7D12094B
:10B61000D2B21343FB623B7E9BB21B029AB27B7E8B
:10B620009BB213437B857B7F9BB29B009AB2BB7F0F
:10B630009B09DBB29BB213433B85FB7F9BB29B0014
:10B640009AB297F820309B09DBB29BB21343FB847C
:10B65000BB7F03F00F0387F8253097F8203003F005
:10B660000F0387F824307B689B68012B1CD1BB68D3
:10B670001B785AB297F820305BB203F020035BB21C
:10B6800013435BB2DAB2BB681A70BB681B785AB25C
:10B6900097F820305BB203F010035BB213435BB248
:10B6A000DAB2BB681A7019E0BB681B785AB2BB7F6C
:10B6B0005BB203F020035BB213435BB2DAB2BB6848
:10B6C0001A70BB681B785AB2BB7F5BB203F01003E1
:10B6D0005BB213435BB2DAB2BB681A70BB681B780B
:10B6E0005BB2002B66DA97F93730002B62D1BB686A
:10B6F0005B785A33D8B2BB68D91C7B680122FEF74D
:10B7000088FE034687F8373097F93730002B0CD185
:10B71000BB685B785033D8B2BB68191D7B680122C7
:10B72000FEF777FE034687F8373097F93730002B5E
:10B730000CD1BB685B786433D8B2BB68591D7B6899
:10B740000122FEF766FE034687F8373097F9373057
:10B75000002B2FD17968F86AFFF762FA0246BB68BE
:10B760009A607968386BFFF7F3FA0246BB68DA60D3
:10B770007B8D79681846FFF74DFC0246BB681A615D
:10B780007B689B68012B0AD197F82420FB8C11461B
:10B790001846FFF7D1FD0246BB685A6124E097F8CE
:10B7A00025103B8D7A681846FFF712FD0246BB68EC
:10B7B0005A6119E097F93730002B07D17B689B6CF1
:10B7C0007A685268114642F21070984797F83630FE
:10B7D000013B87F8363097F83630002B04D097F9C4
:10B7E0003730002B3FF4DDAE97F937301846383745
:10B7F000BD4680BD90B59DB000AF78603960002334
:10B8000087F86F300023BB6207F12C032F22002141
:10B8100018461CF0CDFE0023BB6007F10C0300228C
:10B820001A605A609A60DA601A615A611A837B68FA
:10B830001B68002B0CD17B6804331B68002B07D1DD
:10B840007B6808331B68002B02D1FF2387F86F3019
:10B8500097F96F30002B09D107F128013B6833229B
:10B860001D20FEF7D6FD034687F86F3097F96F303D
:10B87000002B09D107F108013B681E225020FEF77A
:10B88000C8FD034687F86F30002387F86E30CAE1A1
:10B8900097F86E301A461201134487F86D3097F806
:10B8A0006D3070333B4413F8482C97F86E309B0092
:10B8B00079680B441B6822F07F02D2B21A7097F8A5
:10B8C0006D3070333B4413F8482C97F86E309B0072
:10B8D00079680B441B6802F00F02D2B25A7097F8D5
:10B8E0006D305A1C97F86E309B0079680B441B68CA
:10B8F00070323A4412F8482C9A7097F86D3002333F
:10B9000070333B4413F8483C1A0397F86D30033307
:10B9100070333B4413F8483C1B01134397F86D20E8
:10B92000043270323A4412F8482C1209D2B213434E
:10B93000BB6697F86D30053370333B4413F8483CD1
:10B940001A0397F86D30063370333B4413F8483CC4
:10B950001B01134397F86D20073270323A4412F8F6
:10B96000482C1209D2B213437B6697F86D30083326
:10B9700070333B4413F8483C9BB21B029AB297F8D1
:10B980006D30093370333B4413F8483C9BB213438A
:10B99000A7F8623097F86D300D3370333B4413F8DD
:10B9A000483C9BB29B009AB297F86D300E337033CF
:10B9B0003B4413F8483C9B09DBB29BB21343A7F806
:10B9C000603097F86D300F3370333B4413F8483CC8
:10B9D0009BB29B009AB297F86D30103370333B44A2
:10B9E00013F8483C9B09DBB29BB21343A7F85E30C7
:10B9F00097F86D300E3370333B4413F8483C03F036
:10BA00000F0387F85D3097F86D30103370333B4487
:10BA100013F8483C03F00F0387F85C303B689B68E1
:10BA2000012B3AD197F86E309B007A6813441B685B
:10BA30001B785AB297F86D30103370333B4413F8CB
:10BA4000483C5BB203F020035BB2134359B297F852
:10BA50006E309B007A6813441B68CAB21A7097F85C
:10BA60006E309B007A6813441B681B785AB297F8B3
:10BA70006D30103370333B4413F8483C5BB203F035
:10BA800010035BB2134359B297F86E309B007A688B
:10BA900013441B68CAB21A7039E097F86E309B00E5
:10BAA0007A6813441B681B785AB297F86D300E33CE
:10BAB00070333B4413F8483C5BB203F020035BB2A5
:10BAC000134359B297F86E309B007A6813441B6891
:10BAD000CAB21A7097F86E309B007A6813441B68DC
:10BAE0001B785AB297F86D300E3370333B4413F81D
:10BAF000483C5BB203F010035BB2134359B297F8B2
:10BB00006E309B007A6813441B68CAB21A7097F8AB
:10BB10006E309B007A6813441B685B78194697F86F
:10BB20006E309B007A6813441B6801F170023A443E
:10BB300012F8682C1A7197F86E309B007A681344DB
:10BB40001B685B7803F10A0297F86E309B007968F6
:10BB50000B441B6870323A4412F8682CDA7097F87C
:10BB60006E309B007A6813441B685B7803F1140203
:10BB700097F86E309B0079680B441B6870323A442A
:10BB800012F8682C5A7197F86E309B007A6813444B
:10BB90001C683968786EFFF743F80346A36097F88E
:10BBA0006E309B007A6813441C683968B86EFFF7E2
:10BBB000CFF80346E36097F86E309B007A68134431
:10BBC0001C68B7F8623039681846FFF723FA034655
:10BBD00023613B689B68012B10D197F86E309B0066
:10BBE0007A6813441C6897F85C20B7F85E301146F9
:10BBF0001846FFF7A1FB034663610FE097F86E302C
:10BC00009B007A6813441C6897F85D10B7F86030A1
:10BC10003A681846FFF7DCFA0346636197F86E301E
:10BC2000013387F86E3097F86E30022B04D897F9FD
:10BC30006F30002B3FF42CAE97F96F3018467437F5
:10BC4000BD4690BD90B585B000AF03463960FB712D
:10BC5000386800F0B8F80346FB7397F90F30002BF3
:10BC60004FD197F90730002B02DA0023BB7301E0B4
:10BC70001023BB733B685B7BBA7B9A4241D03B6825
:10BC8000BA7B5A733B681C6C3B685B6807F10D011B
:10BC90000122F320A04703461A463B6883F84C2054
:10BCA0003B6893F94C30002B01D0FE23FB7397F9CE
:10BCB0000F30002B25D17B7B23F01003DBB27B738D
:10BCC0003B685B7B5BB203F010035AB27B7B5BB2D9
:10BCD00013435BB2DBB27B733B685C6C3B685B68B5
:10BCE00007F10D0101227320A04703461A463B6865
:10BCF00083F84C203B6893F94C30002B01D0FE2395
:10BD0000FB7397F90F3018461437BD4690BD90B5B8
:10BD100085B000AF7860786800F055F80346FB7393
:10BD200097F90F30002B1BD17B681C6C7B685B681C
:10BD300007F10E010122F320A04703461A467B6853
:10BD400083F84C207B6893F94C30002B02D0FE2303
:10BD5000FB7305E0BB7B03F01003DAB27B685A7318
:10BD600097F90F3018461437BD4690BD80B586B0A0
:10BD700000AFF8600B467A60FB72786800F023F839
:10BD80000346FB75FB68002B15D097F91730002B85
:10BD900011D1FB681B78FA7A9A420ED2FB68FA7AC4
:10BDA0001A707B6893F84D3043F00103DAB27B6878
:10BDB00083F84D2001E0FF23FB7597F917301846F3
:10BDC0001837BD4680BD80B485B000AF78600023D1
:10BDD000FB737B68002B0BD07B681B6C002B07D0A0
:10BDE0007B685B6C002B03D07B689B6C002B01D1C4
:10BDF000FF23FB7397F90F3018461437BD4680BCFC
:10BE00007047000090B593B000AFF8607A603B6077
:10BE10000B46FB72002387F84730002387F8453034
:10BE20006E2387F84330A14A07F1380307CA03C3DA
:10BE30001A809E4A07F12C0307CA03C31A809B4A43
:10BE400007F1200307CA03C31A80984A07F11403B5
:10BE500007CA03C31A80FB7A032B24D0032B00F3F9
:10BE6000F980012B02D0022B7CD0F3E05A2387F813
:10BE70003830FB685B8839681846FFF793FA034649
:10BE800087F82C30642387F82030FB689B8818469D
:10BE9000FFF74CFB03463B757B6800221A700123B9
:10BEA00087F84530DBE0FB68DB68002B03D0FB68DC
:10BEB0009B68002B03D1FF2387F84730CFE0002396
:10BEC00087F846303FE097F8463097F846205A32D8
:10BED000D2B248333B4403F8102CFB689A6897F8B9
:10BEE00046305B0013441B8897F846403968184673
:10BEF000FFF758FA03461A4604F148033B4403F897
:10BF00001C2C97F8463097F846206432D2B248335A
:10BF10003B4403F8282CFB68DA6897F846305B004E
:10BF200013441B8897F846401846FFF7FFFA03466C
:10BF30001A4604F148033B4403F8342C97F8463082
:10BF4000013387F84630FB681B7C97F846209A42FD
:10BF5000B9D3FB681A7C7B681A70FB681B7C87F876
:10BF600045307CE0FB68DB68002B03D0FB689B68F6
:10BF7000002B03D1FF2387F8473070E0FB685B8A12
:10BF8000002B02D1032387F84730002387F846307F
:10BF90003AE097F8463097F846205A32D2B2483302
:10BFA0003B4403F8102CFB689A6897F846305B0016
:10BFB00013441B8897F8464039681846FFF7F2F992
:10BFC00003461A4604F148033B4403F81C2C97F837
:10BFD000463097F846206432D2B248333B4403F8E7
:10BFE000282CFB68DA6897F846305B0013441A88FF
:10BFF00097F84630D2B248333B4403F8342C97F8D4
:10C000004630013387F84630FB681B7C97F84620A2
:10C010009A42BED3FB681A7C7B681A70FB681B7C53
:10C0200087F84530FB685B8A184600F041F8034604
:10C0300087F8443097F94730002B0FD107F14401BE
:10C0400007F143003B680122FEF753F9034687F8E6
:10C05000473003E0012387F8473000E000BF97F93D
:10C060004730002B0BD197F8452007F12C0107F141
:10C0700038003B68FEF73DF9034687F8473097F9EB
:10C080004730002B0BD197F8452007F1140107F139
:10C0900020003B68FEF72DF9034687F8473097F9F3
:10C0A000473018464C37BD4690BD00BF5CFF0208C4
:10C0B00080B485B000AF0346FB800023FB73FB8890
:10C0C00040F28272934202D9FF23BB731DE0FB88CA
:10C0D0004FF47A7203FB02F20F4BA3FB0213D21A46
:10C0E000520813441B0AFB8005E0FB889B08FB8079
:10C0F000FB7B0133FB73FB883F2BF6D8FB88DAB25E
:10C10000FB7B9B01DBB21344BB73BB7B184614372C
:10C11000BD4680BC704700BF9FB8C81280B584B0D0
:10C1200000AF03463A60FB710B46BB71FB799B0085
:10C130003A6813441B689B78FB81BB799B003A6883
:10C1400013441B689B78BB81FB799B003A681344BE
:10C150001B681B785BB2002B21DABB799B003A6825
:10C1600013441B681B785BB2002B18DABA89FB8971
:10C17000D31A9BB27B81B7F90A3013F1020F03DBAC
:10C18000B7F90A30002B03DBB7F90A30022B16DDB2
:10C19000B979FB793A68184600F016F80FE0BB79D8
:10C1A0009B003A6813441B681B785BB2002B07DACC
:10C1B000B979FB793A68184600F006F800E000BF4C
:10C1C00000BF1037BD4680BD80B485B000AF0346C8
:10C1D0003A60FB710B46BB71FB799B003A681344D4
:10C1E0001B68FB60BB799B003A681A44FB799B0093
:10C1F00039680B4412681A60BB799B003A68134493
:10C20000FA681A6000BF1437BD4680BC704780B51D
:10C210008EB000AF786007F10C017B6817228A208E
:10C22000FEF7F7F8034687F8373097F93730002BD9
:10C230000BD107F10C0303F117017B680E22E120FB
:10C24000FEF7E7F8034687F8373097F93730002BC9
:10C250000BD107F10C0303F125017B6805220020B7
:10C26000FEF7D7F8034687F8373097F93730002BB9
:10C2700040F0CB8097F82C301B021AB297F82B3085
:10C280001BB213431BB29AB27B68DA837B7B1B021F
:10C290001AB23B7B1BB213431AB27B681A84BB7B76
:10C2A0005AB27B6883F822207B7C1B021AB23B7C4B
:10C2B0001BB213431BB29AB27B689A84FB7C1B02AD
:10C2C0001AB2BB7C1BB213431AB27B68DA843B7D83
:10C2D0005AB27B6883F82820FB7D1B021AB2BB7D13
:10C2E0001BB213431AB27B685A857B7E1B021AB2BB
:10C2F0003B7E1BB213431AB27B689A85FB7E5AB20F
:10C300007B6883F82E20BB7E5AB27B6883F82F208F
:10C31000FB7F1B021AB2BB7F1BB213431AB27B68AE
:10C320001A8697F821301B021AB297F820301BB2F8
:10C3300013431AB27B685A8697F822207B6883F8E9
:10C34000342097F825301B011AB297F824301BB21D
:10C3500003F00F031BB213431BB29AB27B681A821D
:10C3600097F823301B011AB297F824301B09DBB26F
:10C370001BB213431BB29AB27B685A8297F82630DD
:10C380005AB27B681A7597F827305AB27B685A758B
:10C3900097F828305AB27B689A7597F829207B68FD
:10C3A000DA7597F82A305AB27B681A7697F82F30E8
:10C3B0005AB27B685A7697F82E301B021AB297F859
:10C3C0002D301BB213431AB27B685A8397F8303072
:10C3D0005AB27B681A7797F8333003F03003002B9A
:10C3E00000DA0F331B11DAB27B6883F83C2097F830
:10C3F00031305AB27B6883F83D2097F835305BB214
:10C400001B115AB27B6883F83E2097F937301846E3
:10C410003837BD4680BD80B584B000AF786000235A
:10C42000BB7307F10E017B680122F020FDF7F1FFDD
:10C430000346FB7397F90F30002B03D1BB7B1A46E1
:10C440007B689A6097F90F3018461037BD4680BD5B
:10C4500080B586B000AFB9607A603B600346FB737D
:10C460000023FB7500224FF400414FF0904004F090
:10C470002CFDFB7B03F07F03DAB2134B1A7002230F
:10C4800001221149114806F04BFD0346FB757B68FC
:10C490009AB27B685B00B9680C4806F041FD034620
:10C4A0005BB2DAB2FB7D1344DBB2FB7501224FF4C1
:10C4B00000414FF0904004F008FD97F917301846FE
:10C4C0001837BD4680BD00BFA82E0020282A0020B6
:10C4D00080B588B002AFB9607A603B600346FB73F9
:10C4E0000023FB7500224FF400414FF0904004F010
:10C4F000ECFCFB7B63F07F03DAB2144B1A7002236F
:10C5000001221249124806F00BFD0346FB757B68B9
:10C510009AB27B685B0000931346BA680B490C48DB
:10C5200006F08EFE03465BB2DAB2FB7D1344DBB24B
:10C53000FB7501224FF400414FF0904004F0C5FC20
:10C5400097F9173018461837BD4680BDA82E002031
:10C55000282A002080B582B000AF786039607B68FF
:10C56000054AA2FB03239B091846FAF744FD00BFC6
:10C570000837BD4680BD00BFD34D62102DE9B04FD6
:10C580008EB000AF4FF000024FF00003C7E90C235C
:10C59000FCF7E8F8034600221C461546C7E90C459F
:10C5A000D7E90C4522462B464FF000004FF0000122
:10C5B000590141EAD261500102460B46B2EB040830
:10C5C00063EB05094FF000024FF000034FEA8903C7
:10C5D00043EA98734FEA88029046994618EB0403A1
:10C5E000BB6049EB0503FB604FF000024FF0000316
:10C5F000D7E902452946CB0020462946044643EAAE
:10C6000054730146CA001C461346C7E90C34294B33
:10C610001B680022BB62FA62D7E90C23D7E90A0142
:10C620000446A2428B4104DA234B1B680133224AA1
:10C6300013603B6B1F4A13601F4B1B6800223B6259
:10C640007A62D7E9084522462B464FF000004FF0AA
:10C650000001D90741EA5201D00702460B462046A5
:10C6600029460446B2EB040A0C4663EB040B1AEBB2
:10C670000A033B604BEB0B037B60D7E900AB03463F
:10C680001AEB0303BB610B464BEB0303FB61D7E9DA
:10C690000C23D7E90645214689183961294643EB21
:10C6A00001017961D7E90423104619463837BD46A0
:10C6B000BDE8B08FAC2F0020A82F00202DE9F04F4F
:10C6C000A3B012AFC7E90C01FA6287F82B304FF024
:10C6D00000024FF00003C7E90E23D7E90C013A4AE4
:10C6E0004FF00003F9F738FD02460B46C7E90E2369
:10C6F000364A97F82B301371344AFB6A5361334A38
:10C70000D7F888309361314AFB6E13612F4A3B6F33
:10C7100093602E4ABB6ED360BB6B7B62F86AF8F7FE
:10C7200077FEC7E9060197F82B60B86EF8F770FE40
:10C73000C7E90401F86EF8F76BFEC7E90201386F2C
:10C74000F8F766FEC7E90001F86FF8F761FE824668
:10C750008B46D7F88800F8F75BFE80468946D7F805
:10C760009400F8F755FE04460D46D7F89800F8F700
:10C770004FFE02460B46CDE91023CDE90E45CDE92B
:10C780000C89CDE90AABD7E90034CDE90834D7E903
:10C790000234CDE90634D7E90434CDE904340296F5
:10C7A000D7E90634CDE900347A6A094909481CF012
:10C7B00073FD084B0122002102201AF0CBF900BFC3
:10C7C0004437BD46BDE8F08F40420F00FC2C0020EE
:10C7D00068FF0208B02F002080B483B000AF7860FB
:10C7E0003960002318460C37BD4680BC704780B4C2
:10C7F00083B000AF7860396000BF0C37BD4680BCA5
:10C800007047000080B582B000AF786039607B6807
:10C81000064A184611464FF4E7731A461BF0BAFE53
:10C820004FF4E77318460837BD4680BD600603081D
:10C8300090B5ADF6443D00AF07F53464A4F634344A
:10C84000206007F53460A0F63830016007F53461E8
:10C85000A1F63C310A6007F53462A2F53462136038
:10C86000002387F8283B002387F8293B0023C7F8DB
:10C870008C3A07F529639722002118461BF098FE91
:10C8800007F53463A3F5217300221A6004334FF4D3
:10C89000E572002118461BF08BFE07F53463A3F602
:10C8A000842300221A60043340F2FC7200211846EF
:10C8B0001BF07EFE0D2387F83F3B07F53463A3F69C
:10C8C0002D3308221A70B14BB14A5A60AF4B002287
:10C8D0001A73AE4A07F53463A3F638331B68536402
:10C8E000AA4A07F53463A3F63C331B681364A74ACE
:10C8F00007F53463A3F534631B689364A34B1922D3
:10C900009A73A248FDF7C1FC034687F8283B97F9C4
:10C91000283B002B04D0B7F8283BA7F82C3B27E195
:10C92000F3F738FC034687F8293B97F9293B002B9E
:10C9300004D0B7F8283BA7F82C3B19E107F6BC0256
:10C94000D7F8543B4FF4E771104698470346C7F8B1
:10C95000383BD7F8383B002B15D0D7F8381B07F1F8
:10C96000BC0207F6BC004FF40063F3F745FC034636
:10C9700087F8293B97F9293B002B04D0B7F8283BCF
:10C98000A7F82C3BF4E007F68C22D7F8503B9B210C
:10C99000104698470346C7F8343BD7F8343B002B82
:10C9A00015D0D7F8341B07F1BC0207F68C204FF4E2
:10C9B0000063F3F731FC034687F8293B97F9293BDD
:10C9C000002B04D0B7F8283BA7F82C3BD0E0714AE5
:10C9D00007F53463A3F634331B6813606E4BC7F856
:10C9E000303B07F53463A3F6EC2301221A7107F5F7
:10C9F0003463A3F6EC23D7F8302B1A6007F53463C1
:10CA0000A3F6EC230E221A7307F53463A3F6EC2386
:10CA1000624A9A6007F53463A3F6EC2307221A757D
:10CA200007F53463A3F6EC235C4A1A6107F5346317
:10CA3000A3F6EC230F221A7707F53463A3F6EC2351
:10CA4000564A9A6107F53463A3F6EC23092283F86A
:10CA5000242007F53463A3F6EC23D7F8302B1A62B1
:10CA600007F53463A3F6EC23062283F82C2007F5A0
:10CA70003463A3F6EC23494A9A6207F53463A3F6BC
:10CA8000EC23082283F8342007F53463A3F6EC2363
:10CA9000424A1A6307F53463A3F6EC23022283F8B3
:10CAA0003C2007F53463A3F6EC23D7F8302B9A63C8
:10CAB00007F53463A3F6EC23032283F8442007F53B
:10CAC0003463A3F6EC23D7F8302B1A6407F53463EC
:10CAD000A3F6EC23042283F84C2007F53463A3F675
:10CAE000EC23D7F8302B9A6407F53463A3F6EC23D4
:10CAF0000C2283F8542007F53463A3F6EC23D7F80F
:10CB0000302B1A6507F53463A3F6EC230D2283F866
:10CB10005C2007F53463A3F6EC23D7F8302B9A6535
:10CB200007F53463A3F6EC23152283F8642007F598
:10CB30003463A3F6EC23D7F8302B1A6607F11303FE
:10CB400007F1140297F83F1B07F15400F3F730FB8D
:10CB5000034687F8293B97F9293B002B04D0B7F807
:10CB6000283BA7F82C3B03E0B7F8283BA7F82C3B61
:10CB7000002397F82C2B62F3070397F82D2B62F311
:10CB80000F23184607F64437BD4690BD7830002085
:10CB90008C000020E43000207E735A3B3BAAAA3E62
:10CBA00080B584B000AF786039600023FB737B6888
:10CBB0001B7D002B48D0344B0022DA70324B082208
:10CBC0001A717B68DA7C304B1A707B685A7C2E4B6A
:10CBD0009A707B689A7C2C4B5A702C492A48FDF736
:10CBE0009FFC0346FB737B681A7C294B1A707B6899
:10CBF0009A89274B5A807B68DA89254B9A80234A89
:10CC000023490120FDF784FF0346FB731F490120E0
:10CC1000FDF78AFD0346FB731C4A1B490120FDF703
:10CC200005FE03469AB21A4B9B8819464901C91A58
:10CC300089000B44DB009BB21344BB81BA89134BC0
:10CC400059683B681046984707F10B030F4918468F
:10CC5000FDF7CBFD0346FB730EE00C4B5A683B68B7
:10CC6000114641F28830984707F10B0307491846EF
:10CC7000FDF7BBFD0346FB73FB7A012BEDD000BF34
:10CC800000BF1037BD4680BDC8300020783000207E
:10CC9000D030002080B586B000AFC7E902017A60CD
:10CCA0003B600023FB753B6A002B00F0BD8007F161
:10CCB00016025F4B5F490120FDF72CFE0346FB7512
:10CCC000BB7D002B00F0B0803B6A03F00103002B1A
:10CCD0001DD03B681B781B017A68134401225A73EC
:10CCE0003B681B781B017A681344524AD2689A60E9
:10CCF0003B681B781B017A68D118D7E90223C1E988
:10CD000000233B681B780133DAB23B681A703B6A38
:10CD100003F00403002B3BD03B681B781B017A68AF
:10CD2000134403225A733B681B781B017A6813442F
:10CD3000404A92689A603B681B781B017A68D11858
:10CD4000D7E90223C1E900233B681B780133DAB23B
:10CD50003B681A703B681B781B017A6813440E22EB
:10CD60005A733B681B781B017A681344324A126875
:10CD70009A603B681B781B017A68D118D7E90223B7
:10CD8000C1E900233B681B780133DAB23B681A70B3
:10CD90003B6A03F00203002B1DD03B681B781B018C
:10CDA0007A68134402225A733B681B781B017A6825
:10CDB0001344204A12699A603B681B781B017A6809
:10CDC000D118D7E90223C1E900233B681B7801335E
:10CDD000DAB23B681A703B6A03F00803002B23D0D9
:10CDE000144B1B7803F02003002B1DD03B681B78ED
:10CDF0001B017A68134404225A733B681B781B0199
:10CE00007A6813440B4A52699A603B681B781B018D
:10CE10007A68D118D7E90223C1E900233B681B785F
:10CE20000133DAB23B681A7000BF1837BD4680BDC7
:10CE300078300020E8300020E43000202DE9F04F69
:10CE4000D5B00EAF07F58C73A3F58273186007F5A4
:10CE50008C73A3F586731A6007F58C73A3F2051320
:10CE60000A461A700023FB77002387F81731002346
:10CE700087F807314FF000024FF00003C7E9422363
:10CE800007F58C73A3F205131B78002B00F09A8131
:10CE90000E23FB7707F11F0407F1200207F58C73BF
:10CEA000A3F20513197807F58C73A3F58270234656
:10CEB0000068F3F78FF9034687F80731002387F8F6
:10CEC000173134E197F817311B0103F5887307F127
:10CED00008021344EB3B1B78013B142B00F2218129
:10CEE00001A252F823F000BF3DCF00086FCF000829
:10CEF000A1CF0008D3CF000823D10008A1D000089B
:10CF00001FD00008BBD0000853D0000823D1000870
:10CF100023D100086DD0000887D0000805D0000894
:10CF200039D0000823D1000823D1000823D10008FC
:10CF300023D1000823D10008D5D0000897F8173175
:10CF40001B0103F5887307F108021344F03B1B68CB
:10CF50009F4A136097F817311B0103F5887307F197
:10CF600008021344EA3B1A789A4B1A70CBE097F800
:10CF700017311B0103F5887307F108021344F03BD6
:10CF80001B68954A136097F817311B0103F58873E6
:10CF900007F108021344EA3B1A78904B1A70B2E08A
:10CFA00097F817311B0103F5887307F10802134442
:10CFB000F03B1B688A4A136097F817311B0103F591
:10CFC000887307F108021344EA3B1A78854B1A70FC
:10CFD00099E097F817311B0103F5887307F10802F0
:10CFE0001344F03B1B68804A136097F817311B010C
:10CFF00003F5887307F108021344EA3B1A787B4B68
:10D000001A7080E097F817311B0103F5887307F158
:10D0100008021344F03B1B68754A136073E097F8ED
:10D0200017311B0103F5887307F108021344F03B25
:10D030001B68704A136066E097F817311B0103F50F
:10D04000887307F108021344F03B1B686A4A1360B7
:10D0500059E097F817311B0103F5887307F10802AF
:10D060001344F03B1B68654A13604CE097F8173196
:10D070001B0103F5887307F108021344F03B1B689A
:10D080005F4A13603FE097F817311B0103F588737F
:10D0900007F108021344F03B1B685A4A136032E060
:10D0A00097F817311B0103F5887307F10802134441
:10D0B000F03B1B68544A136025E097F817311B01B9
:10D0C00003F5887307F108021344F03B1B684F4ACD
:10D0D000136018E097F817311B0103F5887307F107
:10D0E00008021344F03B1B68494A136097F8173154
:10D0F0001B0103F5887307F108021344EA3B1A7811
:10D10000444B1A7000BF97F817311B0103F5887361
:10D1100007F108021344F83BD3E90023C7E942238F
:10D1200000E000BF97F81731013387F81731FB7F14
:10D1300097F817219A42FFF4C5AE254B1B68BB60D8
:10D14000244B197879602A4B18682B4B1C68294BA3
:10D150001D682D4B1E682D4BD3F800C0274BD3F80C
:10D1600000E02B4BD3F800801B4BD3F80090244BEE
:10D17000D3F800A0234BD3F800B0194B1A683A60DB
:10D18000194B196807F58C73A3F586720C913968F1
:10D190000B91CDF828B0CDF824A0CDF8209097F9C8
:10D1A00007310793CDF81880CDF814E0CDF810C002
:10D1B000039602950194009014687B68BA68D7E9D9
:10D1C0004201A04700BF07F58E77BD46BDE8F08F4E
:10D1D0000031002004310020083100200C310020F3
:10D1E0001031002014310020183100201C310020A3
:10D1F0002031002024310020283100202C31002053
:10D200003031002034310020383100203C31002002
:10D2100040310020443100202DE9B04FADF6881D8B
:10D2200002AF07F51864A4F65C14206007F51860D7
:10D23000A0F51660016007F51861A1F664110A6097
:10D2400007F51862A2F6681213604FF000024FF063
:10D25000000307F67811C1E900234FF000024FF0F8
:10D26000000307F51761C1E90023002387F8E738B9
:10D2700007F51863A3F6581300221A60002387F8F5
:10D280006F3907F51863A3F516631B6898470246C4
:10D290000B464FF000044FF000055D0145EAD265F2
:10D2A000540122462B46B2EB000863EB01094FF014
:10D2B00000024FF000034FEA890343EA98734FEAF4
:10D2C00088029046994618EB0003BB6049EB0103C6
:10D2D000FB604FF000024FF00003D7E902452946FA
:10D2E000CB0020462946044643EA54730146CA004F
:10D2F0001C46134607F67812C2E9003407F6C80345
:10D300001A4607F67813D3E90001F2F7CDFF03467A
:10D3100087F86F3997F96F39002B16D097F96F3965
:10D32000002B09DA97F96F3900935E4B0122002137
:10D33000022019F00FFC08E097F96F3900935A4B5F
:10D3400001220021022019F005FC584B01221A701D
:10D3500007F51863A3F65C1307F6C80219681046B0
:10D36000FFF71EFC514B00221A70002387F8E738A4
:10D37000D7F8D038194607F6E70307F6E802009118
:10D3800007F67811D1E90001FFF784FC97F8E71858
:10D3900007F51863A3F6641307F6E8001A68FFF7A9
:10D3A0004DFD434B1B680133414A1360404B1B68E2
:10D3B000D7F8A0299A4226D807F12C0207F62C01AB
:10D3C00007F1280301934FF40063009313469B2257
:10D3D0000020F2F74DFF034687F86F3997F96F3950
:10D3E000002B0DD107F51863A3F65813196807F63B
:10D3F0002C0207F51863A3F668131B6810469847BC
:10D400002B4B00221A6007F6C803D3E9004507F545
:10D410001863A3F516631B689847804689464FF04A
:10D4200000024FF000034B0143EAD0634201B8EB26
:10D43000020A69EB030B4FF000024FF000034FEAC2
:10D440008B0343EA9A734FEA8A0292469B46BAEBF1
:10D4500000033B606BEB01037B604FF000024FF079
:10D460000003D7E900894946CB00C44643EA5C7310
:10D470004146CA00A118396145EB03037B610D4A9F
:10D480004FF00003D7E90401F8F766FE02460B46A9
:10D4900007F51761C1E9002300BF07F51867BD460E
:10D4A000BDE8B08FCCFF0208F0FF02081D2D002060
:10D4B0004831002040420F0080B582B002AF42F2F6
:10D4C00010730093044B054A05490648FFF7A4FE74
:10D4D00000BFBD4680BD00BFEFC70008BDC6000845
:10D4E0007DC5000855C5000880B485B000AF7860E0
:10D4F00008E041F6BD23FB6000BFFB685A1EFA60DE
:10D50000002BFAD17B685A1E7A60002BF1D100BF44
:10D5100000BF1437BD4680BC704780B500AF002205
:10D520004FF400714FF0904003F0CFFC0A20FFF75A
:10D53000DBFF01224FF400714FF0904003F0C5FC77
:10D540000A20FFF7D1FF00224FF400714FF0904006
:10D5500003F0BBFC0A20FFF7C7FF01224FF4007164
:10D560004FF0904003F0B1FC0A20FFF7BDFF00220E
:10D570004FF400714FF0904003F0A7FC0A20FFF732
:10D58000B3FF01224FF400714FF0904003F09DFC77
:10D590000A20FFF7A9FF00BF80BD000080B582B060
:10D5A00000AF012000F0AEFA032000F0CFFA002017
:10D5B00000F0CCFA2B2000F0C9FA2B2000F0C6FABC
:10D5C000032000F0C3FA062000F09CFA172000F0B8
:10D5D000BDFA172000F0BAFA172000F0B7FA0420BD
:10D5E00000F090FA00F036FA002000F08BFABF202D
:10D5F00000F0ACFA302000F085FA3C2000F0A6FAEA
:10D60000612000F07FFA802000F0A0FA012000F0F5
:10D610009DFA282000F09AFA822000F073FA142074
:10D6200000F094FA502000F06DFA972000F08EFA86
:10D63000202000F067FA00237B6009E0484A7B68FD
:10D6400013441B78184600F081FA7B6801337B6035
:10D650007B682B2BF2D9212000F054FA00237B6049
:10D6600016E0404B1B78DBB2002B07D03E4A7B68AC
:10D6700013441B78184600F069FA06E03B4A7B68C1
:10D6800013441B78184600F061FA7B6801337B6015
:10D690007B68292BE5D9222000F034FA00237B6037
:10D6A00016E0304B1B78DBB2002B07D0304A7B688A
:10D6B00013441B78184600F049FA06E02D4A7B68AF
:10D6C00013441B78184600F041FA7B6801337B60F5
:10D6D0007B68292BE5D9232000F014FA00237B6016
:10D6E00016E0204B1B78DBB2002B07D0224A7B6868
:10D6F00013441B78184600F029FA06E01F4A7B689D
:10D7000013441B78184600F021FA7B6801337B60D4
:10D710007B68292BE5D9242000F0F4F900237B60F5
:10D7200016E0104B1B78DBB2002B07D0144A7B6845
:10D7300013441B78184600F009FA06E0114A7B688A
:10D7400013441B78184600F001FA7B6801337B60B4
:10D750007B68292BE5D900BF00BF0837BD4680BDD7
:10D76000300803084C3100200C0903085C0803084A
:10D77000380903088808030864090308B408030883
:10D7800090090308E008030880B500AF122000F0FC
:10D79000B9F90220FFF7A8FE00F05CF900BF80BDD8
:10D7A00080B586B000AF78603960FFF7F7FE912052
:10D7B00000F0A8F9902000F0A5F9002000F0C6F9CB
:10D7C0007F2000F0C3F9002000F0C0F9002000F035
:10D7D000BDF9012000F0BAF9272000F0B7F92820A0
:10D7E00000F0B4F910237B814FF494733B81102037
:10D7F00000F088F90023FB8219E00023BB820FE0D0
:10D80000BA8AFB8A798901FB03F313441A467B68C1
:10D8100013441B78184600F099F9BB8A0133BB8288
:10D82000BA8A7B899A42EBD3FB8A0133FB82FA8A5C
:10D830003B899A42E1D3132000F064F900237B82F4
:10D8400019E000233B820FE03A8A7B8A798901FB49
:10D8500003F313441A463B6813441B78184600F040
:10D8600075F93B8A01333B823A8A7B899A42EBD332
:10D870007B8A01337B827B8AB3F5947FE1D3FFF708
:10D8800083FF0023FB8120E00023BB8116E0BA89DF
:10D89000FB89798901FB03F313441A463B681A4458
:10D8A000B989FB89788900FB03F30B4419467B682F
:10D8B0000B4412781A70BB890133BB81BA897B890A
:10D8C0009A42E4D3FB890133FB81FA893B899A426E
:10D8D000DAD300BF00BF1837BD4680BD80B586B023
:10D8E00000AF78601023FB604FF49473BB6010208E
:10D8F00000F008F900233B610FE000237B6105E0A5
:10D90000002000F023F97B6901337B617A69FB68B1
:10D910009A42F5D33B6901333B613A69BB689A424D
:10D92000EBD3132000F0EEF800233B6118E0002356
:10D930007B610EE03B69FA6803FB02F27B691344EA
:10D940007A6813441B78184600F000F97B690133AC
:10D950007B617A69FB689A42ECD33B6901333B6196
:10D960003A69BB689A42E2D3122000F0CBF801205A
:10D97000FFF7BAFD00F06EF800BF1837BD4680BD56
:10D9800080B500AFFAF70EFBFFF7C7FD042000F0EB
:10D99000B9F800F05FF8002000F0B4F89F2000F024
:10D9A000D5F8612000F0AEF8802000F0CFF801201B
:10D9B00000F0CCF8282000F0C9F8502000F0A2F8C0
:10D9C000972000F0C3F800BF80BD80B500AF5020A5
:10D9D00000F098F8F72000F0B9F8022000F092F873
:10D9E00000F038F8072000F08DF8A52000F0AEF820
:10D9F00000BF80BD80B582B000AF102000F082F87B
:10DA000000237B6005E0FF2000F0A0F87B68013375
:10DA10007B607B68B3F5945FF5D3132000F072F858
:10DA200000237B6005E0FF2000F090F87B68013365
:10DA30007B607B68B3F5945FF5D3122000F062F849
:10DA40000120FFF751FD00F005F800BF0837BD4683
:10DA500080BD000080B582B000AF00233B60FAF7C4
:10DA600081FE03463B60712000F04CF84FF480616A
:10DA70000F4803F013FA0346FB71FB79DBB203F0A6
:10DA80000103002B0CBF01230023DBB2FB71FB79E8
:10DA9000DBB2002B07D0FAF765FE02463B68D31ACB
:10DAA000B3F57A6FDFD300BF0837BD4680BD00BF36
:10DAB0000004004880B483B000AF0346FB7100BF90
:10DAC000FB795A1EFA71002BFAD100BF00BF0C3748
:10DAD000BD4680BC7047000080B584B000AF0346EF
:10DAE000FB710023FB73FB79FB7307F10F010A2322
:10DAF0000122034805F014FA00BF1037BD4680BD6F
:10DB00008C2A002080B582B000AF0346FB71012053
:10DB1000FFF7D0FF00224FF400710B4803F0D5F956
:10DB2000002204214FF0904003F0CFF9FB79184612
:10DB3000FFF7D2FF01224FF40071034803F0C5F94B
:10DB400000BF0837BD4680BD0004004880B582B0E4
:10DB500000AF0346FB710120FFF7ACFF00224FF43A
:10DB600000710B4803F0B1F9012204214FF09040FD
:10DB700003F0ABF9FB791846FFF7AEFF01224FF433
:10DB80000071034803F0A1F900BF0837BD4680BD0E
:10DB90000004004880B485B000AF0346FB71FB79F8
:10DBA000224AA2FB03239B08BB73BB7B002B02D141
:10DBB0001323BB7309E0BB7B142B02D90023BB7377
:10DBC00003E0BB7BC3F11403BB730023FB730EE0C4
:10DBD000FB7B03335B00164ABF21D154FB7B5B0008
:10DBE0000733134AE821D154FB7B0133FB73FB7BE2
:10DBF000122BEDD90023FB730EE0FB7B03335B009C
:10DC00000B4A8021D154FB7B5B000733084A082173
:10DC1000D154FB7B0133FB73FA7BBB7B9A42ECD381
:10DC200000BF00BF1437BD4680BC7047CDCCCCCC04
:10DC3000B000002080B485B000AFF86008461146FF
:10DC40001A4603467B810B463B811346FB80214BE2
:10DC500000221A601F4AFB6813601E4A7B891381E9
:10DC60001C4A3B8953811B4A3B8B93817B8903F080
:10DC700007039BB2002B03D17B89DB089BB204E036
:10DC80007B89DB089BB201339BB2124A5382114A53
:10DC90003B8993820F4AFB88D3810E4B00221A8264
:10DCA000FB88002B02D0FB88B42B06D1094A7B8964
:10DCB0009380084A3B89D38006E0064A3B899380DB
:10DCC000044A7B89D38000BF00BF1437BD4680BCA7
:10DCD000704700BF5031002080B483B000AF78603F
:10DCE000034A7B68136000BF0C37BD4680BC704799
:10DCF0005031002080B487B000AF0346FB800B4654
:10DD0000BB8013467B80634B9B88FA889A4200F263
:10DD1000B580604BDB88BA889A4200F2AF805D4BD9
:10DD2000DB89B3F5877F2BD0B3F5877F00F3A8801D
:10DD3000B42B16D0B42B00F3A380002B02D05A2BA7
:10DD400005D09DE0FB88FB82BB88BB8222E0514B63
:10DD50001A89BB88D31A9BB2013BFB82FB88BB822A
:10DD600018E04C4B1A89FB88D31A9BB2013BFB820B
:10DD7000484B5A89BB88D31A9BB2013BBB8209E04E
:10DD8000BB88FB82434B5A89FB88D31A9BB2013B69
:10DD9000BB8200BF3F4B1B8A032B73D801A252F8F2
:10DDA00023F000BFF3DD0008B5DD0008C5DD000885
:10DDB000D5DD0008374B1A89FB8AD31A9BB2013B89
:10DDC000FB8217E0334B5A89BB8AD31A9BB2013BC3
:10DDD000BB820FE02F4B1A89FB8AD31A9BB2013BFF
:10DDE000FB822C4B5A89BB8AD31A9BB2013BBB8264
:10DDF00000E000BF274B1B89FA8A9A4244D8254B82
:10DE00005B89BA8A9A423FD8FB8ADB089BB21946E3
:10DE1000BB8A204A528A02FB03F30B443B611D4B31
:10DE20001A683B6913441B78FB737B88002B13D162
:10DE3000FB8A03F00703802242FA03F35BB2DB4361
:10DE40005AB297F90F30134059B2124B1A683B6916
:10DE50001344CAB21A7018E0FB8A03F00703802249
:10DE600042FA03F35AB297F90F30134359B2094BF0
:10DE70001A683B691344CAB21A7006E000BF04E096
:10DE800000BF02E000BF00E000BF1C37BD4680BC01
:10DE9000704700BF5031002080B485B000AF03460A
:10DEA000FB800023BB811CE00023FB8111E0FA8989
:10DEB000BB891149498A01FB03F31344BB600E4B34
:10DEC0001A68BB681344FA88D2B21A70FB8901330E
:10DED000FB81094B5B8AFA899A42E8D3BB890133FB
:10DEE000BB81054B9B8ABA899A42DDD300BF00BF34
:10DEF0001437BD4680BC70475031002090B585B0C6
:10DF000000AF0446084611461A462346FB800346E6
:10DF1000BB800B467B8013463B80BB88BB8112E0F5
:10DF2000FB88FB8108E03A8CB989FB891846FFF72A
:10DF3000E1FEFB890133FB81FA897B889A42F2D3A7
:10DF4000BB890133BB81BA893B889A42E8D300BFC1
:10DF500000BF1437BD4690BD90B585B000AF0446F4
:10DF6000084611461A462346FB800346BB800B46F3
:10DF70007B8013467B70424B9B88FA889A427AD802
:10DF80003F4BDB88BA889A4275D897F82030012B2E
:10DF900044D10023FB8139E00023BB8129E0FA88CA
:10DFA000B7F90E301A447B78D31A002B28DBBA88D5
:10DFB000B7F90C301A447B78D31A002B20DBFA898E
:10DFC000FB8813449AB27B789BB2D31A98B2BA8971
:10DFD000BB8813449AB27B789BB2D31A9BB27A88DF
:10DFE0001946FFF787FEB7F90C309BB201339BB29D
:10DFF000BB81B7F90C207B785B00013B9A42CEDBFA
:10E00000B7F90E309BB201339BB2FB81B7F90E20FA
:10E010007B785B00013B9A42BEDB2DE00023FB8155
:10E0200023E00023BB8115E0FA89FB8813449BB2EF
:10E03000013B98B2BA89BB8813449BB2013B9BB2A7
:10E040007A881946FFF756FEB7F90C309BB20133B8
:10E050009BB2BB81B7F90C207B789A42E4DBB7F91D
:10E060000E309BB201339BB2FB81B7F90E207B7857
:10E070009A42D6DB00E000BF1437BD4690BD00BF1A
:10E080005031002090B58DB002AF044608461146CD
:10E090001A462346FB800346BB800B467B80134613
:10E0A0003B804B4B9B88FA889A4200F28880484B11
:10E0B000DB88BA889A4200F28280454B9B887A8836
:10E0C0009A427CD8424BDB883A889A4277D8FB88C0
:10E0D000FB84BB88BB847A88FB88D31A002BB8BF2B
:10E0E0005B42BB613A88BB88D31A002BB8BF5B4246
:10E0F0005B427B61FA887B889A4201D2012301E06E
:10E100004FF0FF333B61BA883B889A4201D201232A
:10E1100001E04FF0FF33FB60BA697B6913443B6257
:10E120000023FB77FB7F0133FB7797F83C30012B13
:10E1300017D1FA7F274BA3FB021359080B465B004C
:10E140000B44D31ADBB2002B0BD197F84030B98CBB
:10E15000F88C01220092FF22FFF7FEFE0023FB77DE
:10E1600008E097F840303A8FB98CF88C012400947D
:10E17000FFF7F2FE3B6A5B007A699A420CDCFA8C8C
:10E180007B889A421DD03A6A7B6913443B623B69A3
:10E190009AB2FB8C1344FB843B6A5B00BA699A42D7
:10E1A000C0DBBA8C3B889A420DD03A6ABB691344F3
:10E1B0003B62FB689AB2BB8C1344BB84B2E700BFDE
:10E1C00002E000BF00E000BF2C37BD4690BD00BF9D
:10E1D00050310020ABAAAAAA90B589B004AF04467A
:10E1E000084611461A462346FB800346BB800B4671
:10E1F0007B8013463B80374B9B88FA889A4264D8D1
:10E20000344BDB88BA889A425FD8324B9B887A8835
:10E210009A425AD82F4BDB883A889A4255D897F8B9
:10E220002430002B18D0BB88FB8110E0FC897A8851
:10E23000F989F88897F828300293002301933B8CE2
:10E2400000932346FFF71EFFFB890133FB81FA8908
:10E250003B889A42EAD339E0BC887A88B988F88842
:10E2600097F828300293002301933B8C00932346B8
:10E27000FFF708FF3C88FA88B988F88897F82830B3
:10E280000293002301933B8C00932346FFF7FAFE91
:10E29000BC887A883988788897F8283002930023D8
:10E2A00001933B8C00932346FFF7ECFE3C88FA88F1
:10E2B0003988788897F828300293002301933B8CA3
:10E2C00000932346FFF7DEFE00E000BF1437BD4693
:10E2D00090BD00BF5031002080B588B000AF7B609A
:10E2E0000346FB810B46BB811346FB724C4B9B885C
:10E2F000FA899A4200F28F80494BDB88BA899A42A8
:10E3000000F28980FB7A203B7A68D28802FB03F313
:10E310007A689288D20892B211467A68928802F09E
:10E32000070292B2002A14BF01220022D2B20A448C
:10E3300002FB03F37B617B681A687B691344BB6152
:10E340000023FB8361E00023BB834CE03B8DFF2B6C
:10E3500018D1BB691B781946BB8B03F007038022D9
:10E3600042FA03F30B40002B31D0FA89BB8B1344E4
:10E3700098B2BA89FB8B13449BB2BA8D1946FFF74A
:10E38000B9FC24E0BB691B781946BB8B03F007037B
:10E39000802242FA03F30B40002B0CD0FA89BB8B8E
:10E3A000134498B2BA89FB8B13449BB2BA8D1946B9
:10E3B000FFF7A0FC0BE0FA89BB8B134498B2BA8933
:10E3C000FB8B13449BB23A8D1946FFF793FCBB8B32
:10E3D00003F007039BB2072B02D1BB690133BB617A
:10E3E000BB8B0133BB837B689B88BA8B9A42ADD3CE
:10E3F0007B689B8803F007039BB2002B02D0BB69AC
:10E400000133BB61FB8B0133FB837B68DB88FA8BB9
:10E410009A4298D300E000BF2037BD4680BD00BFC0
:10E420005031002080B588B002AFBA607B600346EF
:10E43000FB810B46BB81FB89FB82BB89BB82214BE5
:10E440009B88FA899A4238D81E4BDB88BA899A424F
:10E4500033D82DE0FB8A7A6892881344194A92884F
:10E46000934206DDFB89FB827B68DA88BB8A134412
:10E47000BB82BB8A7A68D2881344124AD2889342FC
:10E4800003DDFB89FB82BB89BB82BB681A78B98A32
:10E49000F88ABB8C01933B8C00937B68FFF71CFFD1
:10E4A000BB680133BB607B689A88FB8A1344FB829C
:10E4B000BB681B78002BCDD100E000BF1837BD46EC
:10E4C00080BD00BF5031002080B58AB000AF7B60B6
:10E4D0000346FB810B46BB811346FB7200233B6264
:10E4E00000237B610023FB615A4B9B88FA899A4287
:10E4F00000F2AC80574BDB88BA899A4200F2A680C2
:10E500000023FB61FB7A203B7B6100233B6221E01F
:10E510007B681B7A19467B685A683B6A13441B78F0
:10E52000DB08DBB218467B685A683B6A13441B78E9
:10E5300003F00703DBB2002B14BF01230023DBB27F
:10E54000034401FB03F31A46FB691344FB613B6A76
:10E5500001333B623A6A7B699A42D9D37B681A6875
:10E56000FB691344BB610023FB8468E00023BB8488
:10E570004CE0BB8EFF2B18D1BB691B781946BB8CB6
:10E5800003F00703802242FA03F30B40002B31D043
:10E59000FA89BB8C134498B2BA89FB8C13449BB2A2
:10E5A0003A8E1946FFF7A6FB24E0BB691B78194693
:10E5B000BB8C03F00703802242FA03F30B40002BCD
:10E5C0000CD0FA89BB8C134498B2BA89FB8C1344E3
:10E5D0009BB23A8E1946FFF78DFB0BE0FA89BB8C94
:10E5E000134498B2BA89FB8C13449BB2BA8E194675
:10E5F000FFF780FBBB8C03F007039BB2072B02D114
:10E60000BB690133BB61BB8C0133BB847B685A6837
:10E610007B6913441B789BB2BA8C9A42A9D37B685E
:10E620005A687B6913441B7803F00703DBB2002BA5
:10E6300002D0BB690133BB61FB8C0133FB847B6877
:10E640001B7A9BB2FA8C9A4290D300E000BF283725
:10E65000BD4680BD5031002080B588B002AFBA60A1
:10E660007B600346FB810B46BB81FB89FB82BB8938
:10E67000BB8200237B82244B9B88FA899A423FD835
:10E68000214BDB88BA899A423AD834E07B685A68D1
:10E69000BB681B78203B13441B787B82FA8A7B8AF9
:10E6A0001344194A9288934207DDFB89FB827B68F9
:10E6B0001B7A9AB2BB8A1344BB82BB8A7A68127AED
:10E6C0001344114AD288934203DDFB89FB82BB8944
:10E6D000BB82BB681A78B98AF88A3B8C0193BB8CE1
:10E6E00000937B68FFF7F0FEBB680133BB60FA8ADA
:10E6F0007B8A1344FB82BB681B78002BC6D100E0E9
:10E7000000BF1837BD4680BD5031002080B588B0AD
:10E7100000AF7B600346FB810B46BB811346FB7257
:10E72000514B9B88FA899A4200F29A804E4BDB88C3
:10E73000BA899A4200F2948000237B61FB7A3B61A4
:10E740007B685B791A463B6902FB03F37A681279AE
:10E75000D208D2B211467A68127902F00702D2B218
:10E76000002A14BF01220022D2B20A4402FB03F3A2
:10E770007B617B681A687B691344BB617B681A689C
:10E780007B691344BB610023FB8362E00023BB83EE
:10E790004CE03B8DFF2B18D1BB691B781946BB8B16
:10E7A00003F00703802242FA03F30B40002B31D021
:10E7B000FA89BB8B134498B2BA89FB8B13449BB282
:10E7C000BA8D1946FFF796FA24E0BB691B78194603
:10E7D000BB8B03F00703802242FA03F30B40002BAC
:10E7E0000CD0FA89BB8B134498B2BA89FB8B1344C3
:10E7F0009BB2BA8D1946FFF77DFA0BE0FA89BB8B05
:10E80000134498B2BA89FB8B13449BB23A8D1946D4
:10E81000FFF770FABB8B03F007039BB2072B02D103
:10E82000BB690133BB61BB8B0133BB837B681B7945
:10E830009BB2BA8B9A42ACD37B681B7903F0070377
:10E84000DBB2002B02D0BB690133BB61FB8B013310
:10E85000FB837B685B799BB2FA8B9A4296D300E08C
:10E8600000BF2037BD4680BD5031002080B485B048
:10E8700000AF78604FF0B043DA6C4FF0B0417B6886
:10E880001343CB644FF0B043DA6C7B681340FB60FA
:10E89000FB6800BF1437BD4680BC704780B586B0AA
:10E8A00000AF3B1D00221A605A609A60DA601A615C
:10E8B0000120FFF7DBFF10237B600123BB600023F7
:10E8C000FB6003233B613B1D19464FF0904002F073
:10E8D000B7F820237B603B1D19464FF0904002F0B3
:10E8E000AFF8002220214FF0904002F0EEFA002213
:10E8F00010214FF0904002F0E8FA00231846183734
:10E90000BD4680BD80B582B000AF0346FB71FB7988
:10E91000032B3FD801A252F823F000BF2DE90008D5
:10E9200047E9000861E900087BE90008002210219E
:10E930004FF0904002F0C9FA002220214FF09040A1
:10E9400002F0C3FA27E0012210214FF0904002F0BC
:10E95000BCFA002220214FF0904002F0B6FA1AE0F3
:10E96000012210214FF0904002F0AFFA0122202145
:10E970004FF0904002F0A9FA0DE0002210214FF074
:10E98000904002F0A2FA012220214FF0904002F0C4
:10E990009CFA00E000BF002318460837BD4680BD42
:10E9A00080B400AF02231846BD4680BC704780B4D7
:10E9B00000AF01231846BD4680BC704780B400AF4D
:10E9C00001231846BD4680BC704780B400AF00BF2D
:10E9D000BD4680BC7047000080B582B000AF002308
:10E9E000FB71032001F09EF903F04AFB0346094A3C
:10E9F00013600F20F9F7ACFE0346002B02D0012371
:10EA0000FB7101E0F9F770FCFB7918460837BD4649
:10EA100080BD00BF1801002080B400AF044B1B680C
:10EA2000034A23F00203136000BFBD4680BC704759
:10EA300010E000E080B400AF044B1B68034A43F0D1
:10EA40000203136000BFBD4680BC704710E000E0C9
:10EA500080B400AF024B1B681846BD4680BC7047AF
:10EA60009075FF1F80B400AF024B1B681846BD466F
:10EA700080BC70479475FF1F80B400AF024B1B68C9
:10EA80001846BD4680BC70479875FF1F80B483B0A0
:10EA900000AF786039607B681B6823F0E0723B68E8
:10EAA0001A437B681A6000BF0C37BD4680BC7047B4
:10EAB00080B483B000AF78607B681B6803F0E073BC
:10EAC00018460C37BD4680BC704780B485B000AF97
:10EAD000F860B9607A60FB685A69BB6803F00403A8
:10EAE000072101FA03F3DB431A40BB6803F0040378
:10EAF000796801FA03F31A43FB685A6100BF1437BF
:10EB0000BD4680BC704780B483B000AF7860396088
:10EB10007B685A693B6803F00403072101FA03F399
:10EB20001A403B6803F0040322FA03F318460C373B
:10EB3000BD4680BC704780B483B000AF78607B680E
:10EB4000DB6803F44063002B01D1012300E00023C4
:10EB500018460C37BD4680BC704780B485B000AF06
:10EB6000F860B9607A60FB689A6ABB6803F01F03BB
:10EB70000F2101FA03F3DB431A407B689B0E03F07D
:10EB80000F01BB6803F01F0301FA03F31A43FB688C
:10EB90009A6200BF1437BD4680BC704780B483B012
:10EBA00000AF786039607B689A6A3B68C3F31103F1
:10EBB0001A437B689A6200BF0C37BD4680BC704721
:10EBC00080B483B000AF786039607B689A6A3B6834
:10EBD000C3F31103DB431A407B689A6200BF0C3712
:10EBE000BD4680BC704780B485B000AFF860B960A6
:10EBF0007A60FB685A69BB681B02DB431A40BB683A
:10EC000019027B680B4023F07C4323F0FF031A4377
:10EC1000FB685A6100BF1437BD4680BC704780B4A2
:10EC200083B000AF78607B689B6823F0104323F0CB
:10EC3000170343F080527B689A6000BF0C37BD46D3
:10EC400080BC704780B483B000AF78607B689B68FD
:10EC500023F0104323F017037A68936000BF0C374A
:10EC6000BD4680BC704780B483B000AF78607B68DD
:10EC70009B6803F08053B3F1805F01D1012300E072
:10EC8000002318460C37BD4680BC704780B483B063
:10EC900000AF78607B689B6823F0004323F0170384
:10ECA00043F001027B689A6000BF0C37BD4680BC10
:10ECB000704780B483B000AF78607B689B6823F0B6
:10ECC000004323F0170343F002027B689A6000BF01
:10ECD0000C37BD4680BC704780B483B000AF78600D
:10ECE0007B689B6803F00103012B01D1012300E045
:10ECF000002318460C37BD4680BC704780B483B0F3
:10ED000000AF78607B689B6803F00203022B01D19F
:10ED1000012300E0002318460C37BD4680BC704735
:10ED200080B483B000AF78607B689B6823F00043B9
:10ED300023F0170343F004027B689A6000BF0C378E
:10ED4000BD4680BC704780B483B000AF78607B68FC
:10ED50009B6823F0004323F0170343F010027B6805
:10ED60009A6000BF0C37BD4680BC704780B483B04A
:10ED700000AF78607B689B6803F00403042B01D12B
:10ED8000012300E0002318460C37BD4680BC7047C5
:10ED900080B588B000AF78600023FB770023BB61AB
:10EDA00000237B610023BB607B68002B01D1012322
:10EDB0009EE17B681B69002B7B689B6D002B09D152
:10EDC0007868F7F7D1FC7B680022DA657B6800225F
:10EDD00083F854207B681B681846FFF744FF0346FE
:10EDE000002B15D17B681B681846FFF718FF994B5D
:10EDF0001B689B09984AA2FB03239B0901335B0014
:10EE0000BB6002E0BB68013BBB60BB68002BF9D173
:10EE10007B681B681846FFF726FF0346002B0DD1C1
:10EE20007B689B6D43F010027B689A657B68DB6DA5
:10EE300043F001027B68DA650123FB777B681B687E
:10EE40001846FFF793FFF8607B689B6D03F0100393
:10EE5000002B40F04481FB68002B40F040817B6830
:10EE60009B6D23F4817343F002027B689A657B6893
:10EE70001B681846FFF730FF0346002B40F0A780C1
:10EE80007B689A687B681B7E9B031A437B685B7E6A
:10EE9000DB031A437B689B7E5B0313437A68126B28
:10EEA000002A02D04FF4805200E000221A437B680F
:10EEB000DB681A437B681B69002B04DA7B681B69DB
:10EEC00023F0004301E04FF400131A437B6893F8EA
:10EED0002C305B001343BA691343BB617B6893F822
:10EEE0002030012B14D17B689B7E002B04D1BB69A1
:10EEF00043F48033BB610BE07B689B6D43F02002E1
:10EF00007B689A657B68DB6D43F001027B68DA659C
:10EF10007B685B6A002B09D07B685B6A03F4E07254
:10EF20007B689B6A1343BA691343BB617B681B68A8
:10EF3000DB6823F4FE3323F4FF737A681268B9693F
:10EF40000B43D3607B685B6803F040427B68DB6CFB
:10EF500013437A6913437B617B6893F83C30012B40
:10EF600011D17B685B6803F040427B681B6C1A43DD
:10EF70007B685B6C1A437B689B6C1A437B69134309
:10EF800043F001037B617B681B681A69334B1340B4
:10EF90007A68126879690B4313617B685B68B3F127
:10EFA000404F14D07B685B68B3F1804F0FD07B6813
:10EFB0005B68B3F1004F0AD0294B1B6823F4701231
:10EFC0007B685B6803F47013254913430B607B680F
:10EFD00018687B685B6B1A460021FFF776FD7B683B
:10EFE00018687B689B6B1A461E49FFF76EFD7B68AD
:10EFF0001B69002B08D17B681B689A6A7B681B68B9
:10F0000062F00F029A6242E07B681B69B3F5001F51
:10F010003DD100233B610CE07B681A6E3B699B008D
:10F0200022FA03F303F00F030F2B06D03B690133E1
:10F030003B613B69072BEFD900E000BF3B69012B27
:10F0400012D17B681B689A6A7B681B6862F00F02AA
:10F050009A621CE018010020632D3E0502FCFF1F90
:10F060000827014004FFFF037B681B689B6A7B68DD
:10F07000DB69013B9B0003F01C036FF00F0202FAF7
:10F0800003F17B681A6E7B681B680A439A627B688F
:10F090001B6800211846FFF736FD02467B685B6B54
:10F0A0009A420BD17B680022DA657B689B6D23F066
:10F0B000030343F001027B689A6518E07B689B6D4F
:10F0C00023F0120343F010027B689A657B68DB6DC6
:10F0D00043F001027B68DA650123FB7707E07B6878
:10F0E0009B6D43F010027B689A650123FB77FB7FE1
:10F0F00018462037BD4680BD80B584B000AF78602B
:10F100007B68002B01D101236AE07B689B6D43F093
:10F1100002027B689A65786800F0BEFA0346FB73CA
:10F12000FB7B002B0FD1786800F082FB0346FB735A
:10F13000FB7B002B02D17B6801229A657B681B68F0
:10F140001846FFF77FFD7B681B685B687A6812686A
:10F1500023F4677323F0030353607B681B6840F25A
:10F160009F321A607B681B68D9687B681A681E4BDF
:10F170000B40D3607B681B681A697B681B6822F0B0
:10F1800040421A617B681B685A697B681B6822F0E1
:10F1900007025A617B681B681A6A7B681B6802F069
:10F1A000F0221A627B681B689B6A7B681B680022DE
:10F1B0009A620E4B1B680D4A23F0FE731360786849
:10F1C000F7F7E6FA7B6800221A667B680022DA65A8
:10F1D0007B6800229A657B68002283F85420FB7BC1
:10F1E00018461037BD4680BD00023E830827014007
:10F1F00080B584B000AF78607B681B681846FFF765
:10F20000B5FD0346002B32D17B6893F85430012BB7
:10F2100001D102232EE07B68012283F85420786814
:10F2200000F080FA0346FB73FB7B002B1AD17B684E
:10F230009B6D23F4706323F0010343F480727B68B9
:10F240009A657B680022DA657B681B681C221A605D
:10F250007B68002283F854207B681B681846FFF700
:10F260005FFD06E07B68002283F8542001E0022362
:10F27000FB73FB7B18461037BD4680BD80B584B05C
:10F2800000AF78607B6893F85430012B01D10223E2
:10F2900022E07B68012283F85420786800F0FCF9B2
:10F2A0000346FB73FB7B002B11D1786800F0C0FA9A
:10F2B0000346FB73FB7B002B09D17B689B6D23F41A
:10F2C000807323F0010343F001027B689A657B6839
:10F2D000002283F85420FB7B18461037BD4680BDC2
:10F2E00080B584B000AF786039607B685B69082BBB
:10F2F00002D10823FB6010E07B681B68DB6803F029
:10F300000103002B07D07B689B6D43F020027B68D4
:10F310009A65012377E00423FB60F9F723FAB860CC
:10F3200021E03B68B3F1FF3F1DD0F9F71BFA02461D
:10F33000BB68D31A3A689A4202D33B68002B12D1B9
:10F340007B681B681A68FB681340002B0BD17B6835
:10F350009B6D43F004027B689A657B68002283F80A
:10F36000542003234FE07B681B681A68FB68134036
:10F37000002BD6D07B689B6D43F400727B689A6546
:10F380007B681B681846FFF7D6FB0346002B31D07D
:10F390007B689B7E002B2DD17B681B681B6803F06C
:10F3A0000803082B26D17B681B681846FFF7DEFC94
:10F3B0000346002B12D17B681B685A687B681B6868
:10F3C00022F00C025A607B689B6D23F4807323F05B
:10F3D000010343F001027B689A650BE07B689B6D3B
:10F3E00043F020027B689A657B68DB6D43F0010285
:10F3F0007B68DA657B681B7E002B03D17B681B680A
:10F400000C221A60002318461037BD4680BD80B418
:10F4100083B000AF78607B681B681B6C18460C37A4
:10F42000BD4680BC7047000080B588B000AF7860F2
:10F4300039600023FB770023BB607B681B69B3F155
:10F44000004F7B6893F85430012B01D1022310E167
:10F450007B68012283F854207B681B681846FFF7FD
:10F4600085FC0346002B40F0F7803B685B68022B6D
:10F4700000F0B1807B681B69B3F1004F04D07B685A
:10F480001B697E4A934208D17B681A683B681B68F7
:10F4900019461046FFF782FB41E07B681A6E3B6815
:10F4A0005B6803F01F030F2101FA03F3DB431A40EB
:10F4B0003B681B68C3F31103002B05D13B681B6835
:10F4C0009B0E03F01F0311E03B681B683B613B6927
:10F4D00093FAA3F3FB60FB687B617B69002B01D18E
:10F4E000202303E07B69B3FA83F3DBB23968496810
:10F4F00001F01F018B401A437B681A663B685B680A
:10F500009B085A1C7B68DB699A4208D87B6818689C
:10F510003B6859683B681B681A46FFF71EFB7B680F
:10F5200018683B6819683B689B681A46FFF75BFBE5
:10F530003B681B68002B80F297805148FFF7B8FAB0
:10F54000B8613B681B684F4A934220D1BB6903F402
:10F550000003002B1BD1BB6943F400031946484844
:10F56000FFF794FA484B1B689B09484AA2FB032308
:10F570009B095A1C13465B0013449B00BB6002E0CE
:10F58000BB68013BBB60BB68002BF9D16CE03B68FA
:10F590001B683F4A93420CD1BB6903F08073002B78
:10F5A00007D1BB6943F0807319463548FFF76EFAFF
:10F5B0005AE03B681B68374A934255D1BB6903F454
:10F5C0008003002B50D1BB6943F4800319462C48BB
:10F5D000FFF75CFA48E07B681B69B3F1004F04D089
:10F5E0007B681B69254A934207D17B681A683B6890
:10F5F0001B6819461046FFF7E3FA3B681B68002BAF
:10F6000032DA1F48FFF754FAB8613B681B681D4A9D
:10F61000934207D1BB6923F4000319461848FFF74A
:10F6200035FA21E03B681B68194A934207D1BB6950
:10F6300023F0807319461248FFF728FA14E03B685C
:10F640001B68144A93420FD1BB6923F48003194607
:10F650000B48FFF71BFA07E07B689B6D43F0200225
:10F660007B689A650123FB777B68002283F854202E
:10F67000FB7F18462037BD4680BD00BF04000080D8
:10F6800008270140001000B018010020632D3E053E
:10F69000004000B8002000B480B584B000AF7860AE
:10F6A0007B681B681846FFF761FB0346002B33D0CD
:10F6B0007B681B681846FFF721FB0346002B04D12B
:10F6C0007B681B681846FFF73EFBF9F74BF8F860BC
:10F6D0001BE0F9F747F80246FB68D31A022B14D94E
:10F6E0007B681B689B6803F00403002B0DD07B68CC
:10F6F0009B6D43F010027B689A657B68DB6D43F07D
:10F7000001027B68DA65012307E07B681B689B6860
:10F7100003F00403002BDCD1002318461037BD464C
:10F7200080BD000080B584B000AF78600023BB606E
:10F730007B681B681846FFF7CFFA0346002B69D198
:10F740007B681B689A68364B1340002B0DD07B6892
:10F750009B6D43F010027B689A657B68DB6D43F01C
:10F7600001027B68DA65012355E07B681B68184657
:10F77000FFF78CFA2B48FFF79BF9034603F40003CD
:10F78000002B0FD0284B1B689B09284AA2FB0323A0
:10F790009B090133BB6002E0BB68013BBB60BB68F7
:10F7A000002BF9D17B685B7E012B33D0F8F7DAFFB1
:10F7B000F86028E07B681B681846FFF78DFA03465F
:10F7C000002B04D17B681B681846FFF75FFAF8F737
:10F7D000C9FF0246FB68D31A022B14D97B681B6849
:10F7E0001B6803F00103012B0DD07B689B6D43F078
:10F7F00010027B689A657B68DB6D43F001027B68D1
:10F80000DA65012307E07B681B681B6803F00103CE
:10F81000012BCFD1002318461037BD4680BD00BF55
:10F82000170000800827014018010020632D3E05C5
:10F8300080B584B000AF78607B681B681846FFF71E
:10F840005DFAF8607B681B681846FFF745FA0346C7
:10F85000002B47D0FB68002B44D17B681B689B685A
:10F8600003F00503012B0CD17B681B681846FFF7DA
:10F8700020FA7B681B6803221A60F8F773FFB860F0
:10F8800029E07B689B6D43F010027B689A657B687A
:10F89000DB6D43F001027B68DA65012323E0F8F7B2
:10F8A00061FF0246BB68D31A022B14D97B681B6820
:10F8B0009B6803F00103002B0DD07B689B6D43F028
:10F8C00010027B689A657B68DB6D43F001027B6800
:10F8D000DA65012307E07B681B689B6803F001037E
:10F8E000002BDCD1002318461037BD4680BD80B404
:10F8F00083B000AF786039607B68D3F8B43023F010
:10F900007F023B681A437B68C3F8B42000BF0C3702
:10F91000BD4680BC704780B483B000AF78607B6820
:10F92000D3F8B43003F07F0318460C37BD4680BCD3
:10F93000704780B483B000AF78607B689B6823F029
:10F94000004323F0170343F001027B689A6000BF75
:10F950000C37BD4680BC704780B483B000AF786080
:10F960007B689B6823F0004323F0170343F00202F7
:10F970007B689A6000BF0C37BD4680BC704780B47E
:10F9800083B000AF78607B689B6803F00103012BB4
:10F9900001D1012300E0002318460C37BD4680BC8E
:10F9A000704780B483B000AF78607B689B6823F0B9
:10F9B000004323F0170343F000427B689A6000BFC6
:10F9C0000C37BD4680BC704780B483B000AF786010
:10F9D0007B689B6803F00043B3F1004F01D1012322
:10F9E00000E0002318460C37BD4680BC704780B548
:10F9F00088B000AF78600023BB600023BB617B68E8
:10FA000093F85430012B01D10223B9E07B68012225
:10FA100083F854207868FFF70BFF0346FB757B687B
:10FA20001B681846FFF7ABFF0346002B40F09D8094
:10FA30007B689B6D23F4817343F002027B689A65B7
:10FA40007B681B68DA6848F2030313403B617B68FC
:10FA50001B68DB687A68126823F4004323F0030311
:10FA6000D3600023FB612EE07B681B681846FFF71C
:10FA700098FF14E0BB680133BB60BB68B3F52E3F51
:10FA80000DD37B689B6D23F0120343F010027B685B
:10FA90009A657B68002283F85420012370E07B681C
:10FAA0001B681846FFF790FF0346002BE2D17B68E6
:10FAB0001B681846FFF72FFF0246BB691344BB6162
:10FAC000FB690133FB61FB69072BCDD9BA69FB697F
:10FAD000B2FBF3F3BB617B681B681846FFF729FF95
:10FAE0007B681B68B9691846FFF701FF7B681B68D4
:10FAF0001846FFF731FFF8F735FEF8601CE0F8F71D
:10FB000031FE0246FB68D31A022B15D97B681B68AD
:10FB10001846FFF734FF0346002B0DD07B689B6D22
:10FB200043F010027B689A657B68DB6D43F001024D
:10FB30007B68DA65012323E07B681B681846FFF7C2
:10FB40001EFF0346002BDAD17B681B68D9687B68EF
:10FB50001B683A690A43DA607B689B6D23F00303F4
:10FB600043F001027B689A6505E07B689B6D43F07A
:10FB700010027B689A657B68002283F85420FB7D25
:10FB800018462037BD4680BD80B485B000AF786090
:10FB90007B6803F00703FB600C4BDB68BB60BA6853
:10FBA0004FF6FF031340BB60FB681A02BB681343A8
:10FBB00043F0BF6343F40033BB60044ABB68D360C7
:10FBC00000BF1437BD4680BC704700BF00ED00E0A9
:10FBD00080B400AF044BDB681B0A03F00703184630
:10FBE000BD4680BC704700BF00ED00E080B483B02C
:10FBF00000AF0346FB7197F90730002B0BDBFB7955
:10FC000003F01F02064997F907305B09012000FA4B
:10FC100002F241F8232000BF0C37BD4680BC70477C
:10FC200000E100E080B483B000AF0346FB7197F9B8
:10FC30000730002B12DBFB7903F01F020A4997F90A
:10FC400007305B09012000FA02F2203341F823203B
:10FC5000BFF34F8F00BFBFF36F8F00BF00BF0C37E4
:10FC6000BD4680BC704700BF00E100E080B483B0B7
:10FC700000AF03463960FB7197F90730002B0ADBB0
:10FC80003B68DAB20C4997F907301201D2B20B4443
:10FC900083F800230AE03B68DAB20849FB7903F0F5
:10FCA0000F03043B1201D2B20B441A7600BF0C378B
:10FCB000BD4680BC704700BF00E100E000ED00E001
:10FCC00080B489B000AFF860B9607A60FB6803F077
:10FCD0000703FB61FB69C3F10703042B28BF04235F
:10FCE000BB61FB690433062B02D9FB69033B00E0CF
:10FCF00000237B614FF0FF32BB6902FA03F3DA4362
:10FD0000BB681A407B699A404FF0FF317B6901FA6A
:10FD100003F3D9437B680B40134318462437BD4691
:10FD200080BC704780B582B000AF78607868FFF71C
:10FD30002BFF00BF0837BD4680BD80B586B000AF41
:10FD40000346B9607A60FB73FFF742FF78617A6817
:10FD5000B9687869FFF7B4FF024697F90F3011468A
:10FD60001846FFF783FF00BF1837BD4680BD80B53A
:10FD700082B000AF0346FB7197F907301846FFF7D2
:10FD800035FF00BF0837BD4680BD80B582B000AFEB
:10FD90000346FB7197F907301846FFF743FF00BF92
:10FDA0000837BD4680BD000080B582B000AF7860E6
:10FDB0007B68002B01D101238EE07B681B681A460B
:10FDC000474B9A420FD87B681B681A46454B134431
:10FDD000454AA2FB03231B099A007B685A647B688F
:10FDE000424A1A640EE07B681B681A46404B134473
:10FDF0003D4AA2FB03231B099A007B685A647B6877
:10FE00003C4A1A647B68022283F825207B681B68C1
:10FE10001B687A68126823F4FF4323F070031360B1
:10FE20007B681B6819687B689A687B68DB681A4383
:10FE30007B681B691A437B685B691A437B689B6913
:10FE40001A437B68DB691A437B681B6A1A437B6829
:10FE50001B680A431A60786800F024FB7B689B6883
:10FE6000B3F5804F02D17B6800225A607B685A68E4
:10FE70007B689B6C02F07F021A607B68DB6C7A689F
:10FE8000126D5A607B685B68002B10D07B685B68E2
:10FE9000042B0CD8786800F04DFB7B685B6D00226A
:10FEA0001A607B689B6D7A68D26D5A6008E07B6847
:10FEB00000225A657B6800229A657B680022DA6519
:10FEC0007B680022DA637B68012283F825207B6847
:10FED000002283F82420002318460837BD4680BD41
:10FEE00007040240F8FFFDBFCDCCCCCC000002409F
:10FEF000F8FBFDBF0004024080B582B000AF78601F
:10FF00007B68002B01D101237BE07B681B681A68AA
:10FF10007B681B6822F001021A607B681B681A4626
:10FF20003A4B9A420FD87B681B681A46384B1344E9
:10FF3000384AA2FB03231B099A007B685A647B683A
:10FF4000354A1A640EE07B681B681A46334B13442B
:10FF5000304AA2FB03231B099A007B685A647B6822
:10FF60002F4A1A647B681B6800221A607B685B6CEE
:10FF700003F01C027B681B6C012101FA02F25A603B
:10FF8000786800F08FFA7B689B6C00221A607B68AF
:10FF9000DB6C7A68126D5A607B685B68002B0FD04F
:10FFA0007B685B68042B0BD8786800F0C3FA7B6829
:10FFB0005B6D00221A607B689B6D7A68D26D5A6017
:10FFC0007B6800225A657B6800229A657B68002264
:10FFD000DA657B680022DA627B6800221A637B683C
:10FFE00000225A637B6800229A637B680022DA63EE
:10FFF0007B68002283F825207B68002283F8242078
:020000040801F1
:10000000002318460837BD4680BD00BF07040240E4
:10001000F8FFFDBFCDCCCCCC00000240F8FBFDBF0B
:100020000004024080B586B000AFF860B9607A6025
:100030003B600023FB75FB6893F82430012B01D152
:10004000022369E0FB68012283F82420FB6893F80F
:100050002530DBB2012B55D1FB68022283F8252025
:10006000FB680022DA63FB681B681A68FB681B6880
:1000700022F001021A603B687A68B968F86800F0FB
:10008000D3F9FB681B6B002B08D0FB681B681A6850
:10009000FB681B6842F00E021A600FE0FB681B68E9
:1000A0001A68FB681B6822F004021A60FB681B6870
:1000B0001A68FB681B6842F00A021A60FB689B6CB6
:1000C0001B6803F48033002B07D0FB689B6C1A6815
:1000D000FB689B6C42F480721A60FB685B6D002BBE
:1000E00007D0FB685B6D1A68FB685B6D42F4807239
:1000F0001A60FB681B681A68FB681B6842F0010203
:100100001A6008E0FB688022DA63FB68002283F84B
:1001100024200123FB75FB7D18461837BD4680BDA2
:1001200080B483B000AF78607B68002B01D10123DD
:100130004FE07B6893F82530DBB2022B08D07B6858
:100140000422DA637B68002283F82420012340E044
:100150007B681B681A687B681B6822F00E021A60B5
:100160007B689B6C1A687B689B6C22F480721A60B7
:100170007B681B681A687B681B6822F001021A60A2
:100180007B685B6C03F01C027B681B6C012101FA2D
:1001900002F25A607B68DB6C7A68126D5A607B6889
:1001A0005B6D002B0CD07B685B6D1A687B685B6DA8
:1001B00022F480721A607B689B6D7A68D26D5A60F7
:1001C0007B68012283F825207B68002283F82420A5
:1001D000002318460C37BD4680BC704780B584B0FC
:1001E00000AF78600023FB737B6893F82530DBB2A7
:1001F000022B05D07B680422DA630123FB7347E0FE
:100200007B681B681A687B681B6822F00E021A6004
:100210007B681B681A687B681B6822F001021A6001
:100220007B689B6C1A687B689B6C22F480721A60F6
:100230007B685B6C03F01C027B681B6C012101FA7C
:1002400002F25A607B68DB6C7A68126D5A607B68D8
:100250005B6D002B0CD07B685B6D1A687B685B6DF7
:1002600022F480721A607B689B6D7A68D26D5A6046
:100270007B68012283F825207B68002283F82420F4
:100280007B689B6B002B03D07B689B6B78689847DF
:10029000FB7B18461037BD4680BD000080B584B09A
:1002A00000AF78607B681B6C1B68FB607B681B6819
:1002B0001B68BB607B685B6C03F01C0304229A40E4
:1002C000FB681340002B27D0BB6803F00403002B0E
:1002D00022D07B681B681B6803F02003002B07D12A
:1002E0007B681B681A687B681B6822F004021A602E
:1002F0007B685B6C03F01C027B681B6C042101FAB9
:1003000002F25A607B681B6B002B00F081807B68D7
:100310001B6B786898477BE07B685B6C03F01C0381
:1003200002229A40FB681340002B3DD0BB6803F0CB
:100330000203002B38D07B681B681B6803F0200386
:10034000002B0BD17B681B681A687B681B6822F046
:100350000A021A607B68012283F825207B681B68EB
:100360001A462E4B9A4209D97B685B6C03F01C033A
:100370002B4A022101FA03F3536008E07B685B6CAF
:1003800003F01C03274A022101FA03F353607B6840
:10039000002283F824207B68DB6A002B38D07B683E
:1003A000DB6A7868984733E07B685B6C03F01C037A
:1003B00008229A40FB681340002B2AD0BB6803F048
:1003C0000803002B25D07B681B681A687B681B68B4
:1003D00022F00E021A607B685B6C03F01C027B68E3
:1003E0001B6C012101FA02F25A607B680122DA6378
:1003F0007B68012283F825207B68002283F8242073
:100400007B685B6B002B04D07B685B6B78689847DC
:1004100000BF00BF1037BD4680BD00BF8000024056
:10042000000402400000024080B485B000AFF860D4
:10043000B9607A603B60FB68DB6CFA68126D5A60E9
:10044000FB685B6D002B04D0FB689B6DFA68D26D76
:100450005A60FB685B6C03F01C02FB681B6C01219B
:1004600001FA02F25A60FB681B683A685A60FB683E
:100470009B68102B08D1FB681B687A689A60FB6840
:100480001B68BA68DA6007E0FB681B68BA689A60A4
:10049000FB681B687A68DA6000BF1437BD4680BC11
:1004A0007047000080B485B000AF78607B681B683F
:1004B0001A461C4B9A4213D87B685B6C9B089B00C6
:1004C00003F1804303F502337A6893647B681B6809
:1004D000DBB2083B144AA2FB03231B09FB6011E0BB
:1004E0007B685B6C9B089A00104B13447A6893649A
:1004F0007B681B68DBB2083B0B4AA2FB03231B098A
:100500000733FB607B680A4ADA64FB6803F01F0369
:1005100001229A407B681A6500BF1437BD4680BC33
:10052000704700BF07040240CDCCCCCC1C08024071
:100530008008024080B485B000AF78607B685B685B
:1005400003F07F03FB60FA680A4B13449B001A46D2
:100550007B685A657B68084A9A65FB68013B03F033
:10056000030301229A407B68DA6500BF1437BD4659
:1005700080BC70473F8200104009024080B586B0C1
:1005800000AFF860B960C7E900231C4B1B78012B52
:1005900001D102232DE0194B01221A70174B0022C2
:1005A0005A604FF47A7000F069F80346FB75FB7DE2
:1005B000002B1AD1FB68012B05D1D7E90023B868BD
:1005C00000F0BEF804E03B681946B86800F0DEF8B9
:1005D0004FF47A7000F052F80346FB75084B5A69E5
:1005E000FB68DB43064913404B61044B00221A7041
:1005F000FB7D18461837BD4680BD00BF6C3100201A
:100600000040005880B483B000AF0023FB710B4B57
:100610005B69002B0BDA094B094A9A60074B094AC0
:100620009A60064B5B69002B01DA0123FB71FB79B1
:1006300018460C37BD4680BC704700BF00400058CC
:1006400023016745AB89EFCD80B483B000AF0023B1
:10065000FB71094B5B69084A43F000435361064B49
:100660005B69002B01DB0123FB71FB7918460C371A
:10067000BD4680BC704700BF0040005880B584B0C4
:1006800000AF7860F8F76EF8F86009E0F8F76AF8FC
:100690000246FB68D31A7A689A4201D8032347E0DE
:1006A000254B1B6903F48033B3F5803FEED0224B1A
:1006B0001B69BB60BB6803F00103002B02D01E4B1B
:1006C00001221A61BA684CF2FA331340BB60BB686E
:1006D00003F04043002B07D0174B9A69BB6803F027
:1006E0004043154913438B61BB6823F04043002B03
:1006F00004D0114ABB6823F040431361BB68002B50
:100700000ED00E4ABB685360012311E0F8F72AF8B7
:100710000246FB68D31A7A689A4201D8032307E09D
:10072000054B1B6903F48023B3F5802FEED0002323
:1007300018461037BD4680BD004000586C3100207F
:1007400080B485B000AFF860C7E900230E4B5B6949
:100750000D4A43F001035361FB683A681A60BFF326
:100760006F8F00BFD7E900014FF000024FF0000388
:100770000A000023F968043113460B6000BF1437E8
:10078000BD4680BC704700BF0040005880B489B0AF
:1007900000AF786039604023FB777B68BB613B68C2
:1007A0007B61184B5B69174A43F480235361EFF375
:1007B0001083FB60FB683B6172B600BF7B691A68FF
:1007C000BB691A60BB690433BB617B6904337B611D
:1007D000FB7F013BFB77FB7F002BEFD100BF094B79
:1007E0001B6903F48033B3F5803FF8D03B69BB60ED
:1007F000BB6883F3108800BF00BF2437BD4680BCB0
:10080000704700BF0040005880B584B000AF7860EA
:100810003960284B1B78012B01D1022346E0254B80
:1008200001221A70234B00225A604FF47A70FFF7AE
:1008300025FF0346FB73FB7B002B33D17B681B68D2
:10084000042B08D100F080F84FF47A70FFF716FF00
:100850000346FB7324E03B684FF0FF321A607B686D
:100860005B68BB6012E0B86800F07EF84FF47A7005
:10087000FFF704FF0346FB73FB7B002B03D03B68B1
:10088000BA681A600AE0BB680133BB607B685A68CB
:100890007B689B681344BA689A42E4D300F0C0F8BE
:1008A00000F07AF8034B00221A70FB7B18461037D1
:1008B000BD4680BD6C31002080B584B000AF78604B
:1008C0001F4B1B78012B01D1022334E01C4B01226A
:1008D0001A701B4B00225A607B681B68184A936091
:1008E0004FF47A70FFF7CAFE0346FB73FB7B002BC5
:1008F00003D0134B00221A701CE0124B5B69114AA3
:1009000043F0407353617B681B68042B05D10C4B8B
:1009100000221A6100F018F80CE07B689B68084A16
:1009200053617B685B68064A13617B685B681846A5
:1009300000F01AF8FB7B18461037BD4680BD00BF9B
:100940006C3100200040005880B400AF054B5B695B
:10095000044A43F4803343F00403536100BFBD46AF
:1009600080BC70470040005880B483B000AF78600E
:10097000084B5B6923F47E727B68DB001343054AF6
:1009800043F4803343F00203536100BF0C37BD468C
:1009900080BC70470040005880B400AF1F4B1B68FC
:1009A00003F40073012B17D11C4B1B681B4A23F463
:1009B00000731360194B1B68184A43F400631360FB
:1009C000164B1B68154A23F400631360134B1B6816
:1009D000124A43F400731360104B1B6803F48063E6
:1009E000012B17D10D4B1B680C4A23F48063136055
:1009F0000A4B1B68094A43F480531360074B1B687A
:100A0000064A23F480531360044B1B68034A43F4E3
:100A10008063136000BFBD4680BC70470040005833
:100A200080B400AF054B5B69044A23F47E7323F066
:100A30000203536100BFBD4680BC704700400058B0
:100A400080B487B000AF7860396000237B6140E1FB
:100A50003B681A6801217B6901FA03F31340FB60CC
:100A6000FB68002B00F032813B685B6803F00303F6
:100A7000012B05D03B685B6803F00303022B30D1E8
:100A80007B689B683B617B695B00032202FA03F38E
:100A9000DB433A6913403B613B68DA687B695B0082
:100AA00002FA03F33A6913433B617B683A699A603F
:100AB0007B685B683B6101227B6902FA03F3DB43DD
:100AC0003A6913403B613B685B681B0903F0010214
:100AD0007B6902FA03F33A6913433B617B683A6925
:100AE0005A603B685B6803F00303032B17D07B68F5
:100AF000DB683B617B695B00032202FA03F3DB43A3
:100B00003A6913403B613B689A687B695B0002FA73
:100B100003F33A6913433B617B683A69DA603B68E7
:100B20005B6803F00303022B23D17B69DA087B683F
:100B3000083253F822303B617B6903F007039B00C6
:100B40000F2202FA03F3DB433A6913403B613B682F
:100B50001A697B6903F007039B0002FA03F33A6901
:100B600013433B617B69DA087B680832396943F8D3
:100B700022107B681B683B617B695B00032202FAE1
:100B800003F3DB433A6913403B613B685B6803F066
:100B900003027B695B0002FA03F33A6913433B618A
:100BA0007B683A691A603B685B6803F44033002B4A
:100BB00000F08C804E4A7B699B08023352F8233048
:100BC0003B617B6903F003039B00072202FA03F3F6
:100BD000DB433A6913403B617B68B3F1904F0DD022
:100BE0007B68444A934207D07B68434A934201D1D1
:100BF000022304E0072302E0012300E000237A69D6
:100C000002F00302920093403A6913433B61384972
:100C10007B699B0802333A6941F82320374B1B68F4
:100C20003B61FB68DB433A6913403B613B685B68AF
:100C300003F48013002B03D03A69FB6813433B6134
:100C40002E4A3B6913602D4B5B683B61FB68DB43BD
:100C50003A6913403B613B685B6803F40013002B67
:100C600003D03A69FB6813433B61244A3B695360F4
:100C7000224BD3F880303B61FB68DB433A69134079
:100C80003B613B685B6803F48033002B03D03A6917
:100C9000FB6813433B61194A3B69C2F88030174B2C
:100CA000D3F884303B61FB68DB433A6913403B6116
:100CB0003B685B6803F40033002B03D03A69FB68A0
:100CC00013433B610D4A3B69C2F884307B690133B1
:100CD0007B613B681A687B6922FA03F3002B7FF47F
:100CE000B7AE00BF00BF1C37BD4680BC704700BF19
:100CF00000000140000400480008004800080058B7
:100D000080B487B000AF7860396000237B61AFE0CA
:100D100001227B6902FA03F33A6813403B613B69A5
:100D2000002B00F0A280594A7B699B08023352F8DD
:100D30002330FB607B6903F003039B00072202FA68
:100D400003F3FA681340FB607B68B3F1904F0DD05A
:100D50007B684F4A934207D07B684E4A934201D149
:100D6000022304E0072302E0012300E000237A6964
:100D700002F0030292009340FA689A4236D1464B41
:100D8000D3F880203B69DB4343491340C1F88030EE
:100D9000414BD3F884203B69DB433F491340C1F802
:100DA00084303D4B1A683B69DB433B4913400B6081
:100DB000394B5A683B69DB43374913404B607B69C9
:100DC00003F003039B00072202FA03F3FB602F4AA0
:100DD0007B699B08023352F82310FB68DA432B48E7
:100DE0007B699B080A40023340F823207B681A681D
:100DF0007B695B00032101FA03F31A437B681A60E5
:100E00007B69DA087B68083253F822107B6903F0AB
:100E100007039B000F2202FA03F3DB437A69D2082F
:100E200019407B68083243F822107B689A687B6916
:100E30005B00032101FA03F3DB431A407B689A60ED
:100E40007B685A6801217B6901FA03F3DB431A408E
:100E50007B685A607B68DA687B695B00032101FA72
:100E600003F3DB431A407B68DA607B6901337B6103
:100E70003A687B6922FA03F3002B7FF449AF00BF85
:100E800000BF1C37BD4680BC704700BF000001405A
:100E900000040048000800480008005880B485B0ED
:100EA00000AF78600B467B807B681A697B881340B3
:100EB000002B02D00123FB7301E00023FB73FB7BBB
:100EC00018461437BD4680BC704780B483B000AF6D
:100ED00078600B467B8013467B707B78002B03D0B9
:100EE0007A887B689A6102E07A887B689A6200BFA0
:100EF0000C37BD4680BC704780B582B000AF03465A
:100F0000FB80084BDA68FB881340002B06D0054AAB
:100F1000FB88D360FB881846F8F77AFC00BF0837D7
:100F2000BD4680BD0008005880B400AF044B1B686C
:100F3000034A43F48073136000BFBD4680BC704712
:100F40000004005880B582B000AF78600B46FB709B
:100F50007B68002B0CD1134B5B6903F40073B3F572
:100F6000007F0DD100F03CF80346002B08D015E0BF
:100F70000C4B5B6903F40073002B01D100F022F8E5
:100F8000094B1B69084A23F004031361FB78012B0A
:100F900001D130BF02E040BF20BF20BF0837BD46AF
:100FA00080BD00BF0004005800ED00E080B400AF39
:100FB000034B1B6803F4C0631846BD4680BC7047F2
:100FC0000004005880B400AF044B1B68034A43F48C
:100FD0008043136000BFBD4680BC704700040058CA
:100FE00080B483B000AF164B1B68154A23F48043CE
:100FF0001360144B1B68322202FB03F3124AA2FB5C
:1010000003239B0C7B6002E07B68013B7B600C4B05
:101010005B6903F40073B3F5007F02D17B68002B9A
:10102000F2D1074B5B6903F40073B3F5007F01D184
:10103000032300E0002318460C37BD4680BC7047F0
:10104000000400581801002083DE1B4380B483B0E5
:1010500000AF0346FB71104B1B6823F007030E4AD9
:1010600043F0020313600D4B1B690C4A43F0040369
:101070001361FB79012B01D130BF02E040BF20BFDB
:1010800020BF064B1B69054A23F00403136100BF10
:101090000C37BD4680BC70470004005800ED00E0EE
:1010A00080B400AF064B1B6803F48073B3F5807FF8
:1010B00001D1012300E000231846BD4680BC7047E3
:1010C0000004005880B400AF4FF0B0431B684FF0ED
:1010D000B04243F40013136000BFBD4680BC7047AC
:1010E00080B400AF4FF0B0431B684FF0B04223F420
:1010F0000013136000BFBD4680BC704780B400AFD2
:101100004FF0B0431B6803F48013B3F5801F01D187
:10111000012300E000231846BD4680BC704780B420
:1011200000AF4FF0B0431B684FF0B04243F4803340
:10113000136000BFBD4680BC704780B400AF4FF065
:10114000B0431B684FF0B04223F48033136000BFFC
:10115000BD4680BC704780B400AF4FF0B0431B6801
:1011600003F40033B3F5003F01D1012300E0002375
:101170001846BD4680BC704780B400AF4FF0B04306
:101180001B684FF0B04243F48073136000BFBD464C
:1011900080BC704780B400AF4FF0B0431B684FF085
:1011A000B04223F48073136000BFBD4680BC70471B
:1011B00080B400AF4FF0B0431B6803F48063B3F515
:1011C000806F01D1012300E000231846BD4680BC9A
:1011D000704780B483B000AF78604FF0B0435B6875
:1011E00023F0FE427B681B064FF0B04113434B6077
:1011F00000BF0C37BD4680BC704780B400AF4FF0D5
:10120000B043D3F8903003F00203022B01D1012345
:1012100000E000231846BD4680BC704780B400AF94
:101220004FF0B043D3F894304FF0B04243F0010395
:10123000C2F8943000BFBD4680BC704780B400AF98
:101240004FF0B043D3F894304FF0B04223F0010395
:10125000C2F8943000BFBD4680BC704780B400AF78
:101260004FF0B043D3F8943003F00203022B01D1C6
:10127000012300E000231846BD4680BC704780B4BF
:1012800000AF4FF0B0431B684FF0B04243F0010392
:10129000136000BFBD4680BC704780B400AF4FF004
:1012A000B0431B684FF0B04223F00103136000BF4E
:1012B000BD4680BC704780B400AF4FF0B0431B68A0
:1012C00003F00203022B01D1012300E000231846A2
:1012D000BD4680BC704780B400AF4FF0B0431B6880
:1012E00003F00803082B01D1012300E00023184676
:1012F000BD4680BC704780B400AF4FF0B0431B6860
:1013000003F0F0031846BD4680BC704780B400AFC0
:101310004FF0B043D3F8943003F470631846BD46E1
:1013200080BC704780B483B000AF78604FF0B043AA
:101330005B6823F47F427B681B024FF0B04113438C
:101340004B6000BF0C37BD4680BC704780B483B093
:1013500000AF78604FF0B0439B6823F003024FF07A
:10136000B0417B6813438B6000BF0C37BD4680BC27
:10137000704780B400AF4FF0B0439B6803F00C039C
:101380001846BD4680BC704780B483B000AF78601B
:101390004FF0B0439B6823F0F0024FF0B0417B6800
:1013A00013438B6000BF0C37BD4680BC704780B4D0
:1013B00083B000AF78604FF0B043D3F8083123F02A
:1013C0000F027B681B094FF0B0411343C1F808318D
:1013D00000BF0C37BD4680BC704780B483B000AFFF
:1013E00078604FF0B0439B6823F4E0624FF0B04167
:1013F0007B6813438B6000BF0C37BD4680BC7047D1
:1014000080B483B000AF78604FF0B0439B6823F4A2
:1014100060524FF0B0417B6813438B6000BF0C37C4
:10142000BD4680BC704780B400AF4FF0B0439B68AE
:1014300003F0F0031846BD4680BC704780B400AF8F
:101440004FF0B043D3F808311B0103F0F003184606
:10145000BD4680BC704780B400AF4FF0B0439B687E
:1014600003F4E0631846BD4680BC704780B400AF0B
:101470004FF0B0439B6803F460531846BD4680BCF0
:10148000704780B400AF4FF0B0431B684FF0B042DC
:1014900043F08073136000BFBD4680BC704780B4CA
:1014A00000AF4FF0B0431B684FF0B04223F08073A1
:1014B000136000BFBD4680BC704780B400AF4FF0E2
:1014C000B0431B6803F00073B3F1007F01D1012327
:1014D00000E000231846BD4680BC704780B400AFD2
:1014E0004FF0B043DB681B0A03F07F031846BD468C
:1014F00080BC704780B400AF4FF0B043DB6803F0AE
:1015000060431846BD4680BC704780B400AF4FF0C2
:10151000B043DB6803F070031846BD4680BC7047DB
:1015200080B400AF4FF0B043DB6803F0030318460C
:10153000BD4680BC704780B400AF4FF0B0439B689D
:1015400003F48033B3F5803F01D1012300E0002391
:101550001846BD4680BC704780B400AF4FF0B04322
:10156000D3F8083103F48033B3F5803F01D1012370
:1015700000E000231846BD4680BC704780B400AF31
:101580004FF0B0439B6803F40033B3F5003F01D143
:10159000012300E000231846BD4680BC704780B49C
:1015A00000AF4FF0B0439B6803F48023B3F5802F66
:1015B00001D1012300E000231846BD4680BC7047DE
:1015C00080B588B000AF78607B68002B01D1012323
:1015D0008BE3FFF7CEFEF861FFF7A2FFB8617B68EF
:1015E0001B6803F02003002B00F0C980FB69002B6F
:1015F00005D0FB690C2B7BD1BB69012B78D1FFF7A0
:101600005AFE0346002B05D07B681B6A002B01D1D4
:1016100001236AE37B689A6A4FF0B0431B6803F0CA
:101620000803002B05D04FF0B0431B6803F0F00314
:1016300006E04FF0B043D3F894301B0903F0F003F9
:10164000934222D27B689B6A184600F051FD034604
:10165000002B01D0012348E34FF0B0431B684FF04B
:10166000B04243F0080313604FF0B0431B6823F00F
:10167000F0027B689B6A4FF0B04113430B607B68BC
:101680005B6A1846FFF74EFE21E04FF0B0431B683F
:101690004FF0B04243F0080313604FF0B0431B68B3
:1016A00023F0F0027B689B6A4FF0B04113430B605C
:1016B0007B685B6A1846FFF735FE7B689B6A1846B5
:1016C00000F016FD0346002B01D001230DE300F0CE
:1016D000D7FC0346A14A1360A14B1B681846F7F7D5
:1016E00037F80346FB74FB7C002B47D0FB7CFCE205
:1016F0007B681B6A002B2CD0FFF7C1FDF7F732F88F
:10170000786108E0F7F72EF802467B69D31A022BBE
:1017100001D90323E9E2FFF7CEFD0346002BF1D008
:101720004FF0B0431B684FF0B04243F00803136022
:101730004FF0B0431B6823F0F0027B689B6A4FF0C8
:10174000B04113430B607B685B6A1846FFF7EAFD04
:1017500015E0FFF7A2FDF7F705F8786108E0F7F765
:1017600001F802467B69D31A022B01D90323BCE29C
:10177000FFF7A1FD0346002BF1D100E000BF7B681D
:101780001B6803F00103002B5FD0FB69082B05D019
:10179000FB690C2B0DD1BB69032B0AD1FFF7DBFCD6
:1017A0000346002B50D07B685B68002B4CD1012393
:1017B0009BE24FF0B0431B6823F480127B689B6868
:1017C0004FF0B04113430B607B685B68B3F5803F1B
:1017D00002D1FFF7A4FC0DE07B685B68B3F5041F42
:1017E00004D1FFF76FFCFFF79AFC03E0FFF7A5FCBD
:1017F000FFF776FC7B685B68002B12D0F6F7B2FF30
:10180000786108E0F6F7AEFF02467B69D31A642BD5
:1018100001D9032369E2FFF79EFC0346002BF1D0B8
:1018200013E0F6F79FFF786108E0F6F79BFF0246AA
:101830007B69D31A642B01D9032356E2FFF78BFC93
:101840000346002BF1D100E000BF7B681B6803F06A
:101850000203002B4BD0FB69042B05D0FB690C2B3A
:1018600013D1BB69022B10D1FFF7A2FC0346002B5A
:1018700005D07B681B69002B01D1012335E27B6811
:101880005B691846FFF7A5FC31E07B681B69002BFC
:1018900019D0FFF771FCF6F765FF786108E0F6F7FD
:1018A00061FF02467B69D31A022B01D903231CE294
:1018B000FFF77EFC0346002BF1D07B685B6918467E
:1018C000FFF787FC13E0FFF765FCF6F74BFF786145
:1018D00008E0F6F747FF02467B69D31A022B01D9CD
:1018E000032302E2FFF764FC0346002BF1D17B687F
:1018F0001B6803F00803002B6FD07B689B69002BEB
:1019000057D04FF0B043D3F89430FB607B68DA696E
:10191000FB6803F010039A4236D0FB6803F0020321
:10192000002B06D0FB6803F00103002B01D101233B
:10193000DBE1FB6803F00103002B18D0FFF77EFC0E
:10194000F6F710FF78610DE0F6F70CFF02467B69B1
:10195000D31A112B06D90323C7E100BF18010020B9
:101960001C010020FFF77AFC0346002BECD14FF05E
:10197000B043D3F8943023F010027B68DB694FF05A
:10198000B0411343C1F89430FFF748FCF6F7EAFE84
:10199000786108E0F6F7E6FE02467B69D31A112B60
:1019A00001D90323A1E1FFF759FC0346002BF1D035
:1019B00013E0FFF743FCF6F7D5FE786108E0F6F791
:1019C000D1FE02467B69D31A112B01D903238CE186
:1019D000FFF744FC0346002BF1D17B681B6803F042
:1019E0000403002B00F0D880FFF75AFB0346002BBE
:1019F00013D1FFF799FAF6F7B5FE786108E0F6F72C
:101A0000B1FE02467B69D31A022B01D903236CE194
:101A1000FFF746FB0346002BF1D07B68DB68002B09
:101A20007BD07B68DB68852B03D07B68DB68052B6C
:101A300009D14FF0B043D3F890304FF0B04243F0AB
:101A40000403C2F89030F6F78DFE78614FF0B04392
:101A5000D3F890304FF0B04243F00103C2F8903019
:101A60000AE0F6F77FFE02467B69D31A41F288321C
:101A7000934201D9032338E1FFF7BFFB0346002B54
:101A8000EFD07B68DB68812B03D07B68DB68852B1C
:101A900021D1F6F767FE78614FF0B043D3F890306C
:101AA0004FF0B04243F08003C2F890300AE0F6F7FE
:101AB00059FE02467B69D31A41F28832934201D91A
:101AC000032312E14FF0B043D3F8903003F40063E6
:101AD000002BECD060E0F6F745FE78614FF0B043A4
:101AE000D3F890304FF0B04223F08003C2F890302A
:101AF0000AE0F6F737FE02467B69D31A41F28832D4
:101B0000934201D90323F0E04FF0B043D3F8903073
:101B100003F40063002BECD13EE0F6F723FE78617E
:101B20004FF0B043D3F890304FF0B04223F0800331
:101B3000C2F890300AE0F6F715FE02467B69D31A28
:101B400041F28832934201D90323CEE04FF0B043F3
:101B5000D3F8903003F40063002BECD1F6F702FECB
:101B600078614FF0B043D3F890304FF0B04223F09B
:101B70000103C2F890300AE0F6F7F4FD02467B69F3
:101B8000D31A41F28832934201D90323ADE0FFF723
:101B900034FB0346002BEFD17B68DB6A002B00F09F
:101BA000A380FB690C2B76D07B68DB6A022B4BD1C0
:101BB000FFF775FCF6F7D6FD786108E0F6F7D2FD81
:101BC00002467B69D31A0A2B01D903238DE0FFF764
:101BD00074FC0346002BF1D14FF0B043DA68454B5B
:101BE00013407A68116B7A68526B11437A68926B72
:101BF000120211437A68D26B11437A68126C114356
:101C00007A68526C0A434FF0B0411343CB60FFF740
